:1000000008100300795B0200355A0200395A0200D9
:10001000915B0200955B0200995B0200000000000A
:100020000000000000000000000000009D5B0200D6
:10003000A15B0200000000008DCD0000270402003B
:100040000000000000000000A55B0200ED59020066
:10005000891B0100000000000000000000000000FB
:100060000000000000000000815B020000000000B2
:100070000000000000000000ED2D01000000000065
:10008000D32E0100152F01004158020041580200F3
:100090009157020000000000000000000000000076
:1000A00070B500224FF41261DFF8140B02F002F970
:1000B000DFF8104B0022102104F11C0002F0FAF8C6
:1000C000DFF8045B0022182105F10C0002F0F2F8C1
:1000D0000022082104F12C0002F0ECF80022082193
:1000E00004F1340002F0E6F80020E063206460646C
:1000F000A0646862A862E862DFF8D06AB063F06367
:10010000E0642863306470646863A863E863012076
:1001100028640020B064F0644FF0FF306864A86485
:100120000020E864306520657065F06530667066B3
:10013000B066F06202462C21304602F0BBF842F273
:1001400010707081B081002070600220308100202A
:10015000306002460C21204602F0ACF8DFF8700A4D
:100160006060DFF8700A2060012020720020287093
:1001700028656880A880E8806065F0662881A065B1
:1001800030636865A8656066A066E0667067306782
:1001900068662866E86501202867E866A86600208A
:1001A000E867A86768670620B0860020A082F0672D
:1001B000B0672067DFF8200AE06500202066012094
:1001C000E082962068810620F0860C2020830020A3
:1001D000B06502464021DFF85C0D02F06BF80022AA
:1001E000062104F10C00BDE8704002F063B810B5C0
:1001F00084B0DFF8D0490C22214600A802F098F81C
:10020000FFF74EFF0C2200A9204602F091F81FBD17
:100210002DE9F0472DED0C8B90B00024254600A869
:1002200021460A460B460EC0302102F0B9F89FED78
:100230009B8ADFF8906996ED1B0AD6ED140AC6ED8D
:100240001B0ADFF8887997ED149A86ED149ADFF887
:10025000788998ED131AB8EE411ADFED911AC1EEC4
:10026000819AC7ED149AD8F84420D8F83490A9EBB5
:100270000200FA30FA21B0FBF1F1FA2303FB11007E
:1002800080B2002800F0FE834C2880F28180D8F8EC
:10029000401001297CD0D7F84CA0BAF1040F21D32B
:1002A000F4EE490AF1EE10FA1CD5B4EE699AF1EEBB
:1002B00010FA17D59FED7B1A20EE811AB4EE691A59
:1002C000F1EE10FA0ED59FEDDB1AF4EE419AF1EE45
:1002D00010FA07DB87ED149AC6ED140A86ED1B0AA7
:1002E00000F009BC97ED0EAA87ED0FAAD7ED10AA72
:1002F000C7ED11AA014600EE101AB8EE400AD8ED7B
:100300000B8AC8EE800A98ED0C1A81EE001A21467D
:10031000B963396420E0521C92B2FA2A00D1224615
:10032000DFF89C3803EB8203D3ED231A71EEE01A59
:10033000D3F8743402EE103A32EE412AD7ED0E2A89
:1003400041EEA12AC7ED0E2AD7ED101A42EE021A8D
:10035000C7ED101A491C89B28142DCDBD7ED0E0AC9
:1003600080EE80BA87ED0EBAD7ED100A80EE80CA13
:1003700087ED10CAD6ED1ABA98ED150AD8ED160A0F
:1003800070EE60CAC6ED1ACA00F092FF012802D1D1
:100390002046386376E3BAF1000F0BD1388E05287A
:1003A00002DB054620463886788E052802DB451993
:1003B000204678861AFA85F0002824D1B6EE00DAB5
:1003C0003CEE2A0A20EE0D0ADFED9B0AB4EE600A2D
:1003D000F1EE10FA11D43BEE0A0A20EE0D0ADFED21
:1003E000970AB4EE600AF1EE10FA06D4B3EE040AEE
:1003F000F4EE40CAF1EE10FA05D5388E401C38866E
:10040000C8F848903EE3388E002802D045192046AF
:1004100038861AFA85F0002815D1B7EE000AF4EEF6
:10042000409AF1EE10FA00F12D839FED850AF4EE6B
:10043000409AF1EE10FA03DB788E401C788621E3B7
:100440002046788603E0788E45192046788628462F
:1004500080B200F0C3FF012808D187ED149AC7EDE0
:1004600010AAC6ED1ABA87ED0EAA0BE39FED750A26
:10047000F4EE409AF1EE10FA02DBDFF8180C386562
:1004800020463886BAF1000F0ED1386D786586EDBA
:1004900013BAC6ED19CA00F0A5FE3CE0000000004A
:1004A00000007A446666E63FB6EE00DA00F09AFE97
:1004B000012816D197ED140AF0EE000A20EE200A6A
:1004C00087ED140A6BEE0D0AC7ED0E0A2CEE0D1A1D
:1004D00087ED101AC7ED0F0A87ED111A86ED140A81
:1004E0006D1C97ED140AD6ED140A30EE200A20EEAA
:1004F0000D0A87ED150A97ED0E0AD7ED0F0A30EEBB
:10050000200A20EE0D0A86ED130A3BEEAC0A20EE1F
:100510000D0A86ED190A98F80100012840F0A7821B
:10052000D8F80C00009000A8D8F810104160D8F856
:1005300014108160214617E000AB03EB820393EDBA
:10054000010A50F822C000EE90CAB4EE600AF1EE43
:1005500010FA05D500EB820C8CED000AC3ED010A00
:10056000521C022AE8DB491C022901DA2246F8E77C
:100570009DED000AB5EE400AF1EE10FA2AD5B5EE6F
:10058000400AF1EE10FA01DCB1EE400AD0ED020AA9
:1005900030EE800A80ED020A9DED000AB5EE400AB9
:1005A000F1EE10FA01DCB1EE400AD0ED010A30EEB6
:1005B000800A80ED010A9DED000AB5EE400AF1EED9
:1005C00010FA01DCB1EE400ADDED000A30EE800ADF
:1005D0008DED000A90ED010AD0ED020A30EEC01A4E
:1005E000DDED000A30EE600AB4EE401AF1EE10FACA
:1005F00005D5F0EE410AB0EE401AB0EE600AD6ED35
:100600000B0AC6ED0C0A31EE400A80EE010A9FED9E
:100610000E1A20EE010A86ED0B0A706BB063F4EE41
:10062000400AF1EE10FA11D570EE600AC6ED0D0A1F
:1006300010E000BF01004040000016430000A0424F
:10064000666616400100A0400000C84270EEC00A75
:10065000C6ED0D0A386F796F081800EBD0704010A6
:1006600002EE100A86ED0F2AC6ED108AD7ED100AA9
:10067000C6ED110AD7ED141ADFF8300CC0EDC41A1C
:1006800096ED121A31EE611AD6ED122A72EEE12AB7
:1006900021EE221A00F5447181ED011AC6ED121AFD
:1006A000D7ED1B1AC1ED021AD8F81810039103A94F
:1006B000C1ED011AC1ED020AC1ED038AC1ED041AB0
:1006C000C1ED058AC1ED061AB8EEC22A81ED072AEE
:1006D000C1ED081A81ED090AC1ED0A1A81ED0B1A64
:1006E000DDED032A9FEDD03A62EE832A9FEDCF3AEB
:1006F00041EE832A9FEDCE3A20EE833ADFEDCD3AEC
:1007000008EEA33ADFEDCC3A61EEA33A9FEDCB4A77
:1007100048EE843A9FEDCA4A21EE844ADFEDC94A89
:1007200002EE244ADFEDC84A61EEA44A9FEDC75AA3
:1007300040EE054A9FEDC65A21EE855ADFEDC55AB7
:1007400001EE255AF8EE085AF4EE652AF1EE10FA99
:1007500000F18D81DFEDC05AB4EE653AF1EE10FA8A
:1007600000F18581DFEDBD5AF4EE653AF1EE10FA45
:1007700000F17D81DFEDBA5AB4EE654AF1EE10FA70
:1007800000F175819FEDDF6AF4EE464AF1EE10FA52
:1007900000F16D819FEDDC6AB4EE465AF1EE10FA7D
:1007A00000F16581DFEDD96AF4EE662AF1EE10FA08
:1007B000C0F25D81DFEDD62AB4EE623AF1EE10FAB6
:1007C000C0F25581F4EE653AF1EE10FAC0F24F81B5
:1007D000B4EE464AF1EE10FAC0F24981F4EE654AF1
:1007E000F1EE10FAC0F24381DFEDCA2AB4EE625A8C
:1007F000F1EE10FAC0F23B81DFEDC72A9DED033A1E
:10080000B4EE623AF1EE10FA01D5CDED032ADDED3A
:10081000032A9FEDD83AF4EE432AF1EE10FA02DBF8
:10082000DFF8AC2B0392DFEDD42AF4EE621AF1EE7E
:1008300010FA01D5C1ED012A9FEDB83ADFEDB83AC3
:1008400091ED014AB4EE634AF1EE10FA01DB81ED5D
:10085000013A9FEDB44AF4EE440AF1EE10FA01D5E4
:1008600081ED024AD1ED020A9FEDAF4AF4EE440A4F
:10087000F1EE10FA02DBDFF85C2B8A60DFEDBF0AD5
:10088000F4EE608AF1EE10FA01D5C1ED030A9FED96
:10089000BC4AD1ED034AF4EE444AF1EE10FA02DB11
:1008A000DFF8342BCA60F4EE621AF1EE10FA01D5CB
:1008B000C1ED042AD1ED044AF4EE634AF1EE10FAD8
:1008C00001DB81ED043AF4EE608AF1EE10FA01D515
:1008D000C1ED050AD1ED050AF4EE440AF1EE10FA75
:1008E00002DBDFF8F42A4A61F4EE621AF1EE10FA44
:1008F00001D5C1ED062AD1ED060AF4EE630AF1EE48
:1009000010FA01DB81ED063AF1EE000AB4EE602A3E
:10091000F1EE10FA02D54FF08142CA61D1ED070A1B
:100920009FEDA12AF4EE420AF1EE10FA02DBDFF8A5
:100930002C2CCA61F4EE621AF1EE10FA01D5C1ED69
:10094000082AD1ED080AF4EE630AF1EE10FA01DB91
:1009500081ED083ADFED950AB4EE600AF1EE10FA87
:1009600001D5C1ED090A91ED090ADFED910AB4EE56
:10097000600AF1EE10FA02DBDFF8E42B4A62F4EED3
:10098000621AF1EE10FA01D5C1ED0A2A91ED0A0AB8
:10099000B4EE630AF1EE10FA01DB81ED0A3AB5EE2E
:1009A000401AF1EE10FA01D52246CA6291ED0B0A07
:1009B000DFED800AB4EE600AF1EE10FA02DBDFF838
:1009C000A42BCA62214612E01B1FD3ED000A92ED50
:1009D000031AF4EE410AF1EE10FA01D59FED760A02
:1009E000B8EEC00AD2ED020A00EE208A491C312975
:1009F00038DA9FED720A0B011A18D2F804C0BCF164
:100A0000010F0DF10C0C1B580CEB8303DCD11B1FE9
:100A1000D3ED000A92ED031AF4EE410AF1EE10FA5A
:100A2000DEDB9FED650ADBE7168733BDB0568DBD73
:100A300003275BB9E23C9CB9983115BEBF49D3B9D5
:100A40007061FDBD55C128BC36CB05BE3D7FDABB0C
:100A5000DDED0ABEE4BE353E6666A6BF3333F3BFA6
:100A6000CDCC4CBFB5EE408AF1EE10FA0ADC97ED22
:100A7000150A284680B200F0B1F800F057F8044695
:100A8000C8F84890C8F844900020C8F84C00C8F84E
:100A90002C00C8F83000C8F840000246102106F1CA
:100AA0001C0001F007FC00220C2108F10C0001F0F1
:100AB0007BFC4948F06500203066F88800281AD190
:100AC000F86F00280CD0B86C3969401AB98EB0EBB9
:100AD000510F02DB002038810DE0012038810AE04F
:100AE000388E798E11FA80F0032802DB01203881DC
:100AF00001E002203881204610B0BDEC0C8BBDE82F
:100B0000F08700BFCDCC8CBF333333BFCDCC0CC00E
:100B10009A9919BFCDCC4CBE5017C93F15E6684015
:100B200016E668407D90A341A2F2924438B50025B4
:100B3000DFF8BC4B0120E06700F0F0FC2060E06CC7
:100B4000A18E884214D3A06C2061A08DA080E08D7E
:100B5000E080A06DA061E06DE061206E2062606EBB
:100B60006062A06EA0620120A0672846E0670125B0
:100B7000284632BDC9AC4542A9F56E3EBA9F17441E
:100B80003564EC441148016981640021C16441600D
:100B9000022101810021C162016A0166816A8166C8
:100BA0000021C16770470000010058427B4D4F3D56
:100BB00047FFC742BEBA984101000000FFFFFFFF98
:100BC00030460300D03A0300D0390300503A030006
:100BD00000002F430000704200007A442DE9F84FD6
:100BE0002DED048B82B08346F0EE400A00239E4632
:100BF0001846DFF8FC4AE56C05F10F0101F00F0122
:100C0000EA1D02F007020092CA4A02EB8106C6ED15
:100C1000000ABBF1000F15D0064611E04F1EBF1BA6
:100C200010374FEAE70C07EB1C7C4FEA2C1CB7EBA4
:100C30000C1703D402EB8707C7ED000A761C36B207
:100C40005E45EBDB102D02D2294609B200E00F21F0
:100C50009FEDB68A9FEDB51ADFEDB51A06461BE08B
:100C600052F8217000EE107AB5EE400AF1EE10FA5B
:100C700010DD38EE008AB4EE401AF1EE10FA01D51C
:100C8000B0EE401AB4EE610AF1EE10FA01D5F0EEC2
:100C9000401A761C491E09B20029E1D536B2314608
:100CA00003290BDB38EE410A30EE610A891E01EEA2
:100CB000101AB8EEC11A80EE018A07E0012905DB9F
:100CC00000EE106AB8EEC00A88EE008AB5EE408ADF
:100CD000F1EE10FA01D0002E01D1B0EE608A84ED61
:100CE000168A9FED950AB4EE408AF1EE10FA02D50D
:100CF000B0EE408A08E09FED910AB4EE408AF1EE32
:100D000010FA01DBB1EE028AB0EE040AB4EE408ABA
:100D1000F1EE10FA08D494ED1B0AF0EE080AB4EED6
:100D2000600AF1EE10FA02D50321A18501E0042149
:100D3000A185A66C06F00708DFF8BC7908EB070C64
:100D4000A18D8CF8B818BBF1000F0AD0721E02F00A
:100D50000702D21906F00709B94499F8B89882F841
:100D6000B89808220EE0B9F1040F00D1401CA8F198
:100D700001080FFA88F8B8F1000F01D508F108084A
:100D8000521E12B2012A16DB0FFA88F808EB070987
:100D900099F9B898B9F1030F02D10EF1010E03E0F1
:100DA000B9F1040F00D15B1C062AE0DBB9F1030F97
:100DB000D9D1401EDBE7E28D9BB21FFA8EFE734550
:100DC00007D39E4502D20420E0850DE000B2002842
:100DD00002D50320E08507E0012802DB0420E0853E
:100DE00002E09CF9B808E085B4F82E80B8F1040F51
:100DF00001D1184600E07046424509D0002020810C
:100E0000E088002820D1042D1ED3012020811BE082
:100E100013FA8EF2012A15DB052A10DB00EE102AE8
:100E2000B8EEC00AF6EE080A20EE200A00EE900A9C
:100E3000F8EE600AF4EE400AF1EE10FA02D5012055
:100E4000208101E002202081DFF8B09849B2B0EEA5
:100E5000480A484600F020F9DFED8D0AB4EE600A3A
:100E6000F1EE10FA01D5B0EE600A84ED170A58468B
:100E700000F1010A00EE90AAF8EEE08AD4ED180A1B
:100E800048EE800AC4ED180A9FEDCB9A20EE080ABE
:100E900020EE090A009907EB810101F65C0181ED62
:100EA000000ABBF1000F16D0002212E00099491E83
:100EB000891A08318B1001EB5373DB10B1EBC301BE
:100EC00005D407EB810101F65C0181ED000A521C9B
:100ED00012B28242EADB082D02D2284600B203E0B9
:100EE000072001E0401E00B20028FBD584ED190A5E
:100EF000414649B2484600F047F968EE090AB7EEA4
:100F0000001AC1EE200A20EE800AD4ED1A0A48EE3B
:100F1000800AC4ED1A0A0AEB0600A0640AEB050079
:100F2000E06402B0BDEC048BBDE8F18F000000006E
:100F30000000C842A8A903006666A63F01009040D1
:100F400049B2032944D1DFED9D0AB4EE600AF1EE07
:100F500010FA01DBB0EE600A9FED991ADFED990AF5
:100F600040EE010A90ED011A9FED970AB4EE401A87
:100F7000F1EE10FA43DADFED951AB4EE611AF1EEF4
:100F800010FA74DBB4EE401AF1EE10FA6FD59FED53
:100F9000900A31EE000ADFED8F1A60EE211A9FED04
:100FA0008E0A9FED8E2A01EE002A22EE200A20EE04
:100FB000210A9FEDB72ADFEDB72A41EE022A62EE41
:100FC000A00AB7EE001A31EE611A00EE810A56E06F
:100FD000DFED830A60EE200A60EE800A9FEDAE1A14
:100FE00040EE410A9FEDAD0A70EE800A90ED011AC5
:100FF0009FED750AB4EE401AF1EE10FA0ADB90ED9F
:10100000010A9FED751ADFED751A40EE011A21EE07
:10101000A00A34E0DFED6D1AB4EE611AF1EE10FAB9
:1010200025DBB4EE401AF1EE10FA20D59FED680AE8
:1010300031EE000ADFED671A60EE211A9FED660AB5
:101040009FED662A01EE002A22EE200A20EE210AF8
:101050009FED8F2ADFED8F2A41EE022A62EEA00A71
:10106000B7EE001A31EE611A00EE810A07E090ED4A
:10107000010A20EE800ADFED8A0A20EE200A007ABB
:10108000022803D1DFEDCA0A20EE200A70470000D3
:10109000CDCC4C3E0000A04010B52DED028BB0EE43
:1010A000408A0C46DFED7F8A49B2FFF749FF64B200
:1010B000042C31D1DFED7C0AB4EE608AF1EE10FA37
:1010C00016DBB1EE021AB4EE418AF1EE10FA0FD53A
:1010D000DFEDB80A78EE200AB1EE041A60EE810A5C
:1010E000FCEEE00A10EE900AC01D08EE900A3DE00A
:1010F000B4EE608AF1EE10FA03D5072008EE900AEC
:1011000034E0F1EE020AB4EE608AF1EE10FA2DDB63
:10111000122008EE900A29E0F7EE080AB4EE608A81
:10112000F1EE10FA11DBDFEDA40AB4EE608AF1EE05
:1011300010FA0AD5FFEE080A78EE200AB1EE041A7A
:1011400060EE810AFCEEE08A10E0F7EE080AB4EEE9
:10115000608AF1EE10FA09D4DFED970AB4EE608AE6
:10116000F1EE10FA02DB062008EE900ADFF8580DC7
:1011700018EE901A00EB8100D0ED000A20EE200A54
:10118000BDEC028B10BD0000F0EE0C0A49B2042940
:1011900004D19FED8A1A40EE010A03E09FED881A00
:1011A00040EE010A9FEDDB0A20EE800AD0ED000A36
:1011B00020EE200A70470000000070429A99194002
:1011C0006ADEF13D8638163F00002A4300001643D0
:1011D000000016C3CDCC4C3D4260E53A6666263F22
:1011E0002575C23E0020DFF8081591ED140AF7EED0
:1011F000040AB4EE600AF1EE10FA47DADFF8CC2CFC
:10120000D288042A42DAD1ED150A9FED6E1A60EEFB
:10121000810AB4EE600AF1EE10FA03D5022A01DB6E
:10122000012012E0DFF8D41491ED0A0ADFED660A1E
:10123000B4EE600AF1EE10FA07DBDFED640AB4EEFB
:10124000600AF1EE10FA00D5012001281ED1DFF866
:10125000AC1491ED170AD1ED180A70EEC00A9FED9B
:10126000AE1AF4EE410AF1EE10FA07DBF7EE080AC7
:10127000B4EE600AF1EE10FA00D50020DFEDB30AFB
:10128000B4EE600AF1EE10FA00D5002070470000BD
:1012900052491D3BB81E053F7593E83F24975340C4
:1012A000C1C0C03B00000000666606400830030075
:1012B0000021DFF83C24D38D032B1BDA92ED140AB6
:1012C000DFEDA30AB4EE600AF1EE10FA12DB92ED44
:1012D0000E0AF2EE040AB4EE600AF1EE10FA09D535
:1012E00092ED100ADFED9B0AB4EE600AF1EE10FAFF
:1012F00000D5012192ED100AF6EE000A92ED111AC6
:1013000030EE011A21EE201AF3EE0E1AB4EE611A35
:10131000F1EE10FA1CD492ED0E1AD2ED0F1A71EE06
:10132000211A61EEA01AB2EE042AF4EE421AF1EE8E
:1013300010FA0DD4F3EE041AB4EE610AF1EE10FACD
:1013400006D4B1EE040AB4EE401AF1EE10FA00D55C
:10135000012192ED140A9FED801AB4EE410AF1EEDC
:1013600010FA23DBDFF8942392ED090A92ED0A1AB2
:1013700080EE010A9FEDA51AB4EE410AF1EE10FAD3
:1013800014DB00EE100AB8EE400A20EE200AD2ED7F
:10139000070AF4EE400AF1EE10FA07D5D2ED080A7A
:1013A000F4EE400AF1EE10FA00D50121084670472C
:1013B0003333733F666606C09A993940CDCC4C3EB4
:1013C000CDCCCC3D3333333F010020420000C84236
:1013D000C8AC4542A1F292443464EC440021C44AB2
:1013E000D36C13FA80F0022816D392ED140ADFEDC5
:1013F000880AB4EE600AF1EE10FA0DDB92ED110AE4
:10140000D2ED100A80EE200ADFED820AB4EE600A07
:10141000F1EE10FA00DB0121022818D39FED7E0ABD
:10142000D2ED110A92ED101AC0EE810AF4EE400AD4
:10143000F1EE10FA0BDBD2ED0F0A92ED0E1AC0EEB0
:10144000810AF4EE400AF1EE10FA00DB01210028D7
:101450000ED0AA4890ED190ADFED9E0A20EE200A70
:10146000D0ED1A0AF4EE400AF1EE10FA00D501218F
:1014700092ED140ADFED980AB4EE600AF1EE10FA6C
:1014800008DA92ED150ADFED950AB4EE600AF1EE86
:1014900010FA1ADB92ED100ADFED910AB4EE600A41
:1014A000F1EE10FA0DD492ED0E0ADFED8E0AB4EED5
:1014B000600AF1EE10FA04D4DFF8100AC08802289E
:1014C00003DBD08D032800DB01218C4890ED130A4B
:1014D000DFED830AB4EE600AF1EE10FA08D492ED63
:1014E0001B0AF1EE040AB4EE600AF1EE10FA0ED512
:1014F000106F526F101800EE100ABAEEEF0ADFED0F
:101500007A0AB4EE600AF1EE10FA00DB0121084617
:10151000704700000AD7A33B0100C03F0020744978
:101520008A6C12F10A0F0FD29FED700AD1ED180AE2
:10153000F4EE400AF1EE10FA06DAD1ED1A0AF4EEF2
:10154000400AF1EE10FA00DB0120704785EB113FF5
:1015500001000040000020420100404000005842CD
:1015600046FFC742BDBA984110B401460020634A05
:10157000614BD3F8144900EE104AD1ED000AB4EEE5
:10158000600AF1EE10FA08D1147B641C1473E4B203
:10159000FE2C04DB3224147301E00446147303F6BA
:1015A000141393ED010AD1ED010AB4EE600AF1EED5
:1015B00010FA08D1547B641C5473E4B2FE2C04DB93
:1015C0003224547301E00446547393ED020AD1EDC2
:1015D000020AB4EE600AF1EE10FA08D1917B491CC0
:1015E0009173C9B2FE2904DB3221917301E00146F7
:1015F0009173117B322905DA517B322902DA917B12
:10160000322900DB012010BC704700003433333F27
:10161000010060400100A04001007041014600202F
:1016200091ED000AB5EE400AF1EE10FA01DCB1EEE0
:10163000400A324ADFED2F0AB4EE600AF1EE10FAEA
:1016400008DBD37B5B1CD373DBB2FE2B04DB3223C2
:10165000D37301E00346D37391ED010AB5EE400A5E
:10166000F1EE10FA01DCB1EE400AB4EE600AF1EEE0
:1016700010FA08DB137C5B1C1374DBB2FE2B04DB5B
:101680003223137401E00346137491ED020AB5EEA0
:10169000400AF1EE10FA01DCB1EE400AB4EE600A45
:1016A000F1EE10FA08DB517C491C5174C9B2FE29D5
:1016B00004DB3221517401E001465174D17B32299F
:1016C00005DA117C322902DA517C322900DB012053
:1016D000704700009A99993E0100904001008040B7
:1016E0000000C8430000164301005C428096184B7E
:1016F000503A030035336B4130460300D03A0300C3
:101700002DE9F24F2DED048B84B004469FEDE58A60
:10171000DFEDE48A9FEDE39ADFF8405BE888ADF8FF
:101720000800A888ADF8020028898DF8000000277D
:101730003E462046FFF718FF01902046FFF76EFF58
:101740008246DFF888873046C8F85400C8F8580049
:10175000D8F86800DFF8089BD9F8141900EE101AC1
:10176000D4ED000A30EEC01A01EE900AF8EEE11A4C
:1017700021EE211AB5EE401AF1EE10FA1ED598EDC1
:101780001D1A70EE411AF5EE401AF1EE10FA01DC66
:1017900071EE401A9FEDC41AF4EE411AF1EE10FA00
:1017A00007DB296F491C2967D8F85C10491CC8F869
:1017B0005C1088ED1D0A4042C8F8680009F6141054
:1017C00090ED010AD8F86C1094ED011A31EE401A30
:1017D00001EE901AF8EEE11A21EE211AB5EE401A48
:1017E000F1EE10FA1ED598ED1E1A70EE411AF5EEC4
:1017F000401AF1EE10FA01DC71EE401A9FEDAA1AC0
:10180000F4EE411AF1EE10FA07DB2A6F521C2A6738
:10181000D8F86020521CC8F8602088ED1E0A4942A2
:10182000C8F86C1090ED020AD8F8700094ED021A16
:1018300031EE401A01EE900AF8EEE11A21EE211A7B
:10184000B5EE401AF1EE10FA1ED598ED1F1A70EEA3
:10185000411AF5EE401AF1EE10FA01DC71EE401A71
:101860009FED911AF4EE411AF1EE10FA07DB296FA1
:10187000491C2967D8F86410491CC8F8641088ED21
:101880001F0A4042C8F8700098F80000052809D1E6
:101890000120C8F84000304688F80000A8F802008F
:1018A000A8F80400D8F84C0008990818C8F84C00AB
:1018B000D8F83400D8F84410884202D10120C8F882
:1018C0004000D8F8380000EB400109EB810B0BF623
:1018D000C000C0ED000A61684160A168816008999C
:1018E000204600F029FA68610198012802D0BAF177
:1018F000010F32D19FED6B0ADBF8C00800EE900AB1
:1019000060EEA00ADBF8C40801EE100A21EE011A0D
:10191000DBF8C80801EE900A61EEA11ADFF844096D
:10192000017B322904DAC17B322901DA30EE800AE8
:10193000417B322904DA017C322901DA30EE010AD6
:10194000817B322904DA407C322801DA30EE210A28
:1019500000F094FCF0EE409A37E00BF50C60D0ED0F
:10196000020A90ED011ADBF8C00800EE100A20EE22
:10197000000A01EE010A00EEA00A00F07FFCF0EE82
:10198000409AD4ED010A94ED000A20EE000A00EE20
:10199000A00A00F073FCB0EE408AD4ED020A94ED88
:1019A000010A20EE000A00EEA00A00F067FCF0EE4B
:1019B000408AD4ED020A94ED000A20EE000A00EEFF
:1019C000A00A00F05BFCB0EE409AD8F83C0000287A
:1019D0002ED130460CE009EB8001C1ED159A09EBE0
:1019E000800282ED008AC1ED078A81ED0E9A401CCB
:1019F0000728F0DBB1EE0C0A69EE800AC8ED090A8F
:101A0000D8F80C00C8F81800D8F81000C8F81C0066
:101A1000D8F81400C8F8200068EE000AC8ED030AE0
:101A200068EE800AC8ED040A29EE000A88ED050A6E
:101A3000D8F8380009EB800191ED150A39EEC00A9B
:101A4000D8ED090A30EE200A88ED090AC1ED159A91
:101A5000D8F8340009EB800080ED230AD8ED0B0A9A
:101A600070EE800AC8ED0B0AD8F80C20C8F81820D0
:101A7000D8F81020C8F81C20D8F81420C8F8202066
:101A8000D8F8382009EB820282ED008AC1ED078A7E
:101A900081ED0E9A3246DFED030A9FED021ADFED6B
:101AA000011A12E000000000CECC4C3E09EB82038C
:101AB00093ED002A70EE820A93ED072A31EE021AA6
:101AC00093ED0E2A71EE821A521C072AEEDBC8ED46
:101AD000030A88ED041AC8ED051AD1ED1C0A70EE50
:101AE000600A00F27442C2ED000A81ED1C0A98ED12
:101AF0000C0AD0F8741400EE901A30EE200A88ED2B
:101B00000C0A09F6141194EC030A81EC030ADFF8BD
:101B10005417096F01290AD10120C8F84000304646
:101B200088F80000A8F80200A8F804007EE0D8F8C1
:101B30005010491CC8F8501098F80020012A01D014
:101B4000032A3AD102292BD2EA8D042A28DAE96C39
:101B500000296BD198ED0A0ADFEDDA0AB4EE600ACB
:101B6000F1EE10FA08D5D0F8741401EE101AB4EEA4
:101B7000601AF1EE10FA0FDAF9EE0C0AB4EE600A10
:101B8000F1EE10FA52DBD0F8740400EE100AB4EE55
:101B9000600AF1EE10FA49D50120C8F8400045E08E
:101BA00027290AD3B8F80220002A03D011FA82F1BB
:101BB0004B2902D30121C8F84010D0F8740400EE7C
:101BC000900A98ED0A0A00F083F998F800000128BD
:101BD0002CD1B8F80200002828D0B8F80410002949
:101BE00024D0032211FA80F03D2802DB0120C8F83E
:101BF0004000E88D042800DB0222B8F8060082428B
:101C000002D20120C8F840003046C8F86400C8F885
:101C10006000C8F85C00FEF7FBFA0746286F6867AB
:101C200030462867A8F80400A8F80600D8F8340061
:101C3000D8F84810401AFA30FA242146B0FBF1F1E6
:101C400004FB1100B8F80A10884201D100F031FA03
:101C5000D8F83400D8F84810401AFA302146B0FBC2
:101C6000F1F104FB1100642801D100F063FAE88867
:101C7000BDF80810814204D1BDF80210AA88914233
:101C800000D00126002814D0D8F83400D8F8481025
:101C9000401AFA302146B0FBF1F104FB1101322960
:101CA00002D10120288116E04B2914D1002028817F
:101CB00011E0A88800280ED0D8F83400D8F84810D1
:101CC000401AFA302146B0FBF1F104FB11007D28E7
:101CD00001D1012028819DF800002989884200D087
:101CE0000126D8F8340009EB8001D1F87414C8F843
:101CF0002810401CC8F83400FA2802D10020C8F887
:101D00003400D8F83800401CC8F83800072802D141
:101D10000020C8F83800D8F83C00401CC8F83C0047
:101D200047EA0600401E8041C043C00F04B0BDEC2E
:101D3000048BBDE8F28F000030B4DFF8243590ED5D
:101D4000000AD3F8142900EE902A30EE600A03F658
:101D50001412D0ED010A92ED011A70EEC10A90ED55
:101D6000021AD2ED021A31EE611AB5EE400AF1EE16
:101D700010FA02DDF0EE401A01E0F1EE401AF5EE45
:101D8000400AF1EE10FA02DDB0EE602A01E0B1EE99
:101D9000602AB5EE401AF1EE10FA02DDF0EE412AAB
:101DA00001E0F1EE412A71EE821A71EEA21AB5EE4F
:101DB000400AF1EE10FA01DCB1EE400ADFF8A404AB
:101DC00090ED072A32EE000A80ED070AF5EE400A90
:101DD000F1EE10FA01DCF1EE600A90ED080A30EE47
:101DE000200A80ED080AB5EE401AF1EE10FA01DC87
:101DF000B1EE411A90ED090A30EE010A80ED090AB0
:101E000090ED0A0A30EE210A80ED0A0A2F4AD46BBF
:101E1000002C12D1002406E003EB850505F67C05B5
:101E2000C5ED001A641CA4B225460F2DF4DBB2EEFA
:101E30000E0A21EE800A80ED150A148903EB840353
:101E4000D3F87C5800EE105A31EEC00AD0ED150AD6
:101E500030EE200A80ED150A03F67C03C3ED001A6C
:101E6000F2EE0E0A80EE200ADFF8F03383ED1B0A53
:101E7000D0ED170AB4EE600AF1EE10FA01D580ED4C
:101E8000170AD0ED180AF4EE400AF1EE10FA01D567
:101E900080ED180ADFEDA50AB4EE600AF1EE10FA43
:101EA00003D5836DC918816501E000218165611C3E
:101EB000118189B20F2901D100211181806D30BCBF
:101EC000704700000100E040583C0300D039030097
:101ED0009FED971ADFF88403C08D042801DBB0EE74
:101EE000001ADFF88403B5EE400AF1EE10FA07DBC2
:101EF000F5EE400AF1EE10FA02D5C188491CC18006
:101F00000178002905D0022960D02DD3032976D08D
:101F1000B0E0F1EE0C1A31EE211AB4EE401AF1EEF7
:101F200010FA0BDBB4EE601AF1EE10FA06D5016D73
:101F30001029C0F08F80002101658BE0416BDFF834
:101F4000202302EB8101D1F8741401EE901ADFF81E
:101F50001C1391ED010AF4EE401AF1EE10FA40F173
:101F60008980C1ED011A85E0416BDFF8F42202EBB4
:101F70008101D1F8741401EE901ADFF8F01291ED9E
:101F8000002AB4EE612AF1EE10FA01D5C1ED001A73
:101F9000F7EE001AB4EE610AF1EE10FA6ADBB7EE62
:101FA000000AF4EE400AF1EE10FA63D5016D4180AB
:101FB00000210165B9EE0C0A30EE410AF4EE400A48
:101FC000F1EE10FA10D40221017053E0F9EE0C1A70
:101FD00031EEC11AB4EE410AF1EE10FA4ADBF4EE2A
:101FE000410AF1EE10FA45D5032101709C49426B7C
:101FF00001EB8201D1F874149C4A51603AE0416BC4
:10200000974A02EB8101D1F8741401EE901A9749B6
:1020100091ED012AF4EE421AF1EE10FA01D5C1ED6C
:10202000011ADFED7B1AB4EE610AF1EE10FA21D548
:10203000F4EE610AF1EE10FA1CDB016D81800021E3
:102040000165B1EE0C0A31EE000AB4EE600AF1EE61
:1020500010FA0ED50121017084490A6842654A6868
:1020600082657F4A436B02EB8302D2F874240A60D4
:1020700000E0017000787047002803D077492C22D7
:1020800000F056B97047002806D0764942684A6089
:1020900002680A60007A0872704780B5002801D192
:1020A000002002BD54220146714800F041F9012090
:1020B00002BD10B5694CE08DA18D002904D0002827
:1020C00002D00020208106E0084302D001202081B8
:1020D00001E0022020810020E0646062A061A08015
:1020E000A08520636065A06502464021614800F03C
:1020F000E1F8E06F012801D1FEF744FD5948818ADB
:10210000002909D0E28E8A4201D2A18600E0A2868F
:10211000002181820846A067A06F012801D1E08ECE
:10212000A0860020A06710BD00000000EC51383EE2
:102130000000000010B5494CE08DA18D002904D0AD
:10214000002802D00020208106E0084302D00120B0
:10215000208101E00220208100206062A061E085F2
:10216000E08002460821444800F0A4F800202063E3
:10217000E06F012801D1FEF705FDA06F012801D114
:10218000E08EA08610BD80B5012036490867FFF7B4
:10219000D1FFFFF78EFFBDE8014003E00020314989
:1021A000086770472F48008B2C49898E814200D2E6
:1021B00000E070472949CA6C8B8E9A4203D2888608
:1021C0000020886770472749888270472348C16C80
:1021D000002904D1018E408E10FA81F07047002052
:1021E000704701460020002902D0012901D0704724
:1021F00002E01A48C06C70471848818EC26C891A78
:10220000028E891A408E081A00D5002070470000FF
:10221000FEFF7FBF38B504461348124D0F49012C0D
:1022200006D10622CA860C222A839622428105E024
:102230000722CA860F222A8364224281E88AA042AA
:1022400009D0888E082803DAC88EFFF7B3FF02E0B2
:10225000288BFFF7AFFFEC8231BD0000503A03003E
:1022600030460300D03A0300D0390300B0AD03007C
:10227000583C0300A8A90300E84E030081B08DED8F
:10228000000A0098401000F1FE500090DDED000AB9
:10229000C0EE200A9DED001A70EE810ACDED000A15
:1022A000B5EE001ADDED001A80EE210A00EE810A7B
:1022B00001B0704762F30F2262F31F4200B500BF06
:1022C000130096469446103928BFA0E80C50FAD85F
:1022D0005FEA417C28BF0CC048BF40F8042BC90707
:1022E00028BF20F8022B48BF00F8012B00BD50F892
:1022F000041B61B150F8042BD30744BFA9F10103BB
:102300009A180023091F42F8043BFAD1EFE77047FF
:1023100062B38B0708D0521E11F8013B00F8013B55
:1023200000F024808B07F6D1830740F0208000BFA7
:10233000103A07D330B4B1E83810103AA0E838109A
:10234000F9D230BC530724BFB1E80810A0E8081048
:1023500044BF51F8043B40F8043BD20724BF31F896
:10236000022B20F8022B44BF0B7803707047083A09
:1023700007D3B1E80810083A40F8043B40F804CB12
:10238000F7D25307E4E78268521C8260426832B198
:102390000268531C036011704168491E4160704718
:1023A0000022FFF78BBF000062F30F2262F31F428F
:1023B000401810F0030308D0C91A1FD3DB0748BF29
:1023C00000F8012D28BF20F8022D130030B4144668
:1023D0001546103928BF20E93C00FAD8490728BF24
:1023E00020E90C0048BF40F8042D890028BF20F8E0
:1023F000022D48BF00F8012D30BC7047C91818BF26
:1024000000F8012DCB0728BF00F8012D7047000010
:1024100000B583B00FF23800D0E90023CDE90023E6
:1024200000A802F044F89DF900004FF461619DF9A5
:102430000120C2EB02139A0011FB00209DF902104B
:1024400040FA81F04FF47A7148430EBD000000005D
:10245000000000000000000010B500F04DF9DFF8AA
:10246000A84CA078022802D0207A002801D100F0E0
:102470009BFA2079002801D001F03DFCDFF88C0C9C
:102480000078002803D0BDE8104001F027BD10BD42
:1024900080B5DFF87C1C0FF2200002F06DF902F02D
:1024A0003CFADFF8701C48630020DFF85C1C4871C0
:1024B000BDE80140A2E000002573203A534C435F81
:1024C000537461727400000080B5DFF8441C0FF291
:1024D000100002F051F9BDE8014001F04DBD0000CF
:1024E0002573203A534C435F53746F700000000013
:1024F00070B5DFF8204CDFF8105C05F1580120467C
:1025000001F032F9D4E90401DFF80C6CD6E90423B8
:10251000994201D1904215D0002901D1002811D053
:10252000DFF8E80B007800280CD1A879002804D146
:1025300000220321022000F011F83046214620221B
:10254000FFF7F6FEE87829790843DFF8C01B097821
:10255000084301D0206B70BD002070BDF8B5074660
:102560000E461446DFF8AC5B686B002803D0E86ABF
:10257000B0F5FA7F05D902F0D0F968630020E8626F
:102580002863FFF745FF696BEA6A5754EA6A521CF1
:10259000EA625654EA6A521CEA62230E5354EA6A0B
:1025A000521CEA62230C5354EA6A521CEA62230A60
:1025B0005354EA6A521CEA625454EA6A521CEA62B0
:1025C000030E5354EA6A521CEA62030C5354EA6A3B
:1025D000521CEA62030A5354EA6A521CEA625054DB
:1025E000E86A401CE862296BB1F5FA7F00D22863E3
:1025F000B0F5FA7F01D30020E862F1BD38B5DFF80D
:10260000101B0FF2E80002F0B7F8DFF8FC4A0020D8
:10261000207042F21375024601212846C046C0468A
:1026200000206070024602212846C046C0460022B3
:102630003021DFF8E80AFFF73DFE00220C2104F10B
:102640001000FFF737FE00220C2104F13000FFF7E5
:1026500031FE00220C2104F13C00FFF72BFE00228A
:102660002021DFF8B00AFFF725FE00222021DFF845
:10267000A80AFFF71FFE0022182104F15800FFF7F7
:1026800019FE0020E0702071A0673C20A0614FF48B
:102690009670A06301202072607200206071A071AA
:1026A0006073A073E0670120A0700022014642F22F
:1026B0001270C046C0460020207340F6B830206734
:1026C00000200146C4E91401C4E912014FF0FF30B3
:1026D00060670A46142104F11C00FFF7EBFD9FED33
:1026E000D00A84ED070A84ED080A31BD257320471E
:1026F0004320496E69740000F8B5DFF80C4AE078B1
:10270000002800F0F980DFF80C5A2078012808D062
:10271000022823D0042800F08580062800F0C88015
:10272000F1BD288C401C288480B23228C0F2E4809D
:10273000DFF8DC696369A26931460FF2C01002F06C
:102740001BF8227831460FF2D41002F015F804F18C
:10275000100000F07FF900202884F1BD688C322839
:1027600001DB00206884688C002805D1DFF8A019FF
:102770000FF2B81002F000F8688C401C688404F175
:102780005801284600F0F0FFDFF88C7939462846DA
:1027900000F086FB00282FD0002202210120FFF745
:1027A000DDFE0020A8620120E07138462946202283
:1027B000FFF7BEFDA07802280CD10120A0700022F6
:1027C000014642F21270C046C0460022012102209A
:1027D000FFF7C4FE012020700246014642F213704A
:1027E000C046C0462079002800F08680FFF710FE22
:1027F00020640020E063F1BDA86A401CA862FA28AA
:1028000006D1A06D002877D1E079BDE8F240F2E270
:1028100040F2EE2188426FD30020A862E079BDE843
:10282000F240E8E2DFF8E86831460FF21C1001F0F0
:10283000A3FFDFF8E4783946284600F031FB002892
:102840002ED0002206210120FFF788FE0020A8627A
:102850000120E071384629462022FFF769FDA07863
:1028600002280CD10120A0700022014642F2127011
:10287000C046C046002201210220FFF76FFE012062
:1028800020700246014642F21370C046C0462079CD
:10289000002831D0FFF7BCFD20640020E063F1BDCB
:1028A00031460FF2C00001F067FF01202070F1BD3A
:1028B000A88C322801DB0020A884A88C002805D130
:1028C000DFF84C180FF2C80001F056FFA88C401C2E
:1028D000A884206F401E20670ED100F0E3FE022086
:1028E00020700246012142F21370C046C04640F6F5
:1028F000B83020670020E071F1BD0000257320484A
:10290000575F4750535F5052206D696E5F742025AA
:10291000642C206D696E5F64202564002573204857
:10292000575F4750535F505220256400257320485D
:10293000575F4750535F5052204750532074726185
:10294000636B696E6700000025732048575F47502E
:10295000535F5052207061737369766520475053FE
:102960000000000025732048575F4750535F5052C6
:102970002070617373697665204641494C45442D4A
:1029800046414C4C4241434B2041520A000000005A
:1029900025732048575F4750535F5052204750538C
:1029A0002074696D6572000070B5DFF85C57687857
:1029B000012802D0032821D070BDDFF8444E2088C2
:1029C000401C208080B2322814DBDFF844676B6B38
:1029D000AA6B31460FF24C0001F0CEFE6A78314608
:1029E0000FF2600001F0C8FE05F1300000F03AF887
:1029F0000020208043F69820606070BDDFF8004E14
:102A00006068401E606009D100206863A86305F11A
:102A1000300000F09BF843F69820606070BD000025
:102A2000000048432573204E4C505F5052206D6982
:102A30006E5F742025642C206D696E5F64202564B0
:102A4000000000002573204E4C505F50522025643A
:102A50000000000010B5044600F0B2F82046BDE8C2
:102A6000104025E010B5044600F0AAF8204600F01A
:102A70006DF8DFF8780DC168002918D0012902D15E
:102A800000216160C160017801290ED141780229DD
:102A900006DA017A00290AD0C168491EC16010BD5A
:102AA00005D100210172C16010BD0121017210BD6C
:102AB00010B5DFF85446217A002917D08168012922
:102AC00014DA4068012802DB606F00280ED14FF055
:102AD000FF30606700F0E6FD022020700246012111
:102AE00042F21370BDE8104001F0F3B810BDF8B524
:102AF000DFF8F84C2078042810D1FFF789FC00217A
:102B0000DFF80426D2E91467801BB94144F620623D
:102B10000023994216D801D3904213D2207801287D
:102B200012D0FFF775FC0021DFF8DC25D2E9124551
:102B3000001BA9414EF660220023994204D301D81C
:102B4000904201D30120F2BD0020F2BD38B5DFF87C
:102B5000B845617A002932D0816801292FDA4068AE
:102B6000012802DB606F002829D14FF0FF30606739
:102B7000207A002817D0FFF7BAFF002813D000F002
:102B800091FD0220207042F2137502460121284671
:102B9000C046C04600206070024602212846BDE8BB
:102BA000384001F096B801F095F8032060700246B5
:102BB000022142F21370BDE8384001F08AB831BDFD
:102BC0002DE9FC470446002702F0ADFF0546DFF87B
:102BD0003865B06F002800D02F1AB56700A802F042
:102BE00091FFDFF8088C404600A90622FFF790FB12
:102BF000DFF81C9598F80100009098F800302A46FC
:102C000049460FF2701001F0B7FD98F80000012856
:102C100026D1FFF7FDFB0021C6E9120198F801005B
:102C200002280FDAF07B002826D096F90B00002846
:102C300022D096ED200ADFED930A30EE200A86EDD1
:102C4000200A19E018D1F07B002806D096F90B0075
:102C5000002802D008466060A0600846F0730BE0D0
:102C6000042807D1707B042804D0FFF7D1FB002192
:102C7000C6E914010120F07396ED200AF7EE000A70
:102C8000B4EE600AF1EE10FA06DB7F1CFFEE000ADC
:102C900030EE200A86ED200AB07A002822D098F87B
:102CA000000004280ED194ED010AB8EEC00ADFED51
:102CB000B50A80EE200ABDEEC00A86ED1D0A00208E
:102CC000B0720FE005280DD194ED010AB8EEC00AEC
:102CD000DFEDAD0A80EE200ABDEEC00A86ED1D0ACA
:102CE0000020B072F06F002800D1F56798F800005E
:102CF000717B81421CD0ED1B4FF00A0AF16F6A1AFA
:102D000098F801101AFB0011C9B20320FFF726FC46
:102D1000F06F2A1A98F8000098F801101AFB0011B9
:102D200042F21570C046C046F56798F8000070730F
:102D30003B46626849460FF2640001F01DFD606881
:102D4000012808DB012F02DBC01B606003E0002FBD
:102D500001D500206060B07A002804D1706F01288E
:102D600001DB401E7067A068012801DB401EA060E7
:102D7000BDE8F38725732047435F43616C5F415291
:102D800044206375725F643A256420747970653AF3
:102D90002575206163633A2575000000257320477F
:102DA000435F43616C5F415244206D696E3A256414
:102DB00020646966663A25640000000038B5D24C8C
:102DC000A078022816D1002060634FF49670A063AB
:102DD0000120607042F21375024602212846C04667
:102DE000C04600202070024601212846BDE8384038
:102DF00000F06FBF31BD38B505462A46C4490FF211
:102E0000880001F0B9FC00F080FCBF4C002D0ED012
:102E1000062020700246012142F21370C046C046CF
:102E2000002203210120BDE83840FFF797BBA078BE
:102E300001280CD10220A0700022014642F212703B
:102E4000C046C046002202210846FFF787FB607A91
:102E5000002813D000F03EFF0320607042F213758B
:102E6000024602212846C046C04600202070024685
:102E700001212846BDE8384000F02BBFBDE83140B5
:102E80009CE700001F852B3F2573204743204820E7
:102E90004750532074696D656F7574202564000078
:102EA000F0B583B00446D4E90423D1E90467BB42FA
:102EB00001D1B24264D0002B01D1002A60D094ED40
:102EC000000AB5EE400AF1EE10FA06D1D4ED010A7F
:102ED000F5EE400AF1EE10FA1DD0DFED870AB4EEF0
:102EE000600AF1EE10FA16D4DFED840AB4EE600A3F
:102EF000F1EE10FA0FDA94ED010ADFED810AB4EE7B
:102F0000600AF1EE10FA06D4DFED7E0AB4EE600A34
:102F1000F1EE10FA06DB6422FF210420FFF71EFB0E
:102F20000020FEBD7D4900F04DF800F0EEFB764D2F
:102F30003C20A8610120A8722068E86160682862CE
:102F4000FFF766FA686202F0EEFDA862A069E86227
:102F50006F4CAA6A21460FF2340001F00DFC286A7A
:102F600002F070FFCDE90001E86902F06BFF024654
:102F70000B4621460FF22C0001F0FEFB0120FEBDA6
:102F80000020FEBDCDCC5C41CDCCDC40257320477C
:102F9000435F485F4C2061725F64697374202564ED
:102FA0000A00000025732047435F485F4C206C6196
:102FB00074203A2025662C206C6F6E203A202566FE
:102FC0000A0000002DE9F0412DED028B04460D466C
:102FD0004D4E6FF000407061002712E030EE480A5D
:102FE000D6ED050AF8EEE00AB4EE600AF1EE10FA4A
:102FF00006D5BDEEC00A86ED050A38F8010030821C
:103000007F1C0A2F25DA302000FB07F808EB0500AB
:1030100081780029F4D0D0ED031A90ED021AD4ED96
:10302000010A94ED000A00F07BF8B0EE408A3846C1
:1030300080B200F025F8394908EB010090F92C2006
:10304000002A90ED0A0AB8EE400AC7D038EE400ACE
:10305000C6E70120F07200210CE0302000FB015097
:103060008278002A05D090F92C00002801D1002098
:10307000F072491C0A29F0DBBDEC028BBDE8F0813F
:1030800000EB40010901254A885A8918D1ED0A0A46
:10309000F8EE600A283191F90420002A0AD0012AAA
:1030A00018D0B2F1FF3F25D1F4EE400AF1EE10FA4C
:1030B00015D504E0F4EE400AF1EE10FA1AD501221B
:1030C0000A7114498A69D1ED010A91ED000A0121C2
:1030D00000F09ABDB4EE600AF1EE10FA0AD50022B3
:1030E0000A710C498A69D1ED010A91ED000A0021AB
:1030F00000F08ABD704700000000B4C20100B44275
:10310000000034C30100344340390300CCAB03005A
:103110009850000020AA0300E8AB0300688E03006B
:103120002DE9704F2DED108B94B0B0EE418A9FEDDC
:1031300073AA21EE8A1A00EECA1A8DED0B1A00202E
:103140000A9020EE0A0A02F0A5FE9FED6D9BF7EEB5
:10315000000AF0EE608A10EE100A02F073FE53ECE3
:10316000192B02F047FF03F017F800EE100AF0EEFB
:10317000680A03F059F8F0EE408A28EE0A0A02F0D5
:1031800089FEF7EE000AB0EE608A10EE100A02F037
:1031900059FE53EC192B02F02DFF02F0FDFF00EE5B
:1031A000100AF0EE480A03F03FF8B0EE408AB0EEA5
:1031B000680A03F070F88DED090AB0EE480A03F0D2
:1031C0006AF88DED040AB0EE680A03F067F88DED39
:1031D000080AB0EE480A03F061F88DED070A9DED8C
:1031E000090ADDED040A20EE200A8DED060A9DEDA8
:1031F000080ADDED070A20EE200A8DED050A9FED95
:103200003EEA9FED3DAA9DED0B8A002600E0761C6C
:1032100036B2142E80F230828DED0C8AB0EE480A60
:1032200003F039F8F0EE409AB0EE480A03F036F8B1
:10323000B0EE409A9DED040A20EE090ADDED090A80
:103240009DED071A60EE810A9DED081ADDED041A66
:1032500021EE211A41EE690A20EE000A00EEA00AD2
:10326000B5EE400AF1EE10FA0EDB10EE100A02F095
:10327000E9FD41EC100B03F015F851EC100B02F0D6
:103280008BFF08EE900A01E0DFED1B8A9DED060A38
:103290009DED058A00EE298AF0EE480AB0EE680A34
:1032A00002F0C2FFB0EE40EAF5EE408AF1EE10FA0D
:1032B00002D1DFED11EA05E09DED060A20EE090AD4
:1032C000C0EE28EAB7EE00AA0EEEEEAA18EE100A3B
:1032D00002F0B8FDCDE912011AEE100A02F0B2FDBB
:1032E00041EC1B0B9FEDED9BB5EE40AAF1EE10FA01
:1032F0000AD19FED01CA1CE00000000034FA8E3CA8
:10330000000020B588E4EF3F059802F09BFD53ECE8
:10331000192B02F06FFE53EC1B2B03F043F802460F
:103320000B46DDE9120103F061F902F035FF0CEE06
:10333000100A9FEDD90A2AEE000A10EE100A02F0D8
:1033400081FD41EC1A0B0022DFF8803B02F052FEB7
:1033500004460D4651EC1A0B0022DFF8743B02F0D4
:1033600049FE02460B460020DFF8681B03F03EF9D9
:1033700002460B4651EC1A0B02F03CFE0022DFF82D
:10338000583B03F0F3F902460B4651EC1A0B02F0DE
:1033900031FE0022DFF8DC3B03F0E8F922462B4641
:1033A00002F028FE0022DFF8003C03F0DFF902F013
:1033B000F3FE0A9051EC1A0B0022DFF8F03B02F00A
:1033C00019FE04460D4651EC1A0B0022DFF8E03BD3
:1033D00002F010FE02460B460020DFF8D81B03F077
:1033E00005F902460B4651EC1A0B02F003FE0022CF
:1033F000DFF8C43B03F0BAF902460B4651EC1A0B56
:1034000002F0F8FD0022DFF8043C03F0AFF9224699
:103410002B4602F0EFFD02F0BFFE0FEE100A9FED0B
:10342000D0AB51EC1B0B4FF06042DFF8E43B02F0F5
:10343000E1FD04460D4651EC1B0B0022DFF8103C69
:1034400002F0D8FD02460B4651EC1A0B03F0CEF801
:103450004FF06042DFF8FC3B02F0CCFD53EC1A2B3E
:1034600003F084F922462B4602F0C4FD02F094FEDC
:103470000FEE900A2CEE0C0A10EE100A02F0E2FC9D
:10348000CDE9100118EE900A02F0DCFCCDE90E0146
:103490001FEE100A02F0D6FCCDE902011CEE100A64
:1034A00002F0D0FC41EC1B0B9FEDD1CB9FEDD2DBAA
:1034B0002FEE280A10EE100A02F0C4FCCDE900013C
:1034C000DDE902010022DFF8903B02F093FD0446A3
:1034D0000D46DDE9100153EC192B02F08BFD53EC86
:1034E0001D2B03F043F902460B46DDE9120102F001
:1034F00081FD82468B46DDE902010022DFF85C3B5C
:1035000002F050FF53EC1B2B02F074FD80468946FD
:10351000DDE90E2351EC1A0B02F06CFDDDE90E2300
:1035200002F068FD53EC1C2B03F020F942464B4699
:1035300002F060FD80468946DDE9102351EC1A0B4C
:1035400002F058FD53EC1C2B03F010F942464B4699
:1035500002F050FD02460B465046594603F046F82D
:1035600022462B4602F046FD02460B4651EC1B0B51
:1035700003F0FCF8DDE9002302F03CFD02F00CFE54
:103580000AEE100A0B9802F05DFCCDE902011FEE75
:10359000900A02F057FC02460B460020DFF8081A9A
:1035A00003F024F84FF06042DFF8A83A02F022FD61
:1035B00004460D461EEE900A02F044FC22462B46BD
:1035C00002F018FDCDE900011EEE100A02F03AFCEF
:1035D000804689462FEEA80A10EE100A02F032FC4F
:1035E00004460D462FEE880A10EE100A02F02AFC5F
:1035F00082468B4653EC1B2B51EC190B02F0FAFC64
:1036000053EC1B2B02F0F6FC53EC1D2B03F0AEF831
:1036100052465B4602F0EEFC53EC1B2B03F0A6F87F
:1036200022462B4602F0E6FC42464B4603F09EF84B
:10363000DDE9002302F0DEFCDDE9022303F096F869
:1036400002F0AAFD08EE100AB5EE408AF1EE10FA7B
:1036500002D19FEDAF0A05E09DED0C0A38EE400A5D
:1036600080EE080AB0EEC00ADFEDD10AB4EE600ABF
:10367000F1EE10FA7FF5CBAD9DED0A0ADFEDCD0A34
:1036800020EE200A7EEE4A0A20EE200A14B0BDEC9D
:10369000108BBDE8708F000032D6DC3B00000000CC
:1036A0000000004038B5682003F071FA01460020A0
:1036B0008DF80000002921D0DFF8A449A079002866
:1036C00022D10FF6D41500A8C96949688847002897
:1036D000294604D00FF6CC1001F04EF803E00FF6A7
:1036E000D81001F049F80020DFF88819886201201D
:1036F000A07100220146FEF731FF31BD0FF698118F
:103700000FF6C81001F038F831BD38B5682003F065
:103710003EFA014600208DF80000002919D0DFF89C
:103720004049A07900281AD00FF66C1500A8C96985
:10373000C96888470028294604D00FF6A01001F078
:103740001BF803E00FF6A81001F016F80020A07196
:1037500031BD0FF644110FF6741001F00DF831BDB4
:10376000000000000000104070B504460D4603F054
:1037700021FD0646D6E9000102F00EFD2060D6E9E3
:10378000020102F009FD60600020A060E060D6E95F
:103790000A01C4E90401306BA061002D02D096F843
:1037A0003C00286070BD38B5DFF8B4486079002867
:1037B0001BD10FF6E40529460FF6481000F0DCFF98
:1037C000002204F18401432003F0D3F800282946A5
:1037D00005D00FF64010BDE8344000F0CDBF0FF625
:1037E000481000F0C9FF0120607131BD644503003D
:1037F00000000000000008C0000000000000F0BF52
:103800001C46030038B5DFF85848607900281BD003
:103810000FF6840529460FF6241000F0ADFF0022B4
:1038200004F18401432003F0FAF80028294605D06A
:103830000FF61410BDE8344000F09EBF0FF62010C4
:1038400000F09AFF0020607131BD0000F8B52DED49
:10385000028B064608EE101A08EE902A1C46DFF886
:103860000058E87800280FD1FFF79DFF012000F0F5
:10387000D1FB0021DFF8EC07FFF776FF00220121E2
:1038800042F21470C046C0460120E8704FF0FF308D
:10389000E8720021DFF8D03700E0491C0A2921DA5C
:1038A00001EB41021201D71897F802C0BCF1000FDA
:1038B000F3D1D652B8EEC80ADFED9D0A80EE200A99
:1038C00087ED020A07F10801B8EEE80A80EE200A47
:1038D00081ED010A0C6287F82C000120B870287B6A
:1038E000401C2873287A00280ED0A87801280BD114
:1038F000FFF7D8FE022028700246012142F2137021
:10390000C046C0460120E871BDEC028BF1BD00004D
:103910000000000070B54FF0FF31DFF8444701228E
:10392000E27200220AE0EB189D78002D05D093F991
:103930002C30002B01D10023E372521C0A2A08DA32
:1039400030255543DFF82037EE5A8642EBD1114639
:10395000F3E709B211F1010F28D0207B401E20733C
:103960003025DFF8043715FB0130002181700A464D
:103970002946FEF719FD207B002817D10020E070B2
:103980002079DFF8F8164978084301D1FFF73AFFAC
:10399000FFF7BBFE002000F03DFBFEF72FFE0022EC
:1039A000022142F21470BDE8704092E170BD000047
:1039B000CDBC8C2B21FEC14A10B5044622460FF225
:1039C000D8610FF2AC7000F0D7FE012C0ED1DFF8F9
:1039D000904600202072FFF798FE002020700246DB
:1039E000012142F21370BDE8104072E1032C0BD1AB
:1039F000DFF86C460020607260700246022142F2DD
:103A00001370BDE8104064E110BD38B5044622468D
:103A10000FF284610FF2687000F0AEFE022C2DD11F
:103A2000DFF83C46207A00282ED101202072E07871
:103A3000002829D0FFF736FE0220207042F21375CD
:103A4000024601212846C046C0460020607002465A
:103A500002212846C046C04600200A2814DADFF8B2
:103A6000081600EB400201EB02118A78002A03D00D
:103A70004FF0FF3281F82C20401CEEE7042C03D1DC
:103A80000120DFF8DC15487231BDF8B506460C465A
:103A900015460FF2046739460FF2F86000F06CFE2D
:103AA0004FF0FF30002109E0DFF8BC2501EB4103B6
:103AB0001B019A5AB24200D10846491C0A29F3DB7D
:103AC00000B210F1010F15D03021DFF89C2511FB59
:103AD00000208462283090F9041011F1010F07D101
:103AE000DFF87C359978022902D0197A002906D1AD
:103AF000057104E039460FF2B86000F03DFEDFF8D2
:103B000060350120D87200200EE03021DFF8582502
:103B100001FB00218A78002A05D091F92C10002998
:103B200001D10021D972401C0A28EEDBF1BD000052
:103B30008096184BF8B504460D462F463B46224664
:103B40000FF254510FF27C6000F016FEDFF81065A2
:103B5000F078002801D1FFF726FEB078022802D0C5
:103B6000307A002828D1C7EB07108000B063746357
:103B700001207070DFF8080540F2DC518C4202D25F
:103B80000021C16009E00A21B4FBF1F1C160B1F587
:103B9000967F02D24FF49671C16042F213770122F0
:103BA00002213846C046C04600203070024601213E
:103BB0003846C046C04611E074613C20B061012027
:103BC00030700246014642F21370C046C04640F6CD
:103BD000B83030670020F0710120B072FFF795FD1A
:103BE000224629460520BDE8F840FEF7B7BC80B55F
:103BF0000FF2A4410FF2F05000F0BEFDDFF86004B8
:103C000000214170017001BD70B52DED028B84B0B3
:103C100004460D46B0EE408AF0EE608A164618EE75
:103C2000900A02F00FF9CDE9020118EE100A02F035
:103C300009F9CDE900012B4622460FF25C410FF253
:103C4000B85000F099FD9FED9E0AB4EE408AF1EE67
:103C500010FA14D49FED9B0AB4EE408AF1EE10FAEC
:103C60000DDA9FED990AF4EE408AF1EE10FA06D4CF
:103C70009FEDBF0AF4EE408AF1EE10FA09DB22460E
:103C8000FF21042004B0BDEC028BBDE87040FEF7BC
:103C900065BCDFF8D803048085709FEDC20A68EE2A
:103CA000000AFDEEE00AC0ED010A28EE800ABDEE32
:103CB000C00A80ED020AC660012001F057F82246D2
:103CC0002946042004B0BDEC028BBDE87040FEF72D
:103CD00045BC704780B50FF2C0310FF2405000F084
:103CE0004BFD002204210120FEF738FC0320BDE833
:103CF000024001F03BB810B5E04C2078012809D112
:103D00006088401C608080B2322803DB00F003F83A
:103D10000020608010BD7CB5002601F004FFD44C6B
:103D2000A168002900D0461AA060CD4DE86B30187C
:103D3000E86300A801F0E6FE204600A90622FEF78F
:103D4000E7FA2078A97B81420ED0E978002909D1D1
:103D5000EA6B00EB8001480061784118C9B2062087
:103D6000FEF7FCFB2078A87373BD10B50FF2283165
:103D70000FF2B44000F000FDB94C0120207100208A
:103D8000E063FEF745FB606420640120BB490870D6
:103D9000BDE8104007E580B50FF2FC210FF2984016
:103DA00000F0EAFCAE4800210171B44900220A701B
:103DB000C0784978084302D1BDE8014022E501BD41
:103DC00080B50FF2D4210FF2804000F0D5FCA44959
:103DD000C86B0A6C496C511A0BD0A6498A690092CB
:103DE000D1ED010A91ED000AD1E9042300F01EF89B
:103DF00001BD9FEDA40A00210091F0EE400A0A46A1
:103E00000B4600F013F801BD10B50FF28C210FF234
:103E10004C4000F0B1FC924C0020E063FEF7F8FA51
:103E20006064206400209249886010BD38B52DED93
:103E3000048B09EE100A14461D46B0EE408AF0EEDF
:103E4000608A19EE102A0FF250210FF2204000F084
:103E500093FC8948B8EE490AF2EE040A20EE200AE3
:103E6000BCEEC00A80ED000AC0E902459FED4D0A94
:103E700068EE000AFDEEE00AC0ED040A28EE800AB2
:103E8000BDEEC00A80ED050A089981610420BDECF1
:103E9000048BBDE8324000F069BF01280FDB7A498E
:103EA00001220A7000224A618A614A70B0F5167FC9
:103EB00002DA0B300861704740F259200861704700
:103EC0000000B4C20100B442000034C30000103F3F
:103ED00000E0654000007440000088C038B52DED5A
:103EE000028B694C6069411C6161226932235A432B
:103EF000904204D3BDEC028BBDE831403CE0B1F50B
:103F0000FA7F32D36078002807D1FFF7CBFB01207E
:103F1000607022690146FEF721FBA069411CA16186
:103F2000322822D30020A06103F044F9054695F819
:103F30003C00A0809FED558BD5E9002351EC180B78
:103F400002F058F803F0C8F9A060D5E9022351EC5B
:103F5000180B02F04FF803F0BFF9E0600220BDEC4F
:103F6000028BBDE8324000F001BFBDEC028B31BDD9
:103F7000010034430000B04010B5434C20780028C5
:103F80000ED00020207020616061A0616070FFF79A
:103F9000BCFB226905210120BDE81040FEF7DEBA16
:103FA00010BD00008096184B0000F03F0000503F0D
:103FB0000080474000805240000060C038B5044691
:103FC0000FF2C02000F0D8FB25480178022916D056
:103FD00004210170274DD4E9000102F0DDF82860CA
:103FE000D4E9020102F0D8F868600020A860E86017
:103FF000D4E90A01C5E90401206BA86131BD0FF2C3
:10400000A420BDE8324000F0B7BB000000007040C3
:104010004A772B3F10B50FF2800400280CD01D48C2
:1040200003F00CFA012003F03FFA21460FF2A02022
:10403000BDE8104000F0A0BB002003F035FA03F00B
:1040400008FA21460FF2A420BDE8104000F094BB0E
:10405000000008404A776B3F0000D03F0000184046
:1040600040390300E8AB0300688E030058AD03003D
:1040700074AD030020AA030008AC0300F4AD0300F4
:104080006445030000004843CCAB0300000000007F
:10409000D0126341BD4F0000534C4356332E302E97
:1040A000383A0000257320475053207374617274AE
:1040B000206661696C00000025732047505320730F
:1040C0007461727420737563630000002573206748
:1040D000657420475053206661696C002573204742
:1040E00050532073746F70206661696C000000008B
:1040F0002573204750532073746F7020737563636A
:104100000000000025732041522073746172740A0C
:104110000000000025733A20453A204152204F709C
:10412000656E206661696C002573204152207374AE
:104130006172742073756363000000002573204171
:10414000522073746F700A0025733A20453A20415B
:104150005220436C6F7365206661696C000000003B
:1041600025732041522073746F7020737563630050
:1041700025732047435F5061757365203A256400BD
:1041800025732047435F526573756D65203A25643A
:10419000000000002573203A47435F557064617446
:1041A000652047465F5374617475733A2564000057
:1041B0002573203A47435F5570646174655F4552CB
:1041C0005200000025733A47435F53746172745F75
:1041D0004152206D696E5F643A25642C206D696ED2
:1041E0005F743A25640000002573203A47435F530B
:1041F000746F705F415200002573204465746563DD
:10420000745F43422069643A25643A2564206C61F6
:10421000743A2566206C6F6E3A2566002573203A45
:1042200041525F43420000002573203A434C432033
:1042300053746172740000002573203A434C43208C
:1042400053746F70000000002573203A434C4320E4
:104250005265712044697374000000002573203A90
:10426000434C432052657365740000002573203A67
:10427000434C4320446973745F4342203A202564D1
:1042800000000000534C4356204C5349206F6E50A1
:104290006173736976654C6F636174696F6E4362B5
:1042A00000000000534C4356204C5349206F6E5081
:1042B0006173736976654C6F636174696F6E436295
:1042C0002047505320747261636B696E6700000071
:1042D00025732047435F4750535F5265675F5061C6
:1042E00073736976655F4342210A00002573204796
:1042F000435F4750535F556E7265675F50617373DC
:104300006976655F4342210A0000000000B587B06E
:1043100007208DF8000005208DF804000120ADF87D
:1043200007000FF20C4000F027FA00A901A803F0E3
:1043300021FA07B000BDDFF89003704710B586B0D2
:10434000044601A81421FEF72BF8FFF7F4FF0090B4
:104350000D22214601A8FDF7DBFF0420ADF8070080
:1043600000A901A803F006FA06B010BDF0B589B0A7
:10437000044602A81421FEF713F800200146CDE9F7
:104380000001012510E0284602F001FC00280AD0B7
:10439000DDE90067012000212A4603F06FFA30436F
:1043A0003943CDE900016D1C292DECDB0D2221469E
:1043B00002A8FDF7ADFF0820ADF80B0000A902A888
:1043C00003F0D8F909B0F0BD10B5040002D00FF227
:1043D000703101E00FF270310FF25C3000F0CCF977
:1043E000B748047010BDB64800787047B4484078AC
:1043F0007047B3488078704770B586B0044600A80F
:104400001421FDF7CDFF0D22214600A8FDF780FF06
:10441000AB4CD4E90401002901D100280DD00DF1E5
:1044200005052A686B68101A63EB0101A54A012390
:10443000994202D822D3904220D3A44D2878401C20
:104440002870802080F3118800BF00BF6878401C6E
:10445000687003F0E9FB0DF1050632687368C4E982
:104460000423C4E906016878401E6870C0B20028C1
:1044700002D1002080F3118803F012FD06B070BD58
:1044800038B503F0D1FB8E4AD2E9044520186941C2
:10449000D2E90645001BA94134BD894902780A7159
:1044A00042784A718078887100200881704706221E
:1044B0008749FDF72DBF824A136A002B01D0CB1A22
:1044C00000E00346B3F57A7F00D30346108918183D
:1044D000108100B2B0F57A7F05DBA0F57A7010810B
:1044E0009079401C907192F906003C2804DB3C381E
:1044F00090715079401C507192F905003C2804DB02
:104500003C3850711079401C107192F90400182841
:1045100001DB0020107111627047000010B5042803
:1045200001DA022010BD142801DA022400E00A2476
:1045300090FBF4F003F068FD41EC100B03F07CFD00
:1045400051EC100B02F0B2FE03F05EFD41EC110BDA
:104550009FED600B03F0BDFF51EC100B02F0A6FEC7
:10456000604310BD00B587B002A80FF2E411142219
:10457000FDF7DEFE00A800210A4606C003F09AF906
:1045800001788DF8001000A9C2784A7042798DF840
:1045900002208079C87001208DF804000520ADF854
:1045A0000B0002A803F0E6F807B000BD30B59FB0DD
:1045B00005A86421FDF7F4FE00A80FF2A81114224B
:1045C000FDF7B6FE0024FF22642105A8FDF772FE68
:1045D000012517E02846C0B202F0D9FA002810D011
:1045E0002946491E012906D9C91E022903D9091FD6
:1045F00001D01A3905D105A964B26554408A401C1E
:1046000004196D1C092DE5DB64B2ADF8034005A962
:1046100000A803F0AFF800201FB030BD10B504466D
:10462000A0780146491E01290FD9091F012914D973
:10463000891E01291DD9891E012922D9203928D195
:10464000D4F80D00FFF729FF23E0012801D1002055
:1046500000E001201A4908701BE0052801D1012063
:1046600000E0002016498870891C062004F079F9C2
:104670000FE0072801D1012000E000201049C87098
:1046800007E00F49092802D10020487001E001200D
:104690004870A0781438032801D915380ED12C2081
:1046A00002F075FA030009D0D4F80D20B4F8031015
:1046B000A078DB691B69BDE81040184710BD0000F9
:1046C00068AB030000F2052A4C082301A03D03005B
:1046D0006CAB0300000000000000004081780C2952
:1046E00006D0182906D01B2903D02C2903D07047E7
:1046F00024E63BE636E759E780B500228DF8002036
:10470000082801DA002809D1052907DA01208DF8E7
:10471000000000A9052004F024F901BD052805DAF0
:10472000082903DB00A9052004F01BF901BD0000E6
:10473000524553455400000061702025730000006D
:1047400073757370656E6400726573756D650000D6
:1047500004FF18000000000000000000000000003E
:104760000000000004FF2C0000000000000000001A
:1047700000000000000000000EB470B5C1B0044697
:1047800000A84FF48071FDF70BFE45AB22464FF4B5
:10479000807100A804F052F900A804F06DF9441CDF
:1047A000002000A9611801F8010C274D2878401C51
:1047B0002870802080F3118800BF00BF6878401CFB
:1047C0006870224E317808462218FA2A0DDA204AFB
:1047D0008018002902D00A2100F8011C224600A9F5
:1047E000FDF796FD3078201830706878401E6870AC
:1047F000C0B2002802D1002080F3118803F050FBE2
:1048000041B070BC5DF810FB10480078002801D062
:10481000801C00E00020C0B2704738B50B4C2278F5
:10482000002A10D000280ED0032101704270084DDC
:104830002946801CFDF76CFD0022FA212846FDF771
:1048400039FD0020207031BDA03D03000CAE0300F7
:1048500010A303000020704780B50FF65010FFF73B
:104860008BFF00224FF40071DFF81C09FDF722FDD9
:10487000FDF70EFE002002BD80B50FF63C10FFF7DD
:104880007BFFFDF721FE002002BD70B5FFF7B1FDF3
:104890000446DFF8F858012C03D195F904000028EC
:1048A00003D095F90500012828D1FDF721FE064621
:1048B00031460FF61010FFF75FFF00206871FB2EE6
:1048C00008D3FA2100F01CF9314689B2FA2000F031
:1048D00017F905E0002E11D0314689B200F010F929
:1048E00000224FF4007105F10800FDF7E3FC002001
:1048F000DFF89C180860DFF89C1808602C7170BD08
:1049000080B50020DFF88418C880FDF7A5FDFFF70B
:10491000BCFF002002BD00207047DFF86C08704724
:10492000F0B583B004460D4616461F4621460FF6E5
:10493000A800FFF721FF09980190089800903B46D6
:10494000324629462046FEF781FFDFF84008012164
:1049500001700021417044800520BDE8FE4005E261
:1049600010B504460FF68800FFF706FF2046FEF755
:10497000D1FFDFF818080221017000214170448046
:104980000520BDE81040F1E138B50446254629462A
:104990000FF67400FFF7F0FE012D0AD12046FFF755
:1049A0000BF8DFF8E8070321017000214170418016
:1049B00025E0022D0AD12046FFF727F8DFF8CC07C3
:1049C0000421017000214170418018E0032D0AD1BB
:1049D0002046FEF7F1FFDFF8B40705210170002142
:1049E000417041800BE0042D09D12046FFF70DF8FE
:1049F000DFF89807062101700021417041800520F1
:104A0000BDE83240B2E170B504460D4616460FF6D9
:104A10001800FFF7B1FE324629462046FFF735F869
:104A2000DFF86807072101700021417044800520EC
:104A3000BDE870409AE138B504460D462A46214645
:104A40000FF61000FFF798FE29462046FFF772F890
:104A5000DFF83807092101700021417041800520ED
:104A6000BDE8324082E180B50FF60800FFF784FE12
:104A7000FFF7BDF8DFF814070A210170002141702B
:104A800041800520BDE8024070E110B50446214692
:104A90000FF2F070FFF770FE012C06D028D3032C24
:104AA00015D00BD3042C1BD022E0FFF75EF9DFF802
:104AB000DC06002141700B21017019E0FFF76BF952
:104AC000DFF8C806002141700C21017010E0FFF7EB
:104AD00077F9DFF8B806002141700D21017007E079
:104AE000FFF792F9DFF8A406002141700E21017052
:104AF0000020DFF8981648800520BDE8104035E119
:104B000070B586B004460E4622460FF29470FFF749
:104B100033FE301B0A2190FBF1F5ADB2801DADF8DC
:104B2000000001A80FF2FC711422FDF701FCBDF892
:104B30000000C01CADF80700DFF85C660120307093
:104B4000022200A9701CFDF7E3FB0120F070307118
:104B5000372070710620B0712846000AF071357256
:104B6000BDF80000C21EDFF82406201800F108017D
:104B700006F10900FDF7CCFB314601A802F0FAFD71
:104B800006B070BD3EB5054614460A4629460FF2EA
:104B90002C70FFF7F1FD0020ADF80800102D40F05B
:104BA000DF80207801283BD1E07C217D090401EBE6
:104BB0000060617D00EB0120A17D40180190E07B49
:104BC000217C090401EB0060617C00EB0120A17CE9
:104BD00040180090E07A217B090401EB0060617BC2
:104BE00000EB0120A17B4318E079217A090401EB55
:104BF0000060617A00EB0120A17A4218E078217907
:104C0000090401EB0060617900EB0120A1794118F2
:104C10006078A47814EB002080B2FFF781FE9FE05B
:104C2000022807D16078A17811EB002080B2FFF74D
:104C300097FE95E0032807D16078A17811EB00205A
:104C400080B2FFF7A1FE8BE0042812D1E279E07870
:104C50002179090401EB0060617900EB0120A17961
:104C600041186078A37813EB002080B2FFF7CBFEE9
:104C700076E005280BD1DFF81405012141700821E9
:104C8000017000214180052000F070F868E00628DE
:104C90000DD161796078A278120402EB0060E278AD
:104CA00000EB022022798018FFF7C5FE58E00728A4
:104CB00002D1FFF7D8FE53E0082803D16078FFF750
:104CC000E4FE4DE010284BD194F90100012802D0F8
:104CD000102822D041E0E07A217B090401EB00603A
:104CE000617B00EB0120A17B4318E079217A090464
:104CF00001EB0060617A00EB0120A17A4218E078B4
:104D00002179090401EB0060617900EB0120A179B0
:104D10004118A078C046C0461FE094F9020001285F
:104D20001BD10222E11C02A8FDF7F2FABDF808002F
:104D3000BDF90810C1F3072141EA0020ADF80800D1
:104D4000BDF90800FFF7A9F8DFF840040021417021
:104D500011210170BDF808104180052000F006F80F
:104D60000120DFF82814487100203EBD2DE9F043F2
:104D700087B004460020ADF80400DFF81054E8883E
:104D80000646012C0AD0C0F0AD81032C74D0C0F0CF
:104D90005A81052C00F03A8177D3A3E1DFF8FC7348
:104DA0000121C155411CE980DFF8F4030288120A91
:104DB00089B2CA55491CE980028889B2CA55491C82
:104DC000E980827889B2CA55491CE9804268121686
:104DD00089B2CA5501F10109A5F806904168091484
:104DE0001FFA89F909F8071009F10109A5F80690D9
:104DF000416809121FFA89F909F8071009F1010938
:104E0000A5F8069041681FFA89F909F8071009F119
:104E10000102EA808168091692B2D155521CEA80DB
:104E20008168091492B2D155521CEA808168091236
:104E300092B2D155521CEA80816892B2D155521C6F
:104E4000EA80C168090E92B2D155511CE980C2684E
:104E5000120C89B2CA55491CE980C268120A89B28B
:104E6000CA55491CE980C06889B2C855481CE88009
:104E70001020ADF8040035E10321C84A8154401CDC
:104E8000E8800120ADF804002CE1C44F0421C15595
:104E9000411CE980DFF80C83D8F80000000E89B2CD
:104EA000C855491CE980D8F80000000C89B2C855E3
:104EB000491CE980D8F80000000A89B2C855491C8D
:104EC000E980D8F8000089B2C85501F10109A5F8B8
:104ED0000690D8E90201382203F0EAFD1FFA89F9A9
:104EE00009F8070009F10109A5F80690D8E90201BF
:104EF000302203F0DDFD1FFA89F909F8070009F1F6
:104F00000109A5F80690D8E90201282203F0D0FD96
:104F10001FFA89F909F8070009F10102EA80D8E9C6
:104F2000020192B2D155521CEA80D8E90201000E6A
:104F300092B2D055521CEA80D8E90201000C92B21C
:104F4000D055521CEA80D8E9020180B2000A92B220
:104F5000D055521CEA80D8E9020192B2D055511CBA
:104F6000E980D8F81000001689B2C855491CE980BC
:104F7000D8F81000001489B2C855491CE980D8F847
:104F80001000001289B2C855481CE880D8F81010EB
:104F900080B2C155401CE880D8F81410091680B2C0
:104FA000C155401CE880D8F81410091480B2C155CE
:104FB000401CE880D8F81410091280B2C155401C7A
:104FC000E880D8F8141080B2C155401CE880D8F8A9
:104FD0001810090E80B2C155401CE880D8F818108E
:104FE000090C80B2C155401CE880D8F81810090A95
:104FF00080B2C155401CE880D8F8181080B2C15565
:10500000401CE8801920ADF804006BE0634F0521D7
:10501000C155411CE980287889B2C855491CE980EE
:10502000687889B2C855491CE9806888020A89B243
:10503000CA55491CE98089B2C855481CE88005203A
:10504000ADF804004EE0554F0221C155411CE980E6
:1050500055480288120A89B2CA55491CE98002885B
:1050600089B2CA55491CE9804268120E89B2CA55F4
:10507000491CE9804268120C89B2CA5501F1010944
:10508000A5F806904168090A1FFA89F909F807107E
:1050900009F10109A5F8069041681FFA89F909F894
:1050A000071009F10109A5F806908168090E1FFA99
:1050B00089F909F8071009F10102EA808168090CF1
:1050C00092B2D155521CEA808168090A92B2D15538
:1050D000521CEA80806892B2D055501CE8800B20A8
:1050E000ADF804000096BDF80430EA8821460FF2BE
:1050F000E410FFF741FB01206871E888B0F5807F7C
:105100002DDC264FF15D0FF20820FFF735FBBDF8CF
:105110000400C01CADF8040002A80FF21C211422E8
:10512000FDF706F9BDF80400C01CADF80B001A4CE1
:1051300001202070022201A9601CFDF7E9F801207E
:10514000E070207137206071BDF80400C21EF119B3
:10515000A01DFDF7DDF8214602A802F00BFB07B009
:10516000BDE8F0830C4901F58272C26160220270D1
:105170001422826001220273028200224282416173
:1051800010467047000000000888030000880300F4
:105190004CAA030050AA03002433030010A203000A
:1051A00058AD030008AC0300D0AB0300534C4320C0
:1051B0006F70656E0A000000534C4320636C6F7380
:1051C000650A0000736C632053656E644269674D25
:1051D0005347202564000000534C432067656F66E9
:1051E000656E6365206164642069643A25750A0010
:1051F000534C432067656F66656E63652072656D0D
:105200006F76650A00000000534C432067656F66A7
:10521000656E63652070617573652F726573756D5A
:10522000652025750A000000534C432067656F66B2
:10523000656E6365207570646174652069643A25E4
:1052400075207261643A2575207374733A25750A66
:1052500000000000534C432073746172742041526B
:10526000206D696E5F643A2575206D696E5F743AD2
:1052700025750A00534C432073746F702041520A05
:1052800000000000534C432063757272656E7420F9
:105290006C6F636174696F6E203A2025750A000097
:1052A000736C632053656E644269674D53472025D4
:1052B000642C2073746172743A256400736C6320EB
:1052C0007365742076616C756520256420256420E3
:1052D0000A000000534C432063625F747970653AA2
:1052E000256420675F73656E64696E675F636E74C3
:1052F0003A256420636F756E743A25642073746177
:1053000072745F706F696E743A2564200A00000041
:10531000534C4320675F627566666572203A2025AC
:105320006400000005000000000000000000000014
:105330000000000000000000050000000000000068
:1053400000000000000000000000000010B5002276
:105350004FF4A871DFF87C09FCF7ACFFDFF878495F
:10536000002218212046FCF7A5FF0020606210BD36
:105370000020704710B5DFF8644900F079FCA060A8
:10538000002204F11C012C2001F0F3FA002801D0C6
:10539000032010BD002204F11C01652001F0E9FA90
:1053A000002801D0032010BD002204F11C010120BF
:1053B00001F0DFFA002801D0032010BD002010BD4D
:1053C00010B5DFF81849002204F11C012C2001F06F
:1053D00026FB002801D0032010BD002204F11C018F
:1053E000652001F01CFB002801D0032010BD002225
:1053F00004F11C01012001F012FB002801D0032060
:1054000010BDFFF7A3FF002010BD000038B52DED43
:10541000028B84B09FEDB68ADFEDB58ADFF8BC4819
:10542000A0693C30A0612068022801D0032809D17E
:10543000DFF8AC080069216981420CDA401A08EEF5
:10544000100A08E0042802D1DFEDB78A03E005283E
:1054500001D1DFEDB68ADFF8880800692061DFF846
:105460007458B8EE480AD5ED530A30EE200A30EEF3
:10547000280A85ED530ADFEDAE0AB4EE600AF1EEBC
:1054800010FA09DBDFEDCF0A30EE200A85ED530A72
:105490000FF66400FFF770F9A06947F230518842B7
:1054A00014DBD5F84C0100F0CDFCCDE9020118EE7B
:1054B000900A00F0C7FCCDE9000118EE102A21681F
:1054C0000FF64800FFF758F90020A06104B0BDECCA
:1054D000028B31BD70B500F0B1F9FFF797FF00F016
:1054E0009BF900281BD0DFF8EC4704F5C470456831
:1054F000D4F88861701B03F0EAFA03462A46314665
:105500000FF63800FFF738F90020A060DFF8CC076D
:10551000DFF8CC171822FCF70BFF002070BD00F05D
:10552000E9F8002805D0DFF8B007416A41F004012E
:10553000416200F0FFF8002805D0DFF89C07416ABF
:1055400041F00101416200F019F9002805D0DFF8AF
:105550008807416A41F00201416200F035F90028F4
:1055600005D0DFF87407416A41F00801416200F09C
:1055700026F800F046F800F0B1F800F03DFA0020FF
:1055800070BD80B500F092FA002002BD3EB500A9C2
:1055900000231C461D4638C1002A00D100AA342829
:1055A00002D0352805D008E00621104600F014FB93
:1055B00003E00621104600F03DFB20463EBD38B515
:1055C000DFF81047DFF8100790F8240000F01B0008
:1055D00084F8400100F04CFB009004F241150422D5
:1055E00000A92846FCF794FE0421284600F032FB6F
:1055F00004F5A070DFF8E8160A6842714968817105
:1056000031BDFEB50026DFF8D446DFF8D456A868D1
:10561000A168401A00F08FFA029020682968884239
:1056200005D0029841F28831884200DB01260298B9
:10563000DFF8B016884200DB0126DFF89C0690F9FF
:105640001210002906D000218174416A41F0040142
:1056500041620126002E40D0DFF87866B06800EB8A
:1056600080018F1D00280BD1042204F1080106F1EE
:105670000D00FCF74DFE042106F10D0000F0EAFAE2
:10568000B068401CB06070742068B9190873781C49
:10569000471C0299DFF85026914203DB0221801952
:1056A000017302E0002180190173042202A9B819D4
:1056B0000C30FCF72DFE0321B8190C3000F0CAFAAB
:1056C00002980190A86800902B68A26821680FF2E8
:1056D0009060FFF751F8A868A060F7BDDFF8FC05FF
:1056E000DFF8FC154A6842600968016070470000F5
:1056F00000000000DFF8DC05DFF8DC1591F9001090
:10570000012903DA002181600846704781683B293E
:1057100005DA012905DB90F98401002801D0012078
:1057200070470020704700006ABCD43FFA7E2A3FD1
:105730004154094BDFF89C0590F98401002819D0E9
:10574000DFF8940590F90810012913DB90F9131084
:10575000012903D10021C17401207047DFF88005C1
:10576000DFF878150A6803689A4205D149684068ED
:10577000814201D10020704701207047DFF85805B1
:10578000DFF85C15DFF8542512680B689A4201D0E7
:105790000022027490F91020002A01D000207047E6
:1057A0001A46121892F90120012A01DA00207047E6
:1057B0004968012903DB0121017408467047002074
:1057C00070470000405409CB10B5DFF80C45DFF8F6
:1057D0001005DFF808150A6803689A4201D0002214
:1057E000627494F91120002A01D0002010BD0A68CB
:1057F000121992F90920012A01DA002010BD8068EF
:105800008968401A00F097F96169884202DB01203B
:10581000607410BD002010BD80B5DFF8B804D0F86A
:105820008C11D0F88801081A03F051F942F2117175
:10583000884201DB012002BD002002BD30B593B0DB
:1058400001A803F038FA00A804F00CFDFEF7D1FD22
:10585000012801D1012000E00020DFF8784484F81D
:105860008401D4F85001401C6FF0704190FBF1F1BD
:10587000C1EB0171401AC4F8500100F0F9F9DFF8EA
:105880006054A86068619DF80000042805D10420D8
:1058900028609DF80100686021E0BDF8060002283C
:1058A00010DB042802DB0320286001E002202860CE
:1058B000BDF80E0068609DED0F0ABDEEC00A85EDD3
:1058C000040A0CE0D4F85001042806DB012028600B
:1058D00001A800F013F8686001E00020286000F0E3
:1058E000C7F9D4F8501101EBD1725210A1EB42016B
:1058F00004EB8101C1F8880113B030BD2DE9F041FE
:1059000086B00446DFF8CC53D5F8506100A81421C6
:10591000FCF746FD00A9012004F02EFE0C207110BA
:1059200006EB91718910A6EB810100FB0151009AF1
:10593000C1F8542101F5AA71019A4A60029A8A605D
:105940000021324600E0521E331F934239DAD31C45
:105950005F1003EB9777BF10A3EB87035F1C4FEA41
:10596000670C07EB9C7C4FEAAC0CA7EB8C074FF065
:10597000000C0BE030EE600ADFEDAD0AB4EE600A19
:10598000F1EE10FA00DB01210CF1010CBCF1030F68
:10599000D9DA00FB075E0EEB8C08D8ED550A00FB48
:1059A000035E0EEB8C0E9EED550A9EED551A31EE00
:1059B000601AB5EE401AF1EE10FADBD530EEC00AEF
:1059C000DAE7C648C64A012901D1516941615169E6
:1059D0004069081A00F0AFF8C349884201DB022091
:1059E00007E06089022801D0012801D1012000E0F0
:1059F000002006B0BDE8F08170B5B74C606A10F0C9
:105A00001B0F23D0B34E00F01B0086F8400106F5B3
:105A1000A071E1610720608343202083B34D012002
:105A2000287068701A20A8700722E81CFCF770FC28
:105A3000606A20F01B006062608BC01C216A488293
:105A400029464320BDE8704004F0D6BC10F0240F76
:105A50002BD0A04E00F02400307306F10C00E06162
:105A6000B06800EB8000801D6083432020839F4D41
:105A70000120287068701A20A870628B06F10C0152
:105A8000E81CFCF745FCB1680FF2FC20FEF774FE41
:105A900000206062B060608BC01C216A4882294689
:105AA0004320BDE8704004F0A7BC70BD10B40128CD
:105AB00021D18A49884890F908200B6814461C4176
:105AC000E20703D5426A42F0010242621A46121806
:105AD00092F90120012A03DB426A42F0020242628B
:105AE0001946091891F90910012909DB416A41F0A9
:105AF0000801416204E0022802D10120764988743D
:105B000010BC704700B583B075494A688DF8012014
:105B10008A68CDF8022009688DF8001000A90622D5
:105B2000FCF7F6FB0EBD6B4890ED530ABCEEC00AC5
:105B300010EE100A7047002801D56D49081800289A
:105B400000D50020704780B5002805D0022825D058
:105B500009D3032825D001BD5F480272012A3AD13A
:105B60000121C17401BD012007E00B460341DB07A1
:105B700002D5594BC3185A70401C0628F5DB56480D
:105B800090F90510009190F9043090F9032090F9F4
:105B900002100FF20C20FEF7EFFD01BD4E4802701F
:105BA00001BD012007E00B460341DB0702D54A4B4C
:105BB000C3185A72401C0628F5DB474890F90510B7
:105BC000009190F9043090F9032090F902100FF23F
:105BD000F010FEF7D1FD01BDF8B504462578267911
:105BE000207A8DF80000607A8DF80100A07A8DF897
:105BF0000200012231462846FFF7A5FF364F032D4C
:105C000007D1E079217A083188404FF47A7148430E
:105C1000786100A8FEF741FC79690FF2C810FEF721
:105C2000ABFD324629460FF2D810FEF7A5FDF1BDB7
:105C30009B99993E38B5047805790022294620467B
:105C4000FFF781FF2A4621460FF2D410BDE8384005
:105C5000FEF792BD10B40022491E05E0135C0C5CF7
:105C600014540B54521C491E8A42F7DB10BC704777
:105C700000B583B00FF2C410D0E90023CDE90023B2
:105C800000A8FEF714FC9DF900001A499DF90120B7
:105C90004EF660235A4301FB00209DF902104FF499
:105CA0007A7211FB0200BDF9041000FA81F00EBDFA
:105CB000094908622831C161432101703C2181609A
:105CC00001210173018200214182084941610020C4
:105CD000704700001C990300AC3C03002040030007
:105CE00048AC030000BADB0020BF0200AC9D0300FB
:105CF000005C260580EE36004152204469737461D1
:105D00006E63652052657365740A0000534C6F63BF
:105D100041525F547970653A25642C20646973742C
:105D2000312025642064697374322025662C207329
:105D30002D446973742025660A0000002C20323639
:105D40002041542057726F6E672054696D657374DB
:105D5000616D70202564202564202564000000000A
:105D60002C203236204154204348474D4F44205B7D
:105D700025645D3A2564202D3E205B25645D3A252F
:105D800064202564000000002C203236204154207D
:105D9000626174636873697A65202564000000009D
:105DA0002C20323620415420616464496E744D6F5A
:105DB0006465202564202564202564202564000076
:105DC0002C203236204154206164644578496E7439
:105DD0004D6F64652025642025642025642025649A
:105DE000000000002C203236204154206578496E96
:105DF000744475726174696F6E2025642020000000
:105E00002C203236204154207265636569766553D3
:105E1000746172744D73672025642025640000004E
:105E20002C203236204154207265636569766545C1
:105E30006E644D7367202564202564000000000017
:105E4000000000005FF0FF0C1CEAD05114BF614558
:105E500006E0C110400721F0E04101F160517047B8
:105E600079B900F0004100020AD0B0FA80FC00FAD3
:105E70000CF001F16051A1EB0C5101EBD021400578
:105E8000704741020CBF40F4E0016FF000010020B8
:105E900070470000DFED4A0A60EE200AB0EEE01A1B
:105EA000DFED481A00B5B4EE611AF1EE10FA83B0D6
:105EB00036D5F5EE400AF1EE10FAACBFB6EE001A98
:105EC000BEEE001A70EE810AFDEEE00A10EE900AB6
:105ED000A8B1FAEEC90A9FED3C1A00EEC10A9FED87
:105EE0003B1A00EEC10A9FED3A1A00EEC10A9FED7F
:105EF000391A00EEC10A9FED381A00EEC10ADFED33
:105F0000370AB4EE600AF1EE10FA00F003003ADB53
:105F1000DFED330AB4EE600AF1EE10FA33D51FE07C
:105F20008DED000A0098C0F3C750FF2820D010B9AB
:105F30000098400241D08DED010A01A804F08EFBCB
:105F40009DED010ADFED250AB4EE600AF1EE10FACC
:105F500019DBDFED230AB4EE600AF1EE10FA12D578
:105F6000C0072AD5FFEE000A80EE800A03B000BD0C
:105F70000098400221D104F0E7FB212101609FED50
:105F8000190A03B000BD60EE000A9FED171ADFED9D
:105F9000171A40EE811AB7EE001A01EEA01A60EE51
:105FA000200ADFED131A00EEA10AC00746BF81EEFA
:105FB000000AB1EE400A80EE010A03B000BD000005
:105FC00083F9223F0000004F0000C94600A0FD40B9
:105FD0000020A23A000034330030C22EFEFF7FB909
:105FE00000008039FFFFFF7F6D161F3C1EB5DBBE32
:105FF0008329C4BDB0B581EA030C0CF0004C40F21B
:10600000FF7515EA11541DBF15EA1357AC42AF4294
:1060100039E0E41923EA455343F48013C90241F0FF
:10602000004141EA505EC7021100A7FB02020028AE
:106030004FF00000EEFB01204FF00001E3FB0721D1
:1060400018BF42F00102401800214941E3FB0E0154
:10605000A4F580640F0302D252004041494154F13B
:1060600001046CDD470872F1004250F1000051EB71
:106070000451A1F580115CBF41EA0C01B0BD4CEAAE
:1060800005510020B0BD05EA1357AC4214BFAF4222
:1060900041E050EA410E1CBF52EA430E02E0614665
:1060A0000020B0BD24423C441BD15FEA070EF6D06D
:1060B000090302BF01460020AEF1140EB1FA81F7C8
:1060C000AEEB070401FA07FE0C37C7F1200100FA16
:1060D00007F7C8404EEA000E23EA455343F4801305
:1060E000A2E733F00043B3FA83F704BFB2FA82FEAB
:1060F00077440B3FE41BB7F1200E2FBF02FA0EF3DB
:10610000BB40C7F1200E22FA0EFE38BF43EA0E0351
:10611000BA40641C82E750EA410E14BF52EA430EB3
:106120006FF000014FF4001717EB430F8ABF1946B9
:1061300017EB410FB5E74CEA05510020B0BDD4F193
:106140000104B4F120070FDAC4F12007520828BF78
:1061500042F0010210FA07F501FA07F7E1BF2A43FE
:10616000E0403843E1400FE0352C98DCC7F12004D3
:1061700052EA400220FA07F218BF42F0010231FA57
:1061800007F0A1400A43002172F1004250F10000E3
:1061900051EB0C01B0BD00004FEAF17CBCF1E04CCA
:1061A0002CBFBCF5001F11E05FEA4C0C34BFBCF102
:1061B0007F5F2EE05FEA9C0C4FEA0C1C4FEA3C0C20
:1061C000C10071F100414CEB50707047C90241EAC7
:1061D0005051C00218BF41F0010141F000414FEAA7
:1061E0006C50C0F10900212810D240EACC7CCCF1DF
:1061F000200C11FA0CF070F10040CCF1200C21FAC7
:106200000CF00CF0004C40EB0C0070474FEACC70E7
:106210007047490011F5001F04D84FEACC10FF3039
:10622000C0057047C817704710EE101A10EE902A7C
:10623000B0EEC00AC80F49005200F0EEE00A28BFD5
:106240000C3011F1807F38BF12F1807F0CD28A426E
:1062500038BF80F00400124214D034BF80EE800AB0
:1062600080EE200A04F076BA11F1807F08BF80F03A
:10627000040098BF12F1807F08D88A4214BF002220
:106280004FF07E5200EE102A04F064BA6FF0004125
:1062900000EE101A7047012004F0AEBA002004F09E
:1062A000ABBA000051EC100B00B500F003F841EC64
:1062B000100B00BD40F2FF7C0B0D4DD0634566D244
:1062C00030B421EA035141F4801103F2FD3C5FEA4E
:1062D0005C0C01D300184941890041EA90718000AB
:1062E0004FF440140023E202D50AB1F5100107D49F
:1062F0006D081DD2091B641900184941491BF7D5C7
:106300006D080AD20919641B00184941491BEFD5D1
:106310006D08F7D301E0520817D0C01861419B1AED
:10632000AC4100184941801AA941F4D452080AD05E
:10633000C01AA1419B186C4100184941801AA9411B
:10634000E9D45208F4D15B1C6C4161084FEA330078
:1063500001EB0C5130BC704750EA0103FBD030B464
:10636000B1FA81F311B9B0FA80F41B190B3BB3F108
:1063700020042FBF00FA04F19940C3F1200420FA51
:1063800004F438BF21439840D3F101039DE76345EE
:10639000E1D011F5801FDED850EA4101DBD0D943AE
:1063A00004F0E0BAF0B540F2FF7581EA030C0CF09E
:1063B000004C15EA11541DBF15EA1357AC42AF4209
:1063C000E5E0BC41C1F31301C3F31303801A994103
:1063D00043F4801304D2641E40004941801859419F
:1063E000C90241EA5051B1FBF3F603FB1611A2FBBF
:1063F0000675D7EBC020A94102D2761E80185941FC
:10640000C90241EA5051B1FBF3FE03FB1E11A2FB8E
:106410000E75D7EBC020A94103D2AEF1010E801852
:106420005941890241EA9051760546EA8E2EB1FB28
:10643000F3F603FB1611A2FB0675D7EB8020A941EA
:1064400002D2761E80185941C90241EA50514EEAE3
:10645000060EB1FBF3F603FB1611A2FB0675D7EB94
:10646000C020A94102D2761E80185941C90241EAD2
:106470005051B1FBF3F703FB1711A2FB0735D3EB28
:10648000C020A94167F100070CBF004247F0010797
:1064900066F3D5274FEA1E31B80814F5806412DD83
:1064A000BD0775F1004250EB0E5051EB045111F550
:1064B000801F5CBF41EA0C01F0BD4CF07F6141F0F0
:1064C000E0410020F0BDBD076D0840EA0E5041F4E8
:1064D0008011D4F10104B4F120060ADAC4F12006D7
:1064E0000200E04001FA06F3E1401843B2401543D0
:1064F0000EE0342C13DCC6F1200445EA40056D089B
:1065000020FA06F2154321FA06F0A1400D430021BE
:1065100075F1004250F1000051EB0C01F0BD00207C
:106520005FEA0C01F0BDCFB992185B41B3FA83F773
:1065300004BFB2FA82F6BF190B3FB7F120062FBF96
:1065400002FA06F3BB40C7F1200622FA06F638BF6E
:106550003343BA401CB1E419641E33E77F4231F083
:106560000041B1FA81F404BFB0FA80F6A4190B3CE3
:10657000B4F120062FBF00FA06F1A140C4F12006B5
:1065800020FA06F638BF3143A0403C1B1AE7AC4264
:106590001ABF05EA1357AF4212E050EA41061CBF8A
:1065A00052EA4306BFE750EA4107304661461CBF46
:1065B00041EA0551F0BD52EA430C08BFC143F0BDAA
:1065C00000204FF4001616EB410F98BF16EB430F57
:1065D00008BF16EB410F24BFC14305E016EB430F84
:1065E0000CBF61464CEA0551F0BD000070B44FF09D
:1065F000004591EA030F44BF6B4000F0C1B800BFF3
:10660000841A71EB030604D26E40001BB1411219CB
:1066100073414FF4001C1CEB410F34BF7CEB43066D
:1066200084E00C0DA4EB1356362E7DDC012E43DCEA
:1066300045EAC32343EA525312BFD20292025B08D7
:10664000240545EAC12141EA5051D2EBC0209941CD
:1066500025D407D1B0FA80F610FA06F164D00020F4
:10666000203608E0B1FA81F6B140C6F1200220FAE6
:1066700002F21143B0404FEAF474B4EB465434F0E4
:1066800001064FEA74040AD8D6F50016760D04F018
:106690000044F04061FA06F25040F1404840C00A20
:1066A00040EA415021F0004128BF5FEA500550F117
:1066B000000044EBD12137E045EAC323DB0A45EA79
:1066C000C121C90AB6F120050EDD42EA0242120CD0
:1066D000C5F1200603FA06F6EB4042EA06056D42D4
:1066E000984161F100010DE062FA06F5F240554073
:1066F00063FA06FC82EA0C02F3405A406D42904174
:1067000061EB030111F4801F05D1641E620502D004
:106710006D004041494121F48011430875F1004367
:1067200050F1000041EB045170BC70471CEB410F6D
:1067300015D223F0004352EA43060BD04FEA4C0C2B
:10674000BCEB410F04D80C0D661E342EB7DDEBE711
:10675000801A994150EA410608BF0021E4E708BFCA
:106760001CEB430F28BF6FF00001DDE770B44FF062
:10677000004591EA030C44BF6B40FFF741BF00BFE7
:10678000841A71EB030603D2001BB1411219734145
:106790004FF4001C1CEB410F34BF7CEB430443E07F
:1067A0000C0DA4EB1356352E50DC45EAC323DB0A4F
:1067B00045EAC121C912B6F120050DDD63FA05F6DF
:1067C000EB4086EA0305124218BF45F00105C018E8
:1067D00051F100010CD213E062FA06F5F240554087
:1067E000F3415A40B340F3405A408018594107D30F
:1067F00049085FEA30005FEA350528BF45F001052A
:1068000001F58011420875F1004250F1000041EBA2
:10681000045170BC4FF4001C1CEB410F38BF704793
:106820000020090D090570471CEB410F10D252EAF8
:1068300043060BD0BCEB410F05D80C0DAB43661ED5
:10684000342EB5DD02E0AB438018594170BC70476F
:1068500070BC70472DE9F04100242546DFF8207711
:106860001EE0052001F02AF80020F1690968884738
:10687000002804D02046441CC0B20228F1DBE4B258
:10688000032C0BDB0020317847F82100307857F8D3
:106890002000C8F80400304604F082F86D1C002483
:1068A000212D18DA2C2004F063F8064622462C210C
:1068B000FBF700FDDFF8CC86304658F835108847E6
:1068C000307847F8206008EBC508307857F820008A
:1068D000C8F80400C8E72046BDE8F081DFF8A0163C
:1068E000D1F88411082807D1002903D091F8280095
:1068F000002803D1012070470029FBD100207047F8
:1069000010B46FF000410846002214E0DFF8703642
:1069100053F82230002B0DD01C6A002C0AD0DB78F3
:10692000002B07D1E368052A01D1042B02D098423D
:1069300000DD1846521C692AE8DB082801D010281F
:1069400000D10420884200D1002010BC704710B54F
:106950000C468168002901D0A1606160C0780128DF
:1069600001D1002060606068FDF7D8FD6060A06024
:1069700010BD2DE9F04184B0044615462646DFF8E7
:10698000000650F8267008788DF8000048680190DD
:1069900088680290002F01D103203DE000A938460D
:1069A000FFF7D5FF00A907F1200004F0D9F807F19F
:1069B0001C0898F80C00012807D10020F9694968E3
:1069C0008847204603F0FFFD09E03879012806D109
:1069D0009DF80000002802D1204600F044FA2A4623
:1069E00000213420FB691B699847F878002804D1FE
:1069F000DFF89415022004F02DF9D8F808000028DB
:106A000001D0012300E0002398F80C2031460FF25A
:106A10008450FDF7B1FE002004B0BDE8F081FEB562
:106A200006461446DFF8580550F8265008788DF8C9
:106A300000004868019088680290002D08D005F198
:106A40001C079DF8000000280AD1B868002801D171
:106A50000320FEBDC0680190B8680069029003E0A1
:106A600000A92846FFF773FF00A905F1200004F0F4
:106A700097F8EB69387B002803D10020D968884754
:106A800004E02246002135201B699847DFF8F814FE
:106A9000022004F0DFF8B868002801D0012300E0EC
:106AA00000233A7B31460FF2F840FDF765FE0020E7
:106AB000FEBD2DE9F04106460C461546DFF8C00440
:106AC00050F826703846FFF742FF002F05D007F137
:106AD0001C08D8F80800002801D103202BE0C16869
:106AE0006268914205D10169A268914201D10020FA
:106AF00021E000F1080107F1200004F051F800281E
:106B000018D1214607F1200004F02AF82A46002176
:106B10003620FB691B699847DFF86C14022004F0EB
:106B200099F898F80C2031460FF28040FDF724FECA
:106B3000002000E00320BDE8F08110B50C461146AE
:106B40001A46DFF83C3453F82030002B01D10120E5
:106B500010BD2046DB691B699847002010BD10B5A9
:106B60000C4611461A46DFF8183453F82030002B33
:106B700001D1012010BD192C03D1012100F09FF992
:106B800003E02046DB695B699847002010BD0146A1
:106B9000692901DA002801D100207047DFF8E003FD
:106BA00050F82100704710B582B000218DF8001018
:106BB000082804D0102824D0202826D013BD00AAED
:106BC00001213720DFF8B8335B68DB695B699847E0
:106BD0009DF80000800703D50021012001F0C1FECF
:106BE0009DF80000400703D50021022001F0B9FE06
:106BF0009DF80000000720D50021032001F0B1FE20
:106C000013BD042001F0ADFE13BDDD48046AFDF79D
:106C100037FCE2699268904700280AD1606A002830
:106C200007D0C1680069814203D10021082000F02B
:106C300046F90021084601F094FE13BD2DE9F0410C
:106C400086B0044601A80FF29C311422FBF770FBBA
:106C5000FDF7C9FB012801D1012500E00025CB4E3D
:106C6000C6F80042002730E069281BDA0120BDF891
:106C700007108855022200A9BDF807008019401CA2
:106C8000FBF746FB08F11001BDF807008019C01C96
:106C900004F025F8BDF80700BDF80010C91C08185D
:106CA000ADF80700214608F1200003F096FF062FFB
:106CB0000AD1BDF80700002806D0314601A800F02F
:106CC00059FD0020ADF807007F1C212F77DAAD4871
:106CD00000EBC700D0F80480B8F1000FE7D098F8B7
:106CE00028000028E3D098F803000028DFD1D8F866
:106CF00020004069001B012805DAFDF7C1FBD8F828
:106D00001C2092689047D8F824000028CAD08069D7
:106D1000001B0128C6DA002D03D098F80C000028CB
:106D2000C0D008F1100004F016F8ADF8000008F12A
:106D3000100004F01DF8ADF802000028B2D0BDF834
:106D40000700BDF8001011FA80F2101DB0F5007FA9
:106D50000CDD0FF264210FF27420FDF70DFD3146BA
:106D600001A800F007FD0020ADF8070098F800002A
:106D70002928BFF679AF3720BDF80710885598F855
:106D80000000BDF807108919487002220DF10201B8
:106D9000BDF807008019801CFBF7BAFA08F1100152
:106DA000BDF807008019001D03F099FFBDF807002A
:106DB000BDF80010091D0818ADF8070072E7BDF80E
:106DC0000700002803D0314601A800F0D3FC0020C2
:106DD00006B0BDE8F08170B5694951F82050002D2A
:106DE00026D06B4C2078401C2070802080F31188C6
:106DF00000BF00BF6078401C60702E6A09E006F199
:106E000008012846FFF7A3FDF06870613069B061A2
:106E10007668002EF3D16078401E6070C0B2002802
:106E200002D1002080F31188BDE8704001F038B82D
:106E300070BD534951F82000C178002905D10221C5
:106E4000C1705149022003F005BF70474C4951F809
:106E50002000C178022905D10021C1704A490220D1
:106E600003F0F8BE704770B586B0044601A80FF273
:106E700088111422FBF75CFA414850F82400458A37
:106E80000120ADF80000281D03F072FD06463720F2
:106E900030707470022200A9B01CFBF739FA311D62
:106EA000204603F069FB281DADF80700314601A814
:106EB00000F060FC304603F073FD06B070BD2DE9B4
:106EC000F04186B004460D462D4850F8246001A8D4
:106ED0000FF238111422FBF72BFA06F1100003F021
:106EE0003AFF074606F1100003F042FFADF800003C
:106EF000002F01D1002D3FD0002D01D0032000E054
:106F00000020002F01D0391D00E00021081803F0F7
:106F10002FFD8046002F13D0372088F8000088F816
:106F20000140022200A908F10200FBF7F1F906F185
:106F3000100108F1040003F0D2FE381DADF807007F
:106F4000002D12D00520BDF8071001F8080001201F
:106F5000BDF8071041444870BDF8070040448470F4
:106F6000BDF80700C01CADF80700414601A800F0BD
:106F700001FC404603F014FD06B0BDE8F0810000BE
:106F8000789703004034030080580300088A030008
:106F9000A03D030023612025642C25642C2564007A
:106FA00023722025642C25642C256400236320256E
:106FB000642C256400000000636F6C6C6563745F73
:106FC00073656E736F725F646174610025733A203C
:106FD00074785F646174612069732066756C6C28D5
:106FE00025642900050000000000000000000000EA
:106FF000000000000000000005000000000000008C
:10700000000000000000000000000000050000007B
:107010000000000000000000000000000000000070
:1070200030B583B005460FF2AC10FDF7A5FB95ED2A
:10703000020B8DED000BD5E900230FF2B010FDF728
:107040009BFB95ED060B8DED000BD5E90A230FF2A6
:10705000B810FDF791FB296B0FF2D810FDF78CFBF0
:10706000554C95ED000B84ED000B95ED020B84ED76
:10707000020B95ED040B84ED040B95ED060B84EDEE
:10708000060B00200146C4E90801D5E90A01C4E95C
:107090000A01286B2063FDF7F3F9A06337BD0021D7
:1070A000454A006882F83C0092F83C3003E0401CFE
:1070B0009842FCDB491C082901DA0846F8E77047CA
:1070C00010B50FF28410FDF757FB3B4C00226821EE
:1070D0002046FBF7EFF89FED390B84ED000B84EDB4
:1070E000020B00203749087010BD000038B5354C40
:1070F00094F9000000281BD12F4D0022682128465A
:10710000FBF7D8F89FED2D0B85ED000B85ED020BFD
:107110002D4800F08DF92D4800F08DF9012000F088
:107120009CF9014694F900200FF22C10FDF724FB86
:1071300094F90000002803D4401C2070002032BDC8
:10714000032032BD38B51F4C94F900100FF22810FF
:10715000FDF712FB94F90000012814DB401E20709B
:1071600040B200280DD100F095F9054600F069F90C
:1071700000F06BF994F9002029460FF21010FDF78A
:10718000FBFA002032BD032032BD002070470020F2
:107190007047002070470E4901F10C02C26168225D
:1071A00002702422827001220282092242824161FD
:1071B000002070470048704768A7030000000000E7
:1071C000000069400DAE0300218000009F80000098
:1071D00068420300534C4356204C5349206F6E4C79
:1071E0006F636174696F6E4362000000534C4356D5
:1071F000204C5349206C61743A2025662C206C6F1A
:107200006E3A2025660A0000534C4356204C5349E1
:107210002074696D657374616D703A20256C6C75AE
:107220002C207370656564286D2F73292025660AEC
:1072300000000000534C4356204C534920657272A5
:107240006F723A2025750A004C53492067707320ED
:10725000696E6974000000004C534920476E7373D7
:107260005374617274207265742025642C20636EDF
:10727000742025640A0000004C534920476E737344
:1072800053746F70203A2025640000004C5349204D
:10729000476E737353746F70207265742025642C6D
:1072A00020636E742025640A00000000F446400D3F
:1072B00040EAC120490006D200F014F8004248BF5D
:1072C0006FF00040604700F00DF84FF00041884239
:1072D0008CBF084640426047400D40EAC12049004B
:1072E00080F00D8040F00040490DA1F58061491CFF
:1072F00005D4D1F11F0154BFC840C01770474FF0EB
:107300000000704710B54FF4016003F031FB0446F4
:1073100006E04FF401632246DFF8040300F019F998
:107320004FF40161204604F025F801281BDB40F2F0
:1073300045318842EDD040F2454188420BD047F2BA
:107340000A118842ECD14FF401632246DFF8D002E3
:1073500000F07CF9E4E74FF401632246DFF8C00255
:1073600000F0DAF9DCE72046BDE8104003F018BB76
:107370002DE9D0030446DFF8AC82DFF8AC92A8FB1D
:10738000046709FB0477DFF8A402E0FB0167DFF87C
:10739000A002DFF8A01230187941DFF89C32A3FB7D
:1073A0000223801A9941BDE8D00370472DE9F041CE
:1073B00086B004460D4616461F4600208DF815007F
:1073C00001208DF814000020ADF81000002F06D029
:1073D0001820ADF80E0000208DF80C0005E002200A
:1073E000ADF80E0001208DF80C004FF47A70684360
:1073F00002908DF8124070008DF81300102202A93F
:1074000040F2654003F044FF8046019700962B460A
:1074100022460FF220310FF22C3004F04BF8B8F175
:10742000010F01DB012000E0002006B0BDE8F08183
:107430007B49486070477A4988607047784908609E
:107440007047002076494860704700207449886082
:107450007047002072490860704771494A68002AE5
:1074600001D0002801D5002070470246521E9241EB
:10747000D20F8A7501220A750861887D002804D020
:1074800000231A460121104690E700231A46096995
:1074900010468BE762480021817501750161417DCD
:1074A00000230A46184681E7014600205C4A13681B
:1074B000002B07D05175117D002903D1517D034662
:1074C0000A4673E7704756480021016041608160B9
:1074D000C16081754175012101760021C17504F0FB
:1074E00002B8000030B400229FED4C0A134690F918
:1074F000044002E041F82220521CA242FADB012C97
:1075000025DB1A461DE051F8245000EB0515D5ED9A
:10751000030AB4EE600AF1EE10FA02D5B0EE600A8A
:107520002346641C90F90450AC42ECDB51F8224035
:1075300051F8235041F8225041F823409FED370A7B
:10754000521C90F90440A24201DA1446EAE730BC2A
:10755000704770B504461646002C5DD0002E5BD0F7
:10756000382003F005FA0546307900F03F003F2847
:107570004DD1F06800F048FD4FF403722F4BFEF739
:1075800039FDC5E90001306900F03EFD6FF0E7020A
:107590002B4BFEF72FFDC5E90201706900F034FDA9
:1075A0000022284BFEF7FEFEC5E90401708B00F0B7
:1075B00035FD0022244BFEF7F5FEC5E90601B08B30
:1075C00000F02CFD00221F4BFEF7ECFEC5E9080180
:1075D000308B28637279B168F088FFF7C9FEC5E97E
:1075E0000A01207D002805D0616808000AD02846DD
:1075F000884707E0607D002804D02168080001D09A
:1076000028468847A07D002801D0FFF743FF284681
:10761000BDE8704003F0C4B970BD00000000000078
:1076200024AB0300000029F90F26020040420F009E
:10763000000087C14F88620400CA9A3B0080663E02
:10764000FF7F763E0000244000005940F0B5C1B0F5
:1076500004461546A06800285CD0002D5AD00027AB
:1076600040F2044003F084F9064600A92846FFF7DB
:1076700039FF3846306041E000A850F8271005EB8C
:10768000011191ED030AB5EE400AF1EE10FA34DD76
:10769000316806EB011181ED020A50F8271005EB65
:1076A0000111097A326806EB0212117150F82710A5
:1076B00005EB0111497A326806EB0212517150F85C
:1076C000271005EB01110969326806EB02121161FE
:1076D00050F8271005EB01114969326806EB0212D8
:1076E000D16050F8270005EB0010807A316806EB76
:1076F000011188713068401C30607F1C95F90400CE
:107700008742B9DBA168080001D03046884730467F
:1077100003F046F941B0F0BDC168080009D0002A65
:1077200007D0080005D01278501E8041C043C00F1A
:107730000847704773656E644C6F636174696F6E60
:10774000526571005B495D5B202573205D20696493
:107750003A257520726174653A256C6920706173F1
:10776000736976653A257520617661696C3A25758D
:107770000A0000002DE9F04705460E46B5F80370F3
:10778000334C2078401C2070802080F3118800BF8B
:1077900000BF6078401C60702878052803D1FDF791
:1077A00033F8804601E04FF0000808EB070000F1D5
:1077B0000D0A504603F0DCF88146B9F1000F11D1F3
:1077C00051460FF2940003F075FE6078401E607021
:1077D000C0B2002802D1002080F31188BDE8F04734
:1077E00000F05EBBB5F803004044A5F803000D228D
:1077F00029464846FAF78CFD3A46314609F10D0014
:10780000FAF786FDB8F1000F04D007EB09000D3040
:10781000FDF703F8B5F8030000F10D0189B2484601
:1078200000F050F96078401E6070C0B2002802D1AC
:10783000002080F3118800F033FBB9F1000F04D071
:107840004846BDE8F04703F0ABB8BDE8F08700005C
:10785000A03D030000F030B9747862756666657209
:10786000206973206E6F7420616C6C6F6361746546
:10787000642825642921210A00000000D2B2203AA0
:1078800022BF00FA02F1002070475242D041D2F1EB
:10789000200291404140D04090404140704700005C
:1078A00010B5DFF85043002208212046FAF702FD08
:1078B000204610BDDFF83C037047000038B5044691
:1078C00004F05AF84FF47A726243841851EBE2756F
:1078D00000BF00BF00BF00BF00BF04F04DF8A942C9
:1078E000F6D301D8A042F3D331BDB1F5805F03D107
:1078F0000121042004F05BB97047B1F5805F03D12A
:107900000021042004F053B9704738B50446FCF751
:10791000B7FDDFF8E422C2E90801002C27D0DFF828
:10792000DC020078002822D0DFF8D4422078401C06
:107930002070B44D2878401C2870B349102003F003
:1079400089F9802080F3118800BF00BF2078401E95
:1079500020702878012804D16868002801D004F03C
:1079600073FA2878401E2870002080F311881B20AD
:10797000BDE8324004F0C2B938B50446FCF780FDDA
:107980009D4AC2E90601002C25D09C4800780028B9
:1079900021D09B4C2078401C20709A4D2878401CA8
:1079A00028709949082003F055F9802080F3118848
:1079B00000BF00BF2078401E20702878012804D125
:1079C0006868002801D004F03FFA2878401E28702B
:1079D000002080F311881C20BDE8324004F08EB9ED
:1079E00038B50446FCF74CFD834AC2E90001002C7F
:1079F00025D182480078002821D0814C2078401C75
:107A00002070804D2878401C28707F49202003F08A
:107A100021F9802080F3118800BF00BF2078401E2C
:107A200020702878012804D16868002801D004F06B
:107A30000BFA2878401E2870002080F3118820203F
:107A4000BDE8324004F05AB980B5002812D00328AE
:107A500018D16E48009000231A4603211C2004F020
:107A600019F96B48009000231A4603211B2004F0EB
:107A700011F901BD6748009000231A460221202019
:107A800004F008F901BD80B5FFF70AFF04F002FA1F
:107A9000BDE80140CAE080B50846FCF7ADFC5E4990
:107AA0005E4804F01FFA002805D00FF29410BDE8DC
:107AB0000240FCF761BE01BD0023594A40215648EF
:107AC00004F06EBABC230FF2881204F034BAF8B591
:107AD0000C4615461E4605274A480178491C017088
:107AE000002004F04DFB002806D133462A462146EB
:107AF000002004F048FB074600F0D2F93846C0B237
:107B0000F2BDF8B50C4615461E4605273D480178DE
:107B1000491C0170002004F033FB002806D13346D5
:107B20002A462146002004F030FB074600F0B8F951
:107B30003846C0B2F2BD02280BD0052809D006286D
:107B40000BD0082807D00E2803D01D2803D02228E8
:107B500005D1042070470720704709207047002096
:107B600070472DE9F8430C4615461E46052740B2DE
:107B7000FFF7E1FF804615F8019B22480178491C78
:107B800001702849404604F0CAFB002808D100953E
:107B9000731EDBB24A466108404604F0D6FB074636
:107BA00000F07EF93846C0B2BDE8F2832DE9F0411D
:107BB00082B00C4615461E46052740B2FFF7BBFFB4
:107BC000804610480178491C01701649404604F06F
:107BD000A6FB002807D10096089B2A46610840466C
:107BE00004F09EFB074600F05BF93846C0B2BDE8E2
:107BF000F681000098AD030040AB03000FAE030018
:107C000011AE0300A03D03008058030079890000F5
:107C10000B890000E189000028A9030084530300B8
:107C2000978A0000801A060003F08EBE80B5FFF729
:107C300041FE01210170C1704171817101BD0000DF
:107C40004D534720426F782046756C6C0000000051
:107C500073746172745F74785F73747265616D00C0
:107C600030B4802080F3118800BF00BFDFF8941388
:107C7000886800220A7182F3118800281CBF0268FC
:107C8000002A33D0436954699C422FD100E0224638
:107C90001468A4B165699D4211D12246146874B17B
:107CA00065699D420BD12246146844B165699D42C5
:107CB00005D12246146814B165699D42E7D080233E
:107CC00083F3118800BF00BF03680C69844208BFBA
:107CD0000B61016A0B60196202621168016001B1F7
:107CE0000862106092F8290082F82800002080F3D2
:107CF000118830BC704730B5DFF808430020607150
:107D000081B0206AE16900F18040606208001CBF18
:107D100020468847002080F31188E56808E0E8687D
:107D2000616A411A48BF6062002080F311882D68A3
:107D300005B3802080F3118800BF00BF206920B107
:107D4000686921694969884219D3287C4007EBD5C5
:107D5000E868216A401A0128E1DA284600F0BCF8F8
:107D6000802080F3118800BF00BF287C0028D6D176
:107D700001B030BD802080F3118800BF00BF01B08A
:107D800030BD000070B5DFF87C420020607001203B
:107D90002070E06B68B1802080F3118800BF00BFC5
:107DA000E06B8047002080F31188E063606384F813
:107DB0003800A06800281CBFC16A002904D00968E7
:107DC0000A001CBF4068884794F8310040B1A068A1
:107DD00094F8301080F82810207908B1FFF740FFA0
:107DE000206948B304E028682061002080F31188EE
:107DF000802080F3118800BF00BF25690DB32E7C61
:107E0000FEB170070ED5E868216A411A012905DA2A
:107E1000284600F061F8287C20B90DE0616A411A1B
:107E200048BF606206F0FB001028DCD1A8688068BB
:107E30004068007C0028D6D1802080F3118800BFE4
:107E400000BF607950B9206900B32069007C002828
:107E5000206909D080688068406805E0FFF74BFF23
:107E600060790028FAD1EEE7A060A068C16A21B16C
:107E700049680A001CBF40688847A06890F828003D
:107E800084F8300084F83100204670BD84F8310059
:107E900084F83000A060207080F31188204670BD07
:107EA00010B5584C2078401E2070C0B298B9606858
:107EB00088B1802080F3118800BF00BF606830B1B6
:107EC00001202070204603F0ACFF00202070607875
:107ED00008B980F3118810BD30B581B08168494C74
:107EE00041B1226AC2600A68496802B151600A6001
:107EF00000218160017C11F00301017426D1216908
:107F000091B92061207838B901202070204603F013
:107F100088FF0020207001E0012060716078A8B91E
:107F200080F3118801B030BD42694B699342E8D3B8
:107F30008142E7D09A4209D103461B68002BEDD05D
:107F40005D69AA42EAD18B42F7D1DAE701B030BDD0
:107F500030B52C4C227881B04169521C227004F15A
:107F60000C0200E01A461368A3B15D69A94211D260
:107F70001A46136873B15D69A9420BD21A46136899
:107F800043B15D69A94205D21A46136813B15D6910
:107F9000A942E7D303600262106043B118625A69D4
:107FA0008A420CBF90F82910002180F82810017C2B
:107FB00051B9802181F3118800BF00BFFFF78CFF0A
:107FC000607808B980F3118801B0BDE8304067E7F8
:107FD00030B50C4C2578681C207081B0204603F029
:107FE00020FF6078257008B980F3118801B030BD9A
:107FF00000B581B004F020FA02480121017001B0FF
:1080000000BD0000A03D0300010040F10980F446DE
:10801000404200F005F851F000416047010000BF08
:1080200009D0B0FA80F18840C91CC1F58461090506
:1080300001EBD0214005704780B54FF0FF3251EC85
:10804000100B04F015FA41EC100B01BD000000000C
:108050002DE9F8452DED088B0FB486B040F2FF7185
:1080600007989DED080B8DED040BC0F30A50884274
:1080700008D107980024000305BF069800280225B0
:10808000012512E0012807DA06A804F0A1FB012867
:1080900002DB0024002508E0079A40F2FE3161F37C
:1080A0001E520792441A4FF0FF35002104A804F035
:1080B000B0FB1A9F06460FB10020388036B9DDE9C3
:1080C00008230020002104F0E3FB12D0002D13D57B
:1080D00024B2012C15D1DDE906230020DFF88C1332
:1080E00004F0D6FB05D0012E0BD1DF4904F0D0FB04
:1080F0003ED10AB0CD49E8E1022D04D1DDE9060107
:10810000E2E1012E6FDB022E08BFDDE9080100F07D
:10811000DB81012D2AD107980028099806D4002870
:1081200054BF9FEDD50B9FEDD60BCBE100280ED4AD
:1081300056B94FF0FF3104A804F06BFB002848BF8C
:108140009FEDD10B00F1BE819FEDCB0BBAE156B98B
:108150004FF0FF3104A804F05CFB002848BF9FEDFE
:10816000B40B00F1AF819FEDC60BABE1012E11D135
:108170000998002824B206D4012CACBF9FEDBE0B99
:108180009FEDBF0B9EE1012CACBF9FEDBD0B9FEDA2
:10819000BA0B97E10998002810D466B94FF0FF3167
:1081A00004A804F036FB002842BF079800289FED82
:1081B000A00B00F187819FEDB20B83E102F0C4FABE
:1081C0002221016066B94FF0FF3104A804F021FBC1
:1081D000002842BF079800289FEDAB0B00F1728189
:1081E0009FEDA50B6EE10798002848BF002E0CD527
:1081F00002F0AAFA212101600AB04FF0FF30BDEC75
:10820000088B6FF00041BDE8F485DDE9060100222E
:10821000002304F04DFB38BF002509D381F0004155
:10822000CDE906014FF0FF3104A804F0F2FA05464B
:10823000012C13D1DDE906017F4A804B04F050FB8D
:108240000CD2DDE9062300269FED7D8B00204FF048
:108250008041FDF7CFFECDE906011CE0DDE90623F4
:108260009FED798B00207A49FDF7C4FE53EC182B63
:10827000FEF77CFAFFF71AF8A0F120063046FFF768
:10828000C3FE0022734BFDF7B5FE53EC182BFEF72F
:108290006DFA41EC180B0FF2582000EB461ADDE99D
:1082A000060153EC182BFEF7A1F9DDE9062341EC9A
:1082B000190B51EC180BFEF759FA02460B4651EC1C
:1082C000190BFEF76FF841EC1A0B53EC1A2BFDF764
:1082D00091FE41EC1B0B8DED069B04F0FBF953EC7A
:1082E0001B2BFDF787FEDDE90623FEF77FF9064627
:1082F000884600204D4953EC182BFEF777F90022F1
:108300004FF08043FDF776FE32464346FEF72EFAE5
:1083100053EC1A2BFDF76EFEDDE90623FEF726FA75
:1083200041EC180B4C4A4D4BFEF73CF8CDE90401EB
:108330002046FFF769FE41EC190BDAE9000153EC26
:10834000192BFEF713FADDE90423FEF70FFACDE946
:108350000401DDE90823FDF74DFE0022404BCDE985
:10836000020104F0BDFAC0F0938001223D4B04F0FD
:108370009FFA40F291800022002304F0B1FADDE977
:10838000022339BF0020384900203849FEF7EEF9B2
:10839000FEF78CFF0446DDE9080153EC182BFDF7CE
:1083A00029FECDE90201DAE90223DAE904019FEDB1
:1083B000308BFEF7DBF9DDE90823FDF71BFE53ECFC
:1083C000182BFDF717FEDDE90223FEF7CFF9CDE903
:1083D0000201DAE9002351EC190BFEF7C7F9DDE9D8
:1083E0000823FDF707FE064688462046FFF70CFEE9
:1083F00002460B4630464146FEF7F8F853EC182B80
:10840000FDF7F8FDDDE90223FEF7B0F9CDE9020141
:108410000FB13C80002400940022044B02A804F019
:1084200077FAA8B3012837D042E000BF0000F03F40
:108430000000000000000080CD3B7F669EA0E63F6C
:10844000000000000000F03F000000000000E03FDE
:10845000000050400000903FEF39FAFE422EE63F08
:108460000000E0C00000E0400000E0BF0000E03F8E
:10847000EF39FAFE422EE63F000000000000F07FD8
:108480000000000000000000000000000000F0FFFD
:108490000020CDE9020007E00020014902E000BF12
:1084A0000000F07FCDE9020102F04EF922210160C7
:1084B000002D1DBFDDE9020181F0004141EC100BF0
:1084C0009DED020B51EC100B0AB0BDEC088BBDE822
:1084D000F48580B50020009053EC112B51EC100B6B
:1084E000FFF7B6FD41EC100B01BD000000000000DD
:1084F000000000000000F0BF00000000000000804D
:1085000000000000000000800000000000000000EB
:10851000000000C05294EEBF00000048204E51BE43
:10852000000000F86467BCBC000000000000000010
:10853000000000208133EDBF00000080B3DB14BEDB
:10854000000000506706A3BC00000000000000000F
:10855000000000D0E9DCEBBF00000008C39259BE68
:1085600000000080B0D3B8BC000000000000000094
:1085700000000070F98FEABF000000C0A51028BEFF
:10858000000000E8BFC0B0BC000000000000000018
:1085900000000070284CE9BF00000060134B42BE91
:1085A000000000C03D20B8BC00000000000000003A
:1085B00000000050FA10E8BF000000C05FF62BBEBC
:1085C000000000905C71A7BC0000000000000000EB
:1085D00000000020FCDDE6BF000000C0F8F154BE42
:1085E00000000018E9F6B9BC00000000000000001F
:1085F000000000D0C3B2E5BF00000070E43254BEFA
:1086000000000050DB06B4BC0000000000000000C9
:1086100000000010EF8EE4BF00000020F36252BEA5
:10862000000000C02A879ABC000000000000000083
:10863000000000B02272E3BF000000F0E8E056BE88
:1086400000000028352DBDBC000000000000000027
:10865000000000000A5CE2BF000000B0FA8E41BEDC
:1086600000000040AE6FBDBC000000000000000034
:1086700000000000564CE1BF000000F015CD5FBEC9
:1086800000000000141C90BC00000000000000006E
:1086900000000040BD42E0BF00000030F93457BE8A
:1086A000000000E06C1E93BC000000000000000011
:1086B000000000E0F57DDEBF000000B08A535EBE22
:1086C00000000080DA77AABC000000000000000073
:1086D000000000C09D81DCBF00000000FFA226BE9C
:1086E0000000006057E2B0BC000000000000000085
:1086F00000000060F98FDABF000000580A8151BE07
:10870000000000F05F60B8BC000000000000000046
:108710000000000098A8D8BF000000607A7F45BE26
:10872000000000D05433A3BC000000000000000093
:10873000000000600FCBD6BF000000D091CB40BE40
:10874000000000406D1BA0BC000000000000000005
:10875000000000A0FBF6D4BF00000098C5CE52BEBA
:10876000000000003A397EBC00000000000000005C
:10877000000000E0FE2BD3BF0000004073872BBE3B
:1087800000000000926879BC0000000000000000BA
:1087900000000040C069D1BF00000058F16353BE23
:1087A00000000080438D7CBC000000000000000041
:1087B00000000080D85FCFBF000000181F8354BEA8
:1087C000000000B03F42A2BC00000000000000001A
:1087D0000000008067FCCBBF00000060FAFF53BEC2
:1087E00000000050E00DB8BC0000000000000000D8
:1087F0000000000098A8C8BF000000607A7F35BE66
:10880000000000C0543393BC0000000000000000D2
:1088100000000000DC63C5BF00000058D6FF54BE56
:1088200000000000396490BC00000000000000005F
:10883000000000C0AD2DC2BF00000080A45915BECD
:10884000000000E0484BABBC00000000000000004E
:10885000000000801A0BBEBF00000050BF3C5ABE93
:10886000000000A0B364B6BC0000000000000000DF
:108870000000008004D6B7BF00000040BBCF36BE6A
:108880000000008076CEA8BC0000000000000000C0
:108890000000008032BBB1BF000000402A0043BE90
:1088A00000000028C60CBDBC000000000000000055
:1088B000000000009473A7BF000000182B3B59BEB6
:1088C000000000C0E55DA5BC000000000000000045
:1088D00000000000EE4397BF000000A0E6C340BECA
:1088E00000000020958DB5BC0000000000000000D5
:1088F0000000000000000080000000000000008078
:1089000000000000000000800000000000000000E7
:10891000506002604160086070470A68F8E748608C
:108920000160704701684068F9E7002007E03649B8
:1089300001EBC00241F8302011464960401C072875
:10894000F5DB704710B402680B4600E01268824203
:1089500004D09468A342F9D1104600E0002010BC76
:1089600070472DE9F04104460D462646264F57F83C
:10897000368008E0D8F80820100002D029462046AA
:108980009047D8F8008007EBC6008045F2D1002060
:10899000BDE8F08138B50C46072801DA210007D17F
:1089A000224601460FF2640002F084FD032032BD2E
:1089B000154901EBC00521462846FFF7C3FF0028F3
:1089C00006D10C2001F0D4FF84602946FFF7A5FFF3
:1089D000002032BD70B504460D460B4800EBC400C4
:1089E000FFF7B0FF060007D12A4621460FF23400F8
:1089F00002F060FD032070BDFFF794FF304601F0E8
:108A0000CFFF002070BD0000E8A9030061626E6F17
:108A1000726D616C20726567692028256420257855
:108A20002900000061626E6F726D616C20756E725C
:108A30006567692825642C257829000008B584B06D
:108A40000023029311B90093019302E00090481EA5
:108A5000019004AB00A907487844183004F0BCF832
:108A6000009911B1009A00211170002858BF029896
:108A700005B000BD1399FFFF00F10103810704D089
:108A800010F8011B89B18107FAD10268B2F10131F6
:108A9000914311F0803F04BF50F8042FF6E710F81F
:108AA000011B11B110F8011BFBE7C01A7047000051
:108AB000D2B2203A22BF21FA02F0002170472032C0
:108AC000D141D04048409140D140484070470028B3
:108AD00048BF404270470000DFF81009C17B00EB3F
:108AE000810181ED050AC17B00EB8101C1ED090A1D
:108AF000C17B00EB810181ED0D1A017C042901DAB3
:108B0000491C0174C17B491CC173C9B2042901DB32
:108B10000021C173704700000FB470B52DED048BB8
:108B200088B0B0EE408A0490DDED118ACDED058A63
:108B30009DED129A8DED069A0A25DFF8B048B4F93A
:108B4000660010FB05F0B4F96810461A04F1440001
:108B500001F088FB94F8440010FB05F094F84510F0
:108B60004518ADB22A2D0FD136B2002E0CD5606853
:108B7000002806D10120F9F734FBF9F704FB0120A6
:108B800060600120206015E06068012807D1F9F7D6
:108B900005FB002060600FF67000FBF7EDFD20681C
:108BA000282D3BDA012803D10FF68800FBF7E4FDFE
:108BB0000020206094ED150ADDED100AB4EE600A85
:108BC000F1EE10FA37D194ED160AB4EE680AF1EE20
:108BD00010FA30D194ED170AB4EE490AF1EE10FA0A
:108BE00029D1DFF80C582868401C286015282CD3A0
:108BF000E06DFDF727F9CDE90201A06DFDF722F93F
:108C0000CDE90001606DFDF71DF902460B460FF638
:108C10003000FBF7B1FD0020286016E0002805D1E8
:108C2000002229460FF2EC70FBF7A6FD0120206020
:108C3000F9F7B8FABEE7049860650598A06506984C
:108C4000E0650020DFF8A817086004A890EC030A8C
:108C5000FFF742FF159D284680B2B0EE480A04F0A7
:108C60009FFE294604A8F8F74BFD04F16000F9F7D0
:108C700003FA206E012811D1F7F7B9FA04F1600068
:108C8000F9F7FAF92C2204F1600104F18C00F9F7EC
:108C90004FFB0FF2C070FBF76FFD01E000F002F92F
:108CA000002008B0BDEC048B70BC5DF814FBDFF84D
:108CB0003C07807B7047002806D0DFF83017D1F8DA
:108CC000B8104422F9F734BB704710B500281CD106
:108CD000DFF81847483400EE101AB8EE400A84ED69
:108CE000010A2046F9F7CFF994ED010AF2EE0A0ADB
:108CF00020EE200A10EE100AFDF7A4F802460B46FB
:108D00000FF25870FBF738FD2FE001281CD1DFF877
:108D1000DC4600EE101AB8EE400A84ED120A04F1A7
:108D20004800F9F7B0F994ED120AF2EE0A0A20EEC3
:108D3000200A10EE100AFDF785F802460B460FF2E6
:108D40002870FBF719FD10E002280ED1DFF89C46D1
:108D5000483421722046F9F796F9207A0D2111FB4B
:108D600000F10FF21070FBF707FD0FF21470FBF724
:108D700003FD42F26A7001460FF21070FBF7FCFC33
:108D800040F2EE7001460FF21070BDE81040FBF7A4
:108D9000F3BC2DE9F0412DED028B84B006460F4661
:108DA00090460FF2DC60FBF7E7FC42F26A70014686
:108DB0000FF2D860FBF7E0FC40F2EE7001460FF2D4
:108DC000D860FBF7D9FCDFF8244600224FF4E671A7
:108DD0002046F9F76FFA04F58075C4F8B85000EE34
:108DE000106AB8EE408A84ED138A00EE107AB8EE6D
:108DF000400A84ED120A84F85080F2EE0A8A404656
:108E00000D2111FB00F0029020EE280A10EE100A4E
:108E1000FDF718F8CDE9000128EE280A10EE100A37
:108E2000FDF710F802460B460FF27C60FBF7A4FC3E
:108E3000F7F736F904F14800F9F725F942F2107016
:108E4000A4F8C200A4F8C4000020A4F8BC00A4F850
:108E5000BE000220A4F8C6002C2204F1BC01284662
:108E6000F9F766FA0220A07304F08CFD012060730C
:108E700004F1440001F0F6F900206060206004B0C5
:108E8000BDEC028BBDE8F08110B592B0F9F79EF908
:108E9000044600A8FFF70FFF0498001912B010BD98
:108EA000000000002DE9F0412DED028BDFF83C457C
:108EB00004F17005E86A216F814205D1B4F866209B
:108EC0006B8C9A4200F08880B1EB000802D5DFF885
:108ED0002405804495ED060AD5ED110A70EE608AEE
:108EE000F5EE408AF1EE10FA03D59FED950A78EE83
:108EF000808A95ED040AD5ED0F0A30EE608AB5EE52
:108F0000408AF1EE10FA03D59FED8D0A38EE008A03
:108F1000B4F86600C0B295ED050A04F03DFEB0EE6F
:108F2000401A04F10C067078012802D002282BD0D8
:108F300033E004F5A27739469FED821AF0EE480A35
:108F4000B0EE680A404600F057F8207B404420739A
:108F5000C0B2062821DB04F5AA7004F1BC019FED24
:108F6000791AD0ED0A0A90ED080AD4F8540100F0FD
:108F700043F8207B401C2073002244213846F9F737
:108F800099F90220707008E004F1BC01F0EE480A83
:108F9000B0EE680A404600F02FF8B4F866000028EA
:108FA00009D10022442104F5A270F9F783F90020C9
:108FB0002073012070702C2204F1600104F18C00F8
:108FC000F9F7B6F904F1BC01A96404F580764422EE
:108FD0003046F9F7ADF9AE6404F166004088B4F8A4
:108FE0000A11884203D0A4F8C600A4F80A01BDEC17
:108FF000028BBDE8F08100002DE9F0412DED048BDE
:109000008AB0B0EE409AB0EE608AF0EE418A0C462B
:10901000DFF8D87307F164056E88B7F86480A6801E
:10902000B0EE680A00F0BDF8B868002819D194EDD8
:109030000C0A30EE090A84ED0C0A00F0AFF984ED59
:109040000C0A6680A4F80080A869606394ED0E0A9B
:1090500030EE080A84ED0E0A00F094F984ED0E0A51
:109060004AE007F1480007AA0AC80AC20368136069
:1090700007F1600184B068462C22F9F759F90FBC5A
:10908000B0EE680A00F030F9D4ED0C0A30EE800A38
:1090900084ED0C0A00F082F984ED0C0AF5EE408AAA
:1090A000F1EE10FA0BDD032E03D106206080208044
:1090B00010E0042E0ED10820608020800AE0032EEC
:1090C00003D107206080208004E0042E02D1092013
:1090D00060802080F6EE000A95ED060A20EE200A58
:1090E00084ED0D0A94ED0E0A08EE200A84ED0E0AB6
:1090F00000F048F984ED0E0A95ED080ADFEDB00A9C
:1091000020EE200A84ED0F0ADFEDAE0AB4EE600A0D
:10911000F1EE10FA01DBB848E0636869206460880A
:10912000002801D1002020642869E060288920817E
:10913000A88860810AB0BDEC048BBDE8F081000016
:10914000002474490000000010B50C46A1880329D2
:1091500012D1B5EE400AF1EE10FA06DD216A401890
:10916000206200F027F9206210BD616A4018606239
:1091700000F020F9606210BD042911D1B5EE400A5B
:10918000F1EE10FA06DDA16A4018A06200F012F9B3
:10919000A06210BDE16A4018E06200F00BF9E062E5
:1091A00010BDF8B52DED028B0546B0EE408A0C4699
:1091B00020692818206100F0FDF82061B5EE408A92
:1091C000F1EE10FA02DDB0EE480A01E0B1EE480A15
:1091D000B5EE400AF1EE10FA43DD844EB068002887
:1091E00030D106F5CE77B86806280ED261880429FA
:1091F00003D179686918796004E0D6F89C11691880
:10920000C6F89C112818B86051E0E1694018E06187
:1092100000F0D0F8E0612146B0EE480AB868FFF7E8
:1092200093FFE0692818E06100F0C4F8E06121468E
:10923000B0EE480A2846FFF787FF00F03BF8012010
:10924000B06034E0E0692818E06100F0B3F8E06154
:109250002146B0EE480A2846BDEC028BBDE8F4403A
:1092600072E76088032802D0042807D00DE0606907
:109270002818606100F09EF860610CE0A069281871
:10928000A06100F097F8A06105E0606928186061AE
:1092900000F090F86061554E06F5CE7080680028A9
:1092A00001D000F010F800F005F80020B060BDEC2F
:1092B000028BF1BD4D480021C0F89C1100F5CE7025
:1092C0004160816070474948D0F8D010D0F89C21A7
:1092D0005118C0F8D01000F1D0014A68D0F8A001B0
:1092E00080184860704700000FB4DFED370A9FED2B
:1092F000361AF0EE0C1A9DED092ABDF80600042876
:109300000FD1DFED322A42EE221AB5EE400AF1EE1D
:1093100010FA15D49FED2E1A22EE011A21EE001A32
:109320000EE0DFED2C2A42EE221AB5EE400AF1EEF5
:1093300010FA05D49FED281A22EE011A21EE001A28
:10934000B5EE402AF1EE10FA0ED09DED060AB5EE0C
:10935000400AF1EE10FA07D0DFED200A20EE200AD5
:10936000F7EE000AC0EE800A31EE810A9FED1C1A6A
:1093700020EE010A9DED0B1A20EE010A20EE200AD4
:1093800004B07047DFED170AB4EE600AF1EE10FA90
:1093900003DBDFED150A30EE200A7047DFED110A1E
:1093A000B4EE600AF1EE10FA03DBDFED0F0A30EEE7
:1093B000200A70470F49884201D3104908187047A6
:1093C0008FC2753D0100C84100000000CDCC4C3E6D
:1093D0006666663FCDCCCC3D6666E63F00007042D7
:1093E0000AD7A33B01247449002474C920920300C6
:1093F000ECAD0300819698000000C841806967FFCA
:10940000F8F708BFF8F749BE50443A2042505F4F82
:109410004646000050443A2053746570436E7455BC
:10942000702056482825642920435943282564295B
:109430000000000050443A20455849542056480046
:1094400050443A204E41432025662025662025665B
:109450000000000050443A204F46520050443A2049
:10946000312025660000000050443A203220256655
:109470000000000050443A20332025640000000022
:1094800050443A20303246454231350050443A206B
:109490004D50445F7625640050443A205052495064
:1094A000445F76256400000050443A203120256650
:1094B0002032202566203320256400002DE9F0436A
:1094C000002300E05B1C032B4ADA002433E005F1A3
:1094D000070EAEEB060E4FF007089EFBF8F8C8EB40
:1094E000C808AEEB080E5FFA8EFE0FF66468C3EB99
:1094F000C30908EBC90808EB8609D9ED070A07EB91
:10950000000909EB8E0999ED3F1A60EE810A08EB1C
:10951000860898ED001A0CEB8E0EDEED001A41EE77
:10952000610A30EE800A761C072ED0DB0CEB850535
:1095300085ED000A641C032CC4DAC4EBC405AF003B
:10954000542515FB030507EB050C0D46002A03D136
:1095500000264CF82560EDE79FED440A0026E3E77E
:10956000BDE8F083D2B218B400230CE094ED031AE6
:1095700021EE001AF7EE001A71EEC01A01EEA01AE1
:1095800084ED001A5B1C032B0ADA51F8234000EE2D
:10959000904A002A00EB8304E8D1C4ED000AF1E709
:1095A0000C2201460C3018BCF8F7C2BE38B5044690
:1095B0000D4600200AE0C0EBC00204EB820202EB81
:1095C000810155F82020C1F8FC20401C04F5F272FE
:1095D00092F902100328EEDB5278C9B22046FFF759
:1095E0006DFF94F8E4219FED220A294604F5A87046
:1095F000BDE83840B6E70000F8B5044694F9E651F6
:10960000EDB2002617E0542212FB064211FB0021A6
:1096100051F8251000EE901A00EEA00A401C1C2103
:109620000328F0DB11FB064000EB850704F084FC07
:1096300087ED5D0A761C032E03DA9FED0C0A0020ED
:10964000EDE704EB850000F5C87191ED070AB5EE72
:10965000400AF1EE10FA06D0D0ED640A80EE800ADE
:1096600081ED0E0AF1BD00208863F1BD000000000D
:10967000A4707D3F10B5044604F5A870D0ED020A31
:1096800090ED011A94ED540A20EE000A01EE010A51
:1096900000EEA00A04F050FC002002E000228A61E3
:1096A000401C03280FDA04EB800202F5A871B5EE26
:1096B000400AF1EE10FAF1D0D2ED540AC0EE800A61
:1096C000C1ED060AECE710BDD0ED000A70EE800A8D
:1096D000C0ED000AD0ED010A40EE000AC0ED010A1B
:1096E00089B2531E994215D100EE102AB8EE400AF5
:1096F000D0ED000AC0EE800AC0ED000AD0ED010AEC
:1097000080EE800A80ED010AD0ED000A00EEE00A4A
:1097100080ED020A70472DE9F84F04460D4694F992
:10972000E601C0B200902E88322096FBF0F0322184
:1097300001FB1067B5F878804FF000092AE004EBD0
:10974000890A09EB490005EB800B4FF4FA723146A8
:109750000BF140009AED5A0AFFF7B6FF40F2DC52D7
:1097600041460BF190009AED5A0AFFF7ADFF322205
:10977000394689B20BF11C00C9EBC90304EB830322
:10978000DDF800C003EB8C0393ED3F0AFFF79CFF6D
:1097900009F10109B9F1030FD1DBBDE8F18F8A1D91
:1097A000072392FBF3F3C3EBC303D21A50F8222032
:1097B00000EE102A00EB8100D0ED000A30EEC00A66
:1097C000B0EEC00A704730B40A460021931D07244A
:1097D00093FBF4F4C4EBC4041B1BDBB2541D07253C
:1097E00094FBF5F5C5EBC505641BE4B250F82330D6
:1097F00000EE103A50F8222000EE902AF4EE400AD3
:10980000F1EE10FA0AD500EB840292ED001AB4EEE4
:10981000401AF1EE10FA01D501210EE0B4EE600A13
:10982000F1EE10FA09D500EB8400D0ED000AB4EE99
:10983000600AF1EE10FA00D50121084630BC7047ED
:109840002DE9FE4306460C4696F8E651208800288E
:1098500000F08A8000273CE0C7EBC70006EB8009D8
:10986000294609F15400FFF79AFF08EB870080EDC5
:10987000000AD4ED030A30EE800A84ED030A09F1F0
:10988000A80829464046FFF78AFFD4ED050A30EEC6
:10989000800A84ED050A294609F15400FFF793FF79
:1098A00000EE100AB8EE400AD4ED040A30EE200AA9
:1098B00084ED040A29464046FFF785FF00EE100AB2
:1098C000B8EE400AD4ED060A30EE200A84ED060A0E
:1098D0007F1C0DF10008032FBEDB00200AE094ED91
:1098E000010A08EB8001D1ED000A30EE200A84ED78
:1098F000010A401C0228F2DB94ED020AD8ED020AAC
:1099000030EE200A84ED020A294606F5C870FFF7FA
:1099100046FFD4ED030A30EE800A84ED030A29469F
:1099200006F5D670FFF73BFFD4ED050A30EE800A4E
:1099300084ED050A06F5E47629463046FFF72FFF49
:10994000D4ED1B0A30EE800A84ED1B0A294630460E
:10995000FFF739FF00EE100AB8EE400AD4ED1A0AFC
:1099600030EE200A84ED1A0ABDE8F7830A8890F9E0
:10997000E631DBB200EB830090ED5D0A3220034656
:1099800092FBF3F300FB1323002B04D181ED020AB9
:1099900081ED030A7047D1ED020AF4EE400AF1EEC0
:1099A00010FA02D581ED020A08E0D1ED030AB4EE07
:1099B000600AF1EE10FA01D581ED030A521C03464C
:1099C00092FBF3F300FB132000281BD191ED020A58
:1099D000D1ED030A30EE600AD1ED040A70EE800A80
:1099E000C1ED040A022B0BDBD1ED010A70EE600A17
:1099F000F0EEE00A91ED051A71EE200AC1ED050ABC
:109A000081ED010A088840F2DB52904209D191EDC4
:109A1000040AF3EE0E0A80EE200A81ED040A01200A
:109A200088707047F8B52DED048B84B00C4600218A
:109A3000642749E0C1EBC10200EB820290F9E631F4
:109A400052F8232000EE102A00AA02EB810282EDD8
:109A5000000A04EB810202F2B445D5ED030A70EE70
:109A6000800AC5ED030A4FF4C87313FB014394F851
:109A7000B06403EB860696ED001A70EEC10AC5EDE0
:109A8000030AD2F8B45400EE905A70EE800A02F243
:109A9000B445C5ED000A94F8B05432353E4695FB06
:109AA000F6F607FB165503EB850595ED001A70EEEB
:109AB000C10A02F2B442C2ED000A94F8B02403EBEA
:109AC000820282ED000A491C0329B3DB94F8D80412
:109AD000002816D100200EE004EB8001D1F8B42458
:109AE00000EE102ADFED850A80EE200A01F2CC415B
:109AF00081ED000A401C0328EEDB012084F8D80425
:109B000058E004F5966090ED040ADFED7D0A80EEE2
:109B1000200A8DED000A90ED050A80EE200A8DEDF9
:109B2000010A90ED060A80EE200A8DED020A9FEDF3
:109B3000758A9FED740ADFED738A002011E004EB53
:109B40008001D1F8CC1400EE901A00A951F8201031
:109B500001EE101A00EE818A00EEA00A41EE018AA1
:109B6000401C0328EBDB04F0E7F9B0EE409AB0EEBE
:109B7000680A04F0E1F929EE000AB5EE400AF1EEB8
:109B800010FA01D088EE008AB0EE480A04F0E2F93B
:109B9000DFEDC80A20EE200AF3EE0E0AB4EE600AEA
:109BA000F1EE10FA03DB002084F8D80402E0012073
:109BB00084F8D80494F8B004401C84F8B004C0B20F
:109BC000642802D1002084F8B00404B0BDEC048BFA
:109BD000F1BD000070B52DED048B0646301D90EDF3
:109BE000018A7068FCF72EF941EC190B18EE100A87
:109BF000FCF728F902460B4614461D4653EC192B78
:109C0000DFF8F406DFF8F416FCF7F4F922462B46E9
:109C100002F066FE1CD253EC192BDFF8E406DFF8E5
:109C2000E416FCF7E7F902460B4614461D469FED85
:109C3000DD0A38EE000A10EE100AFCF703F922469E
:109C40002B4602F04DFE03D2012086F8740002E09C
:109C5000002086F87400BDEC048B70BD70B504461E
:109C60000D461646FFF7C8FC2046FFF703FD2946C0
:109C70002046FFF750FD29462046FFF7E1FD05F19C
:109C800078012046FFF772FE31462046BDE870405D
:109C9000C8E6000038B52DED028B90ED050A90ED79
:109CA000038AFBEE040A9FED841A08EE201AB4EE34
:109CB000401AF1EE10FA1DD510EE100AFCF7C2F8AA
:109CC00002460B4614461D4618EE100AFCF7BAF879
:109CD000DFF83426DFF83436FCF78CF90022DFF8A1
:109CE0003036FCF743FD22462B4602F0F9FD01D247
:109CF000012000E00020BDEC028B32BD0000484294
:109D00000000C842000000002DE9F0412DED028B5B
:109D1000804600200CE098ED190A01EB410208EBA7
:109D20008201D1ED120A30EE200A88ED190A401C9A
:109D3000C0B201460329EEDB98ED1A0AD8ED1B0AE2
:109D40009FED8F1ADFED8F1A40EE011AF4EE610AD3
:109D5000F1EE10FA15DB9FED8C1ADFED8C1A40EE58
:109D6000011AF4EE610AF1EE10FA0ADB9FED881A8F
:109D7000DFED881A40EE011AF4EE610AF1EE10FAF6
:109D80004DDA9FED850AF4EE400AF1EE10FA46D462
:109D90009FED828BD8F81400FCF754F804460D466A
:109DA000D8F80C00FCF74EF853EC182BFCF7DEFC4F
:109DB00002460B4620462946FCF7F4FA0022DFF85B
:109DC0005435FCF717F9DFF85025DFF85035FCF76C
:109DD000CDFC02460B4616461F46D8F81800FCF785
:109DE00031F804460D46D8F81000FCF72BF853EC78
:109DF000182BFCF7BBFC02460B4620462946FCF715
:109E0000D1FA32463B4602F06BFD08D398ED190AB1
:109E1000DFEDCC0AB4EE600AF1EE10FA01DB0020AF
:109E200000E00120BDEC028BBDE8F0812DE9F0419E
:109E3000804698ED1A0ADFEDA10A80EE200AD8EDDF
:109E40001B0A9FED9E1AC0EE810A20EE200A10EE3A
:109E5000100AFBF7F7FF02460B4616461F46D8F8D6
:109E60000C00FBF7EFFF0022DFF8B434FCF7C2F878
:109E700004460D46D8F81400FBF7E4FFDFF8A424ED
:109E8000DFF8A434FCF772FC02460B462046294654
:109E9000FCF788FADFF86824DFF89034FCF766FCFA
:109EA00032463B4602F004FD01D8012000E00020CC
:109EB000BDE8F081ED2E65420000FA4338B52DED86
:109EC000048B05460C4600200CE095ED0F0A01EBD3
:109ED000410205EB8201D1ED080A30EE200A85ED42
:109EE0000F0A401CC0B201460329EEDB6869FBF78C
:109EF000A9FF41EC180B2869FBF7A4FF41EC190BF3
:109F000053EC182BDFF82804DFF82814FCF772F85C
:109F100002460B4651EC190B02F0E2FC2CD253EC3A
:109F2000182BDFF81404DFF81414FCF763F853EC73
:109F3000192B02F0D5FC1FD253EC182BDFF80004CC
:109F4000DFF80014FCF756F8DFF8CC23DFF8F8331D
:109F5000FCF70CFC53EC192B02F0C2FC0CD295ED73
:109F60000F0ADFEDC40AB4EE600AF1EE10FA03D571
:109F7000002C01D1012000E00020BDEC048B32BD9B
:109F800000C028C500854F49000048C400E87D484E
:109F90000000C8C200C82F4701806D458DEDB5A0F7
:109FA000F7C6B03E0000CDC338B505460C460020CC
:109FB000A070607095F87A00002806D095F87410AB
:109FC00005F17800FFF77AFFA07095F8740000287B
:109FD00013D12846FFF75EFE00280CD12846FFF774
:109FE00093FE002807D12846FFF720FF401E80413E
:109FF000C043C00F00E0012060706078002805D1E8
:10A00000A178481E8041C043C00F00E001202070AD
:10A0100031BD70B400220378447B2418E370437B85
:10A02000144610E05B1CDBB20A2593FBF5F505EB4B
:10A030008506A3EB4603DBB21D18ED78661C16FB04
:10A04000052292B2641C0A2CECDB042008702D2A35
:10A0500002DB022048700BE0222A02DB012048705C
:10A0600006E00F2A02DB0020487001E000200870A3
:10A0700070BC704710B504469FED9C0A002008E0B4
:10A0800000EB400104EB8101D1ED090A00EEA00ACA
:10A09000401C0328F4DB03F04FFF84ED1C0ADFEDC6
:10A0A000940AB4EE600AF1EE10FA05D500221146CA
:10A0B0000846BDE81040B3E010BD000000401C465B
:10A0C00070B50C4604F59B65E97BAA7B121992F8E2
:10A0D000E124891AE973A97B091990ED1C0ADFEDC7
:10A0E000850AB4EE600AF1EE10FA03DB012081F874
:10A0F000E10402E0002081F8E104E87BA97B091972
:10A1000091F8E1140818E873904E0022242106F516
:10A110000170F8F7CFF896F89A07042810D196F84E
:10A120009B0700280CD0E87B022803DA94F8D804B7
:10A13000002805D1002204210220BDE870406FE014
:10A1400070BD0000CDCC4C3E30B591B07F4C04F5D5
:10A15000F2718878401C88704A78002A0BD194F8F4
:10A16000E421002A02D1012284F8E42140B2072828
:10A1700001D101224A7040B2072290FBF2F2C2EBF9
:10A18000C202801A88708888401C8880B4F86012E7
:10A19000491CA4F8601280B2322190FBF1F1322206
:10A1A00002FB110131290BD194F88617491CC9B261
:10A1B000052291FBF2F202EB8202891A84F88617DB
:10A1C000B0F5FA7F24D104F518754022294600A87D
:10A1D000F8F7AEF80022B82104F5F470F8F76AF841
:10A1E000BDF8000040F2DC51884204D0402200A9B2
:10A1F0002846F8F79DF804F28670C17C491CC9B264
:10A200000A2291FBF2F202EB8203A1EB4301C1743B
:10A2100011B030BD002240F29C714C48F8F74AB8AA
:10A220002DE9F04106460C461546484F97F8990728
:10A2300009300A2190FBF1F101EB8102A0EB420809
:10A2400000220A2107F28F70F8F7AEF85FFA88F85B
:10A2500008EB070080F88F6707F2997044708570EB
:10A26000BDE8F081002803D03849B1F89A17018081
:10A27000704700009A99993EF8B5344C0146204643
:10A28000FFF794F904F5F47504F52876324629466B
:10A290002046FFF7E3FCB4F8E80140F2F3118842EE
:10A2A0000DD12846FFF796FC04F28C7739462846F4
:10A2B000FFF77AFE04F29A713846FFF7AAFEB4F867
:10A2C000E801322190FBF1F1322202FB110031282A
:10A2D00008D12846FFF7CEFE04F28C72314628469C
:10A2E000FFF7EEFEBDE8F1402EE7000000000000A1
:10A2F00052499D390100C04085EB51B81E85F73F9A
:10A30000D7A3703D0AD71540CDCCCCCCCCCC0040E7
:10A3100000005440000004C09A99999999991B40F3
:10A320000000F8BF8DEDB5A0F7C6B03E0AD7E33FF9
:10A33000E17A14AE47E1BA3FC976BE9F1A2FAD3F0E
:10A34000EC51B81E85EBA13F9999E93F0C690300D8
:10A3500000000000FDF881C0232FE340DA1ED9C0C1
:10A36000F3456E40EDE88DBF0B030F3E2D8AE038BC
:10A37000A267283A8A81D23A5C560C3B8A81D23A4B
:10A38000A267283A2D8AE03800000000AD9D27C062
:10A39000EE695740790B1FC088848C3F61738ABE79
:10A3A0009135EC3C61A1F13A0939353C4B87E23CEF
:10A3B000DD04173D4B87E23C0939353C61A1F13A98
:10A3C000000000001D1073BE20794C3FAE63E7BD56
:10A3D0002813F53D5676F9BB3631F43A42CE113D9D
:10A3E00063B55ABE5EB1083FD24136BF5EB1083F89
:10A3F00063B55ABE42CE113DF8B52DED028B0C4629
:10A400008A4951F82050002601280DD0042833D065
:10A4100005285CD0082867D0252800F084804A28C9
:10A4200074D04D2878D08EE09FED810A834FB4F927
:10A43000000000EE900AF8EEE00A60EE800AC7ED38
:10A44000000AB4F9020000EE900AF8EEE00A60EEAD
:10A45000800AC7ED010AB4F9040000EE900AF8EE94
:10A46000E00A20EE800A87ED020A2088B881608821
:10A47000F881A088388266E09FED6E8B6F4FB4F94B
:10A480000000FDF7C1FD53EC182BFBF7B3FDFBF704
:10A4900083FE7861B4F90200FDF7B6FD53EC182B8A
:10A4A000FBF7A8FDFBF778FEB861B4F90400FDF7EF
:10A4B000ABFD53EC182BFBF79DFDFBF76DFEF86130
:10A4C0002088388460887884A088B8843BE05B4F1B
:10A4D000786B2168884200D101261822214607F1B5
:10A4E0003400F7F715FF2EE02078544F97F84C1002
:10A4F000814200D1012687F84C00B4F80100A7F88A
:10A500004E00B4F80B00A7F850001CE00C222146C6
:10A510004B48F7F7FDFE16E0012608222146494880
:10A52000F7F7F6FE0FE0454FF86D2168884204D139
:10A53000386E6168884200D101260822214607F161
:10A540005C00F7F7E5FE002D13D0002E11D1686AEC
:10A5500000280ED0406940490968401A012808DAED
:10A56000214605F11000BDEC028BBDE8F44000F07F
:10A5700095BBBDEC028BF1BD02460846012A0AD00C
:10A58000042A0CD0052A0ED0082A10D04A2A12D04C
:10A590004D2A14D0704714222849F7F7B9BE142267
:10A5A0002949F7F7B5BE18222849F7F7B1BE0622A8
:10A5B0002749F7F7ADBE0C222149F7F7A9BE0822BB
:10A5C0002049F7F7A5BE10B5184951F820400128D9
:10A5D00008D004280CD0052810D008281AD0252827
:10A5E00012D01CE0FF2214211448F7F763FE16E096
:10A5F000FF2214211448F7F75DFE10E0FF22182116
:10A600001248F7F757FE0AE0FF2208211148F7F732
:10A6100051FE04E0FF2206210D48F7F74BFE04F13E
:10A620001000BDE8104000F033BB00007897030035
:10A63000FDF61C3B0597A11D4F04443F34A80300C1
:10A640005CA8030088A8030048A8030068A80300CA
:10A6500080A8030090A80300088C030010B52DED1E
:10A66000028B044682B094ED008A9FED2D0A28EEFD
:10A67000000AB5EE400AF1EE10FA8DED000AACBF0B
:10A68000F6EE000AFEEE000A30EE200A8DED000A1A
:10A69000002100A803F090FC9DED000AB5EE400AF1
:10A6A000F1EE10FA17D0DFED1F0A20EE200ADFEDE1
:10A6B0001E0A00EE608ADFED1D0A00EE608ADFED03
:10A6C0001C0A00EE608ADFED1B0A00EE608ADFEDF7
:10A6D0001A0A00EE608A84ED008ADFED180A9DED0B
:10A6E000000AB4EE600AF1EE10FA06D4DFED140AA7
:10A6F000B4EE600AF1EE10FA05DBDFED120A03F0AA
:10A7000083FC8DED000A9DED000A02B0BDEEC00A8B
:10A7100010EE100ABDEC028B00F0030010BD00002B
:10A7200083F9223F000080380000C94600A0FD40A8
:10A730000020A23A000034330030C22E000000CFC7
:10A740000100004F0000004F014803F0FBBC000077
:10A75000000003001AA210EE101ADFF860C0F2EC3D
:10A76000060A614509DB00EE803A70EE800A83EE4E
:10A77000200A40F0020010EE101A21F0004CDCF12B
:10A78000665C0BD860EE000A20EE203A03EE010A68
:10A7900001EEA02A42EE202A80EE220A400810F0A4
:10A7A000020F18BFB1EE400A02EB8002D2ED000AA0
:10A7B00030EE200A28BFB1EE400A7047A430893E2F
:10A7C000D7B3DD3F6AD5033F2B94A93DB82A593F43
:10A7D0000000803F000080BF00000000920A063F9A
:10A7E000DB0FC93F920A863FDB0FC93F920A064042
:10A7F000DB0F4940368D2740DFED4A0A60EE200A24
:10A8000010B5B0EEE01ADFED481AB4EE611AF1EEC1
:10A8100010FA82B0044629D5F5EE400AF1EE10FA9E
:10A82000ACBFB6EE001ABEEE001A70EE810AFDEE65
:10A83000E00A10EE900AA8B1FAEEC90A9FED3B1AA1
:10A8400000EEC10A9FED3A1A00EEC10A9FED391AD7
:10A8500000EEC10A9FED381A00EEC10A9FED371ACB
:10A8600000EEC10A00F00300041921E08DED000A9A
:10A870000098C0F3C750FF2808D088B9009840025C
:10A880000ED1002C4CD0B7EE000A13BD0098400248
:10A8900046D1FFF759FF212101609FED290A13BD21
:10A8A0008DED000A00A8FFF7D9FE04199DED000AFE
:10A8B000DFED240AB4EE600AF1EE10FA0BDBDFEDF7
:10A8C000220AB4EE600AF1EE10FA04D5E00723D5AF
:10A8D000B7EE000A20E0E00760EE000A0ED59FED1B
:10A8E0001B0A9FED1B1A00EE801ADFED1A1A41EECB
:10A8F000201AB7EE000A01EEA00A0DE0DFED161AED
:10A900009FED162A00EEA12ADFED151A20EE201A7F
:10A9100042EE201A01EE210AA00748BFB1EE400A1C
:10A9200013BD000083F9223F0000004F0000C9461C
:10A9300000A0FD400020A23A000034330030C22EB7
:10A94000FFFFFF7FFEFF7FB9000080399349B2BA55
:10A9500036A02A3DDFFFFFBE6E8C4CB94283083C17
:10A96000A1AA2ABE1FB5FFF7EFFE212101601FBD7E
:10A9700030B5134D0446287881B020B9281D03F066
:10A980000BFC01202870281D03F01FFC204604F05A
:10A99000FEFA0446281D03F03EFC204601B030BDFF
:10A9A00030B50446064D81B0281D03F00EFC20464C
:10A9B00004F04DFC281D01B0BDE8304003F02BBC75
:10A9C00004AD030038B50446002500E06468002C9F
:10A9D0000CD0207A0A789042F8D1E0684A68904218
:10A9E000F4D120698A689042F0D1012529460FF2FE
:10A9F0005C20F9F7C1FE002D00D10024204632BDB5
:10AA000038B504462020FFF7B3FF05460022202179
:10AA1000F7F750FC0C22214605F10800F7F788FCF7
:10AA200060686861A068A86101202877284632BD67
:10AA3000F8B500231C4601F10805834A1678761CF8
:10AA40001670802686F3118800BF00BF5678761CEA
:10AA5000567006686F6801E034467668002E04D0B0
:10AA6000D6F80CC06745F7DA0123002B0AD033680B
:10AA70000B604E603368002B01D0596000E001602C
:10AA8000316005E0002C02D061600C6000E00160E4
:10AA90005078401E5070C0B2002802D1002080F3D0
:10AAA0001188FDF7FDF90020F2BD10B5664C227843
:10AAB000521C2270802282F3118800BF00BF62788E
:10AAC000521C62704A680B68002B01D05A6000E08B
:10AAD00002604868002801D00A6802600846FFF753
:10AAE0005FFF6078401E6070C0B2002802D1002075
:10AAF00080F31188FDF7D4F9002010BD30B442680E
:10AB0000002A00D10268002A28D04F490B785B1C2C
:10AB10000B70802383F3118800BF00BF4B785B1C50
:10AB20004B70D36852699A1AC3689C1A92FBF3F56A
:10AB300003FB0543436103699C1A92FBF3F203FB99
:10AB4000024282614878401E4870C0B2002802D19B
:10AB5000002080F3118830BCFDF7A2B930BC7047EB
:10AB600070B504460D462068FFF72CFF06000BD198
:10AB70002846FFF745FF064631462046FFF758FFB7
:10AB80003046FFF7BBFF02E0307F401C3077207A71
:10AB9000401C2072307A002800D16660002070BD11
:10ABA00010B504462068FFF70DFF002801D10320EF
:10ABB00010BD017F491E0177217A491E2172017A59
:10ABC000002901D100216160017F002903D10146E4
:10ABD0002046FFF76AFF002010BD70B51A4A1378AF
:10ABE0005B1C1370802383F3118800BF00BF537870
:10ABF0005B1C5370006801E083614068002815D039
:10AC000043695C1A83695B1A012C05DAC568661909
:10AC100094FBF5F405FB14644461012BECDA046940
:10AC20001D1993FBF4F304FB1353E5E75078401E22
:10AC30005070C0B2002802D1002080F31188FDF7C7
:10AC40002FF9002070BD0000A03D030023666320A3
:10AC50002564000000B581B0802282F3118800BF16
:10AC600000BF8A69104388610A7C02F0F802082A52
:10AC700005D1CA6902421CBF0846FDF72DF90348F9
:10AC8000407808B980F3118801B000BDA03D0300F1
:10AC90004FF0FF31018100218172704738B50446C1
:10ACA00000291BD0002C19D0B4F90800401C2288C0
:10ACB00090FBF2F302FB1300208160880246636878
:10ACC000B4F9085000FB0530F7F722FBB4F908008F
:10ACD0002188491E884201D10120A07231BD70B582
:10ACE00004460D0036D0002C34D0A87A01281FD19C
:10ACF000B5F90800411C2A8891420ADA6B88521E75
:10AD0000101A03FB00F2686803FB01012046F7F705
:10AD1000FFFA6888B5F90830591C00FB01F2696830
:10AD20002E88761EF31A00FB0340F7F7F1FA0CE0C9
:10AD3000284600F010F8002807D0284600F00BF84D
:10AD4000024669682046F7F7E3FA0020A8724FF040
:10AD5000FF30288170BD817A002901D0018802E08E
:10AD6000B0F90810491C408811FB00F080B2704710
:10AD7000817A002901D0008802E0B0F90800401C67
:10AD800080B27047F0B591B004460D46002600AF82
:10AD900017E0DFF8D805335D1B111B5C3B70335D9A
:10ADA00003F00F03185C07F8010F761C002007F86A
:10ADB000010F491C9142ECDB00A90FF2786000F012
:10ADC00079FBAE4205DAAA1B212A00DB20220021F2
:10ADD000F0E711B0F0BD01684A1C026008787047C6
:10ADE00001688A1C02600878497840EA01207047AF
:10ADF00001680A1D026008784A7840EA02208A78D1
:10AE000040EA0240C97840EA0160704781B00168B9
:10AE10000A1D026008784A7840EA02208A7840EAEF
:10AE20000240C97840EA016000909DED000A01B03F
:10AE3000704713B50446012201A92068F7F768FAA4
:10AE40002068401C2060012016BD13B50446022274
:10AE500001A92068F7F75CFA2068801C20600220B6
:10AE600016BD13B50446042201A92068F7F750FA6D
:10AE70002068001D2060042016BD10B50446FFF7B1
:10AE800077FD002806D001E00021215421464C1E08
:10AE90000029F9D110BDFFF783BD38B504460D4632
:10AEA0000094297800A8FFF7C4FF697800A8FFF78D
:10AEB000C0FFA97800A8FFF7BCFFE97800A8FFF75A
:10AEC000B8FF297900A8FFF7B4FF697900A8FFF758
:10AED000B0FFA97900A8FFF7ACFFE97900A8FFF758
:10AEE000A8FF297A00A8FFF7A4FF697A00A8FFF756
:10AEF000A0FFA97A00A8FFF79CFFE97A00A8FFF756
:10AF000098FF297B00A8FFF794FF697B00A8FFF753
:10AF100090FFA97B00A8FFF78CFFE97B00A8FFF753
:10AF200088FF297C00A8FFF784FF697C00A8FFF751
:10AF300080FFA97C00A8FFF77CFFE97C00A8FFF751
:10AF400078FF297D00A8FFF774FF697D00A8FFF74F
:10AF500070FFA97D00A8FFF76CFFE97D00A8FFF74F
:10AF600068FF297E00A8FFF764FF697E00A8FFF74D
:10AF700060FFA97E00A8FFF75CFFE97E00A8FFF74D
:10AF800058FF297F00A8FFF754FF697F00A8FFF74B
:10AF900050FFA97F00A8FFF74CFFE97F00A8FFF74B
:10AFA00048FF95F8201000A8FFF743FF95F82110FF
:10AFB00000A8FFF73EFF95F8221000A8FFF739FF21
:10AFC00095F8231000A8FFF734FF95F8241000A887
:10AFD000FFF72FFF95F8251000A8FFF72AFF95F837
:10AFE000261000A8FFF725FF95F8271000A8FFF707
:10AFF00020FF95F8281000A8FFF71BFF95F82910EF
:10B0000000A8FFF716FF95F82A1000A8FFF711FF18
:10B0100095F82B1000A8FFF70CFF95F82C1000A84E
:10B02000FFF707FF95F82D1000A8FFF702FF95F82E
:10B030002E1000A8FFF7FDFE95F82F1000A8FFF7CF
:10B04000F8FE95F8301000A8FFF7F3FE95F83110E0
:10B0500000A8FFF7EEFE95F8321000A8FFF7E9FE12
:10B0600095F8331000A8FFF7E4FE0098001B32BDEE
:10B0700038B504460D460094296800A8FFF7F1FE94
:10B08000297900A8FFF7D5FEE98800A8FFF7DDFEC3
:10B09000298900A8FFF7D9FEA97A00A8FFF7C9FE01
:10B0A000E97A00A8FFF7C5FE297B00A8FFF7C1FEDB
:10B0B000697B00A8FFF7BDFE0098001B32BD10B5EC
:10B0C00082B004460094097800A8FFF7B2FE009809
:10B0D000001B16BD38B504460D460094297800A81B
:10B0E000FFF7A7FE697800A8FFF7A3FE0098001BF2
:10B0F00032BD10B582B004460094097800A8FFF76D
:10B1000098FE0098001B16BD38B504460D46009504
:10B1100000A8FFF760FE207000A8FFF75CFE6070DB
:10B1200000A8FFF758FEA07000A8FFF754FEE070DB
:10B1300000A8FFF750FE207100A8FFF74CFE6071D9
:10B1400000A8FFF74DFEE08000A8FFF751FEA060C9
:10B1500000A8FFF74DFEE06000A8FFF749FE206160
:10B1600000A8FFF745FE606100A8FFF739FE2083C5
:10B1700000A8FFF735FE608300A8FFF731FEA0832B
:10B1800000A8FFF728FEA0770098401B32BD38B515
:10B1900004460D46009500A8FFF71DFE207000A88C
:10B1A000FFF719FE607000A8FFF715FEA07000A859
:10B1B000FFF72CFE84ED010A00A8FFF727FE84EDBF
:10B1C000020A00A8FFF722FE84ED030A0098401B44
:10B1D00032BDF8B505460C4600263746009400A857
:10B1E000FFF7F9FD287000A8FFF7F5FD687000A8CB
:10B1F000FFF7F1FDA87000A8FFF7EDFDE87000A8CB
:10B20000FFF7E9FD287195F9040041280EDBA0F154
:10B2100040074020287109E0009905EB061008302E
:10B22000FFF7B5FF009940180090761C95F90400CF
:10B230008642F1DB002F03D0009800EB071000904E
:10B240000098001BF2BD38B504460D46009500A8D5
:10B25000FFF7C1FD20700098401B32BD38B5044691
:10B260000D46009500A8FFF7B6FD207000A8FFF777
:10B27000B2FD60700098401B32BD38B504460D46E3
:10B28000009500A8FFF7A7FD20700098401B32BD75
:10B29000F0B583B006460F46002502F10E00FFF719
:10B2A000ECFD04005ED00FF20422D2E90001CDE9EA
:10B2B00000013046ADF8040004F108003146E439DD
:10B2C0000CD040F26132891A1CD020390BD0AB3936
:10B2D0000ED040F2C712891A0FD018E03946FFF796
:10B2E000DCFD05461AE03946FFF7C2FE054615E0CB
:10B2F0003946FFF7E4FE054610E03946FFF7EAFE5F
:10B3000005460BE03946FFF7F4FE054606E03246F7
:10B310000FF238110FF2401000F0CCF82846ADF8CB
:10B320000000A0202070A3206070062200A9A01CAD
:10B33000F6F7EEFF05F10800B0210155B32102191F
:10B340005170851C0A480078002803D02946204601
:10B35000FFF718FD2946204600F05EF90546204615
:10B36000FFF799FD2846FEBD00000000544503008C
:10B370002C460300F8B50446002601F112073846B2
:10B38000FFF77BFD050053D0394600F0E5F80828AB
:10B390004ADB2878A02848D16878A32845D1A81C82
:10B3A0004188090401D5042100E03146028811FAE0
:10B3B00082F108318688485DB02836D14819407836
:10B3C000B32832D105F10801304640F24532801AE7
:10B3D0000ED04FF48072801A1AD0CB3810D040F2C1
:10B3E000C712801A10D046F63322801A04D013E018
:10B3F0002046FFF789FE18E02046FFF7EAFE14E03A
:10B400002046FFF720FF10E02046FFF727FF0CE063
:10B410002046FFF732FF08E032460FF260010FF2DC
:10B420006C0000F047F800E006462846FFF733FDC1
:10B430003046F2BD5B495D5B20676E737350726F7F
:10B44000746F636F6C205D2025730A0062657470F1
:10B4500057726170706572005B495D5B20257320D7
:10B460005D20556E68616E646C6564206D657373F4
:10B4700061676520256C750A0000000062657470C4
:10B48000556E777261707065720000005B495D5B9C
:10B49000202573205D20556E68616E646C656420A4
:10B4A0006D6573736167652025690A0000000200FD
:10B4B000000000000EB400B582B003A9009102465E
:10B4C00000AB0121034878440A3001F085FB06BC3B
:10B4D0005DF810FB7B96010010F0030001D0C0F175
:10B4E000040080B2704738B5744C0020E060A06062
:10B4F000606020600120206160610FF2E825E36850
:10B500006F4A29460FF2E820FFF7D4FFA3686D4A7F
:10B5100029460FF20430FFF7CDFF63686A4A2946D7
:10B520000FF21C30FFF7C6FF2368224629460FF2B0
:10B530003830FFF7BFFF2369644A29460FF25030C5
:10B54000FFF7B8FF6369624A29460FF2703001B015
:10B55000BDE83040FFF7AEBF2DE9F04188B00446AA
:10B560000D46002604A80FF280318CC98CC05948C2
:10B570004088ADF812002846ADF81600514F7868A3
:10B580000090386801904FF4006002904FF47D30D5
:10B5900003900098019988423AD00C2204A900A88F
:10B5A00000F09AF80C282FD1BDF810004AF6CD31E2
:10B5B000884229D1BDF816804046FFF78DFF10FA6A
:10B5C00088F0A0F10C08BDF81400C10BC0F3803066
:10B5D00090EA010F05D06FF00106019840443860F1
:10B5E00016E0A84502D34FF0FF3611E0424621464F
:10B5F00000A800F071F840450AD101983860BDF804
:10B600001600A0F10C0603E06FF002060098386007
:10B61000304608B0BDE8F0812DE9F04188B004461D
:10B620000D4605A80FF2CC214CC94CC0294E70889C
:10B63000ADF8160005F10C00ADF81A0030888DF851
:10B640001D000027DFF87480D8F804000190D8F8B6
:10B65000000002904FF47A7003904FF47F30049012
:10B660000C2205A901A800F07BF80C2822D12A465B
:10B67000214601A800F074F8A8421BD100A8394661
:10B680000160284680B2FFF727FF0446224600A942
:10B6900001A800F065F8A0420CD17088401C7080B1
:10B6A0003088401C30800198C8F80400022004F063
:10B6B0005FF82F46384608B0BDE8F081E8FF030088
:10B6C000F4FF0300F0FF0300ECFF0300F8FF0300AA
:10B6D000FCFF0300E0AD03002DE9F84F04460D46E2
:10B6E00016462768D4F804B0A0685F4503D239181D
:10B6F000A1EB0B0801E0A7EB0B085F4502D2A0EB22
:10B700000B0901E0A7EB0B09CA46B14500D9B246C7
:10B710005246E0680BEB00012846F6F7F9FDD344EA
:10B72000A068834501D14FF0000BB1450ED2C14551
:10B730000CD2A6EB0A00874200D90746BB465A4600
:10B74000E1680AEB0500F6F7E3FDDA44A0688345FB
:10B7500001D14FF0000BC4F804B05046BDE8F28FA1
:10B760002DE9F04704460D461646E768D4F80080F8
:10B770006068804503D2A0EB0801491E04E0A1687F
:10B780004118A1EB0801491EB14201D2002027E077
:10B79000804504D2A0EB0800A0F1010902E0A068F6
:10B7A000A0EB0809CA46B14500D9B246524629461F
:10B7B00008EB0700F6F7ACFDD044B14508D2A6EB84
:10B7C0000A0842460AEB05013846F6F7A1FDC244D5
:10B7D000A068804501D14FF00008C4F800805046B1
:10B7E000BDE8F08773686D6970635F696E697400A6
:10B7F0005B495D25733A434855425F53484D495074
:10B80000435F52585F4845414428307825782920C5
:10B810003D20307825780A005B495D25733A43481E
:10B8200055425F53484D4950435F52585F54414918
:10B830004C283078257829203D20307825780A005A
:10B840005B495D25733A434855425F53484D495023
:10B85000435F54585F484541442830782578292073
:10B860003D20307825780A005B495D25733A4348CE
:10B8700055425F53484D4950435F54585F544149C6
:10B880004C283078257829203D20307825780A000A
:10B890005B495D25733A434855425F53484D4950D3
:10B8A000435F54585F4950435F4D534728307825D4
:10B8B0007829203D20307825780A00005B495D25F5
:10B8C000733A434855425F53484D4950435F52587D
:10B8D0005F4950435F4D5347283078257829203DF4
:10B8E00020307825780A0000CDAB0000C0000000B1
:10B8F00000000000CDAB0000C00000000000000010
:10B90000012100F01F029140DFF84C21400942F86C
:10B9100020107047012100F01F029140DFF83C2108
:10B92000400942F82010704780B50FF24810FFF729
:10B93000C1FDDFF82C010021016041610161BDE81A
:10B94000014003F092BF70477CB503F09AFF0446B4
:10B950000D46444ED6E900239D4208D801D39442B7
:10B9600005D2CDE900450FF28410FFF7A3FDC6E92B
:10B970000045204629467CBD80B503F082FF4FF488
:10B980007A72BDE8084004F0E3B8F8B504460D4605
:10B9900016461F4645EA040030430FD121460FF2F8
:10B9A0009010FFF787FD4FF4AD720FF2E4010FF234
:10B9B000D400FFF77FFD0020C046C046B6F57A7F71
:10B9C00008D34FF47A70B6FBF0F045194FF47A7152
:10B9D00001FB1066B5F57A7F08D34FF47A70B5FB9A
:10B9E000F0F004194FF47A7101FB105500F025F8BE
:10B9F0001B4A069810701C486421694300FB041020
:10BA000030180021C2E90201380000D01761324627
:10BA10002946204603F05FFFBDE8F14002E01048F0
:10BA20000078704780B5012004F05FF801200C49D0
:10BA300088701420BDE8024062E780B5002004F061
:10BA400054F8074800218170C078002803D11420E1
:10BA5000BDE802405EE701BD00E100E080E100E0FA
:10BA6000C0AC0300B8AD030040420F000020014607
:10BA7000704700005B495D727463496E69742E2ED5
:10BA80002E0A00005B455D25732C2025640A00000A
:10BA9000443A5C576F726B73706163655F31373125
:10BAA000335C4D4153535F4445565C706C61746622
:10BAB0006F726D5C6578796E6F73393631305C66A4
:10BAC00069726D776172655C6F735C706C617466CE
:10BAD0006F726D5C6578796E6F735C7372635C72A4
:10BAE00074635C7274632E63000000005B455D4FFD
:10BAF0006F7073212C206C6173745F73797374653C
:10BB00006D5F74696D655F6E7365632028256C6C6D
:10BB100075292C2073797374656D5F74696D655F29
:10BB20006E7365632028256C6C75290A000000007F
:10BB30005B455D7274635365745469636B54696DDE
:10BB4000652829202D2073656328256429206973C1
:10BB500020696E76616C69640A00000004F02CB8FC
:10BB600080B521280BDB25220FF2C4110FF2B4108F
:10BB7000FFF7A0FC0020BDE8024004F0E3BFBDE8F1
:10BB8000044004F029B880B521280CDB2E220FF2E6
:10BB9000A0110FF29010FFF78DFC0020C046C046A8
:10BBA0004FF0FF3002BDBDE8024004F033B880B56D
:10BBB00021280BDB39220FF278110FF26810FFF702
:10BBC00079FC0020BDE8024004F0BCBFBDE80440A1
:10BBD00004F03DB880B521280CDB45220FF250114E
:10BBE0000FF24010FFF766FC0020C046C0464FF041
:10BBF000FF3002BDBDE8024004F047B880B52128FF
:10BC00000BDB51220FF228110FF21810FFF752FC34
:10BC10000020BDE8024004F095BFBDE8044004F0F8
:10BC200053B880B521280BDB5E220FF204110FF20E
:10BC3000F400FFF73FFC0020BDE8024004F082BFA3
:10BC4000BDE8044004F05EB880B521280BDB6A2211
:10BC50000FF2DC010FF2CC00FFF72CFC0020BDE856
:10BC6000024004F06FBFBDE8044004F069B880B53D
:10BC700021280BDB76220FF2B8010FF2A800FFF7A4
:10BC800019FC0020BDE8024004F05CBFBDE80440A0
:10BC900004F074B838B521280BDB85220FF290012F
:10BCA0000FF28000FFF706FC0020BDE8324004F0F0
:10BCB00049BF05290BDB8A220FF274010FF26400E1
:10BCC000FFF7F8FB0020BDE8324004F03BBF012A3B
:10BCD0000DD1802B0BD38F220FF254010FF24400B1
:10BCE000FFF7E8FB0020BDE8324004F02BBF049CC6
:10BCF000250002D0009404F039FF31BD80B5212821
:10BD00000CDB4FF487720FF228010FF21800FFF7D7
:10BD1000D1FB0020BDE8024004F014BFBDE80240A2
:10BD200004F0DCB85B455D25732C2025640A000017
:10BD3000443A5C576F726B73706163655F31373182
:10BD4000335C4D4153535F4445565C706C6174667F
:10BD50006F726D5C6578796E6F73393631305C6601
:10BD600069726D776172655C6F735C706C6174662B
:10BD70006F726D5C6578796E6F735C7372635C670C
:10BD800070696F5C6770696F2E6300003548816869
:10BD9000002904BF08B008E0EFF30982A2F12802ED
:10BDA000036882E8F84F83685A60FBF7EBFF81680D
:10BDB00079B14A6892E8F84F036002F1280282F3F1
:10BDC000098890692849814202D013F47F4F43D0FB
:10BDD0007047264826490968401A80F308884FF0C2
:10BDE0008071C161234981617FF0060E704701BCFB
:10BDF0002046DFF884E000BDFEE7204800681C49CB
:10BE00000968401A203820F0070080F308884FF0B6
:10BE100000011448417081F3118862B600F018F8EF
:10BE2000FEE703680CB44FF0000141704FF00001D1
:10BE300081F311881249134A0A604FF0800181F39F
:10BE400011880CBC036070470D490E4A0A607047A8
:10BE50000B490C4A0A6070474FF0000181F31188CA
:10BE600070470000A03D03003ECE0000E80F030035
:10BE70004C900000D1050200F9CD00000010000038
:10BE800004ED00E00000001080B504F060FF0D49F3
:10BE9000086001BD80B500F043F80B4805F08EFE48
:10BEA000012005F0AAFEFFF759FE05F0F9FE05F0A6
:10BEB0000BFFFFF739FD0FF21400BDE80240FFF75A
:10BEC000F9BA00002846030000EA32065379737479
:10BED000656D20626F6F7420646F6E652021212173
:10BEE0000A00000030B50D4D2A78521C2A7081B02E
:10BEF0000124802282F3118800BF00BF8268C368DA
:10BF00009A4202D205F0EAFE0024687808B980F36C
:10BF10001188FBF7C5FF204601B030BDA03D0300EE
:10BF200080B506F013F806F0E5F806F062F9BDE812
:10BF3000014003F04BBCF8B504460D4616461F46BB
:10BF4000002C0DD10FF2F000FFF7B4FA36220FF2F9
:10BF500018110FF20810FFF7ADFA0020C046C046D6
:10BF6000002D0DD10FF26410FFF7A4FA3B220FF25F
:10BF7000F8010FF2E800FFF79DFA0020C046C04626
:10BF800006F07AF9002805D13A4631460FF25C10E6
:10BF9000FFF790FA29462046BDE8F44006F0A4B821
:10BFA000F8B504460D4616461F46002C0DD10FF27B
:10BFB0005810FFF77FFA49220FF2AC010FF29C00F4
:10BFC000FFF778FA0020C046C046002D0DD10FF2D1
:10BFD0005810FFF76FFA4E220FF28C010FF27C001F
:10BFE000FFF768FA0020C046C04630000DD10FF2BE
:10BFF0005810FFF75FFA53220FF26C010FF25C004A
:10C00000FFF758FA0020C046C0463B463246294654
:10C01000204601B0BDE8F04006F060B810B5044617
:10C0200006F0D4F8012C04D02046BDE8104006F0FC
:10C03000B2B810BD000000005B455D6D61696C62C7
:10C040006F7857726974652829202D2062756620E3
:10C050006973204E554C4C0A000000005B455D257D
:10C06000732C2025640A0000443A5C576F726B738E
:10C07000706163655F313731335C4D4153535F44C9
:10C0800045565C706C6174666F726D5C6578796E34
:10C090006F73393631305C6669726D776172655CD9
:10C0A0006F735C706C6174666F726D5C6578796ECD
:10C0B0006F735C7372635C6D61696C626F785C6DE9
:10C0C00061696C626F782E63000000005B455D6DF6
:10C0D00061696C626F7857726974652829202D2018
:10C0E00073697A6520697320300A00005B495D6DD1
:10C0F00061696C626F7857726974654576743A202D
:10C100002573282564290A005B455D6D61696C62B1
:10C110006F78526561642829202D20627566206938
:10C1200073204E554C4C0A005B455D6D61696C6235
:10C130006F78526561642829202D2073697A652003
:10C14000697320300A0000005B455D6D61696C62B7
:10C150006F78526561642829202D2063616C6C62C0
:10C1600061636B206973204E554C4C0A000000003F
:10C1700010B5044606F068FA01200549605410BD68
:10C18000002106F0D0BA06F01ABC06F071BC00001F
:10C19000C0AD03000C2802D36FF400407047854AFD
:10C1A00042F8201006F0E9BD2DE9F84F04460C2CAA
:10C1B00080F0898006F054FF05467F4810F814602F
:10C1C00000EB440047783046FFF7DDFC80463846F8
:10C1D000FFF7D9FC8146204606F00BFE3846FFF7F4
:10C1E000F9FC83463046FFF7F5FC82465246594635
:10C1F0000FF2C810FFF75EF9BBF1010F63D0BAF17F
:10C20000000F1AD14FF0000B04E00A2004F088FC64
:10C210000BF10A0BBBF5FA7F08D23046FFF7DAFCC8
:10C220008246BAF1000FF0D14FF0000BBBF1000FC6
:10C2300003D00FF2A810FFF73DF93846FFF7CAFC0C
:10C240008346BBF1000F2DD101213046FFF788FC5A
:10C2500000213846FFF784FC4FF0000A01E00AF1A4
:10C26000010ABAF1640F16DA00213046FFF79FFC8D
:10C27000052004F041FC01213046FFF798FC052021
:10C2800004F03AFC3846FFF7A5FC0128E7D10FF28D
:10C290006C10FFF70FF9BAF1640F03D10FF27810A9
:10C2A000FFF708F941463046FFF75AFC4946384641
:10C2B000FFF756FC204606F067FC29462046BDE8FD
:10C2C000F44F06F05ABDBDE8F18FF0B587B00446D3
:10C2D0001D460C2C01D2080602D56FF400401CE06C
:10C2E00001910D9E03960C9805900495069201A964
:10C2F000204606F061FE070004D02046FFF754FFF9
:10C3000038460AE00E98010006D00021009133461D
:10C310002A460F9906F0ACFF002007B0F0BD39E7C0
:10C320001FB5069C002C01D0002B02D16FF40040F9
:10C3300009E02270002203920292019300940123EB
:10C340002246FFF7C2FF04B010BD2DE9FF470546A6
:10C350000E4690469946DDF830A0BAF1000F02D0A3
:10C36000B9F1000F02D16FF4004020E009F101079C
:10C370003846FEF7FDFA040002D14FF0FF3016E018
:10C380004A465146601CF5F7C3FF84F80080002040
:10C3900003900290019000903B4622463146284689
:10C3A000FFF793FF05462046FEF7FAFA284604B049
:10C3B000BDE8F087F4AA0300984403005B495D538D
:10C3C0004441206C696E653A25642C2053434C200F
:10C3D0006C696E653A25640A000000005B455D5398
:10C3E000434C206C696E65206973207374696C6CB2
:10C3F000204C4F572121210A000000005B495D536A
:10C400004441206C696E65206973207265636F76A4
:10C41000657265640A0000005B455D534441206C11
:10C42000696E65206973206E6F74207265636F7624
:10C43000657265640A00000010B5EFF3108072B6F3
:10C440000A4C216841F47F01216080F31088A06EBE
:10C4500010F4700F04BFA72006F012FF4FF0007019
:10C46000C4F81C020020C4F8140210BD20ED00E046
:10C470002DE9F84C2DED068B154603B4C1F30A5097
:10C4800040F2FF7188420CD101980024000304BFE0
:10C490000098002802D1019800281BD4DDE9000192
:10C4A00013E101280FDA00A800F092F901280ADB55
:10C4B000FEF74AF92221016002B00020BDEC068B94
:10C4C000A249BDE8F48C019A40F2FE3161F31E529C
:10C4D0000192441A019800280CD5FEF735F9212164
:10C4E000016002B04FF0FF30BDEC068B6FF00041F1
:10C4F000BDE8F48CDDE90001954A964B00F0F0F9B7
:10C5000009D2DDE9002300204FF08041F9F772FDE8
:10C51000CDE90001641EDDE9002300208E49FAF711
:10C5200025F9DDE9002341EC180B00208B49FAF7CF
:10C530001DF902460B4651EC180BF9F733FF41EC9D
:10C54000190B53EC192BF9F755FD41EC1A0B53EC71
:10C550001A2B83488349F9F74DFD834A834BFAF739
:10C5600005F953EC1A2BF9F745FD814A814BFAF78F
:10C57000FDF853EC1A2BF9F73DFD7F4A7F4BFAF794
:10C58000F5F853EC1A2BF9F735FD7D4A7D4BFAF798
:10C59000EDF853EC1A2BF9F72DFD7B4A7B4BFAF79C
:10C5A000E5F853EC1A2BF9F725FD794A794BFAF7A0
:10C5B000DDF853EC1A2BF9F71DFD02460B4651EC42
:10C5C000180BFAF713F853EC192BF9F713FD41EC9C
:10C5D000190B20B2FBF718FD41EC1A0BCDB953EC47
:10C5E0001A2B6D486D49F9F705FD53EC192BF9F736
:10C5F000FDFF53EC182BFAF7B9F804460D4653EC3F
:10C600001A2B4FF040406649F9F7F4FC22462B46BE
:10C6100059E0012D53EC182B34DB00206149F9F768
:10C62000E9FC82468B4653EC182B5F485F49F9F7CB
:10C63000E1FC06460F4653EC1A2B5D485D49F9F7BD
:10C64000D9FC04460D4653EC192B5B485549F9F7C4
:10C65000D1FC02460B4620462946F9F7C7FF324671
:10C660003B46FAF783F852465B46FAF77FF80446F2
:10C670000D4653EC1A2B00205049F9F7BBFC22461B
:10C680002B4620E04FF0C0404D49F9F7B3FC04467B
:10C690000D4653EC182B4B484B49F9F7ABFC0646BB
:10C6A0000F4653EC192B49484549F9F7A3FC0246BC
:10C6B0000B4630463946F9F799FF22462B46FAF7E2
:10C6C00055F853EC1A2BFAF751F802B0BDEC068B73
:10C6D000BDE8F48C80B52DED028B41EC180B53ECCA
:10C6E000182B1F481F49F9F785FC1F4A1F4BFAF703
:10C6F0003DF853EC182BF9F77DFC1D4A1D4BFAF75A
:10C7000035F853EC182BF9F775FC1B4A1B4BFAF75D
:10C710002DF853EC182BF9F76DFC194A194BFAF761
:10C7200025F853EC182BF9F765FC174A174BFAF765
:10C730001DF853EC182BF9F75DFC154A154BBDECB1
:10C74000028BBDE80050FAF711B800000000F0FFBE
:10C75000CD3B7F669EA0E63F0000F0BF0000F03FAB
:10C76000F7DE29BFD8F8C23FF4B3FECC1A99C33F15
:10C7700062CB68D96F46C73FC6C912DAC471CC3FD5
:10C780004AE98A942449D23FF75F97999999D93F0A
:10C79000BC5555555555E53F9EBC9AF71C7D7F3ECF
:10C7A000422EE63F7BCBDB3FABA6320EE526553E65
:10C7B0007CC4BC7FDE27743E0EE526151344D33FB0
:10C7C0004715F73F44DF5DF80BAE543EFE822B6504
:10C7D00030B4436803F0004201211B031B0B43608C
:10C7E00004BF0368002B08D10DE00368DD0F45EAA4
:10C7F000440444605B000360491E4468E302F4D5CE
:10C8000023031B0B436043681A434260084630BC55
:10C8100070474268C2F30A5240F2FF739A4209D14C
:10C820004168090304BF0068002801D10120704756
:10C830000220704743685B0004BF0368002B25D0CB
:10C8400040F233439A1A521A012A1FDB352A06DBBB
:10C85000416801F0004141600021016013E00121C5
:10C8600002F01F039940491E920607D54268114005
:10C870004A40426002681143002202E0026811400F
:10C880004A40026011B14FF0FF30704700207047FE
:10C8900090420CD141EA030C50EA4C0C07D099426B
:10C8A00005D14FF4001C1CEB410F38BF8942704783
:10C8B0004FF4001C1CEB410F94BF1CEB430F09E02D
:10C8C00041EA030C50EA4C0C52EA0C0C03D28B42A6
:10C8D00008BF8242704714BF9942904270470000DF
:10C8E0004FF4001C1CEB410F94BF1CEB430F09E0FD
:10C8F00041EA030C50EA4C0C52EA0C0C03D2994268
:10C9000008BF9042704714BF8B42824270470000BC
:10C910002DE9704C04462DED088B94ED009B43EC03
:10C92000182B51EC190B06F0BFFC064651EC180B06
:10C9300006F0BAFC31000E9D06D500284DD4022821
:10C9400005D184ED008B42E1022EF8D121E050B9EF
:10C9500051EC190B0022344BFFF79AFF0FD084EDF6
:10C96000008B002033E1012818D151EC190B002273
:10C970002E4BFFF78DFF18BF84ED008B51D1FDF7D3
:10C98000E3FE212101604FF0FF306FF00041C4E968
:10C990000001BDEC088B0220BDE8708C7EB984EDEF
:10C9A000008B2946204606F09FFC040018BF012C8E
:10C9B00040F00C81FDF7C8FE2221016006E151EC38
:10C9C000190B0022184BFFF763FF0DD151EC180B28
:10C9D000F9F710FBC4E9000123E051EC190B002228
:10C9E000134BFFF77DFF0BD251EC180B0023F9F727
:10C9F00001FBC4E90001BDEC088B0020BDE8708C90
:10CA000001220C4BFFF754FF16D851EC180B0022F3
:10CA1000054BF9F7EFFAC4E90001FDF795FE222175
:10CA200001600120D3E000BF0000F07F0000F0FFB4
:10CA300000C89CC000C89C40384A394BF9F7DAFA64
:10CA400000220023FFF74CFF34BF9FED360B9FED14
:10CA5000370B53EC102BF9F789FEFAF727FC064643
:10CA6000FBF7D2FA41EC1A0B4FF07842314BF9F751
:10CA7000C1FA02460B4651EC190BF9F7B7FD824695
:10CA80008B4653EC1A2B2C482C49F9F7B3FA024683
:10CA90000B4650465946F9F7A9FD6FF00102284BA5
:10CAA000FFF706FF41EC190B05D80022254BFFF7D5
:10CAB00017FFC0F07D8053EC192BF9F79BFA41EC7E
:10CAC0001A0B214A214BF9F795FA214A214BF9F724
:10CAD0004DFE53EC1A2BF9F78DFA1F4A1F4B41EC10
:10CAE0001B0B51EC1A0BF9F785FA1D4A1D4BF9F790
:10CAF0003DFE53EC1A2BF9F77DFA1B4B0022F9F798
:10CB000035FE53EC192BF9F775FA41EC190B9FED33
:10CB100001AB2BE0000000000000F03FFE822B651F
:10CB20004715F73F000000000000E0BF00000000D4
:10CB30000000E03F422EE63FF2E4D5BCE7E84B3E82
:10CB4000FFFF8FBC0000903C112E5781A03F503F4B
:10CB50005843128C8F71BC3F4BE8A541B752013F3F
:10CB60000BBDF3DAE8708C3F0000E03F51EC1B0B8B
:10CB700053EC192BF9F7FAFD53EC1A2BF9F7F6FDE4
:10CB800082468B4651EC1B0B53EC192BF9F72EFD0B
:10CB900053EC1A2BF9F7EAFD02460B46504659466C
:10CBA000F9F700FC53EC182BF9F724FA41EC180BB9
:10CBB00084ED008BA919204606F096FB040018BFEF
:10CBC000012C03D1FDF7C0FD222101602046BDEC00
:10CBD000088BBDE8708C00002DE9F04FA1B08246B3
:10CBE000002017461D4602910B900DF1440B6FF08B
:10CBF00000490AE017F8011B0298D047029000286C
:10CC000000F0A8820B98401C0B90387808B90B985C
:10CC1000A2E22528EED1002005900690079008900A
:10CC200009900A9001E040F0010017F8011F202947
:10CC3000F9D023290DD02B2904D02D2906D0302955
:10CC40000AD00CE040F0020080B2EEE740F00400B1
:10CC5000FAE740F00800F7E740F01000F4E72A296F
:10CC60000ED12968296051F8042B2960002A0D9201
:10CC700004D5514240F004000D9180B27F1C11E0B8
:10CC800000210D9109E00D99494505D001EB810383
:10CC900002EB430130390D917F1C3A78A2F130014B
:10CCA0000A29F0D339782E2903D04FF0FF310C91A7
:10CCB0001DE017F8011F2A2907D1296829607F1C68
:10CCC00051F8042B29600C9211E000210C9109E02D
:10CCD0000C99494505D001EB810302EB4301303942
:10CCE0000C917F1C3A78A2F130010A29F0D3ADF8FB
:10CCF00038000FF67440397806F082FB08B117F857
:10CD0000010B8DF83A009DF83A00682802BF397887
:10CD10006829622005D06C2804BF38786C2803D1BC
:10CD200071208DF83A007F1C11A8049017F8014B70
:10CD3000B4F125002AD01C3800F0CC80001F022856
:10CD400040F2C880133800F0EE80093800F0C2804D
:10CD5000801E00F04F81401E00F02481401E0228FA
:10CD600040F2B880001F00F01D81401F00F083805A
:10CD7000401E00F0D880401E29D0C01E0CD0801E5E
:10CD800000F0D180C01E00F0CE803DE10120059072
:10CD900025208DF8440043E12868286050F8044BB2
:10CDA00028600394DDF83080B8F1000F04D52046E8
:10CDB000FBF762FE804607E042460021204606F06F
:10CDC0002BFB08B1A0EB0408CDF8188028E12968F6
:10CDD00029604FF03C0851F8040B29600021CDE98F
:10CDE000000111A80390DDE90001049C11B908B904
:10CDF0000C9AC2B10206120FA0EB02123032D2B26C
:10CE00003A2AA8BF27320009A8F1010340EA0170BD
:10CE100009091A5508BF0028984604D0039A08EB60
:10CE200004039A42E6D308EB04000390C8F13C01E6
:10CE30000C980691814209DA401A08904FF6EF717A
:10CE4000BDF838000840ADF83800E9E0002840F1AE
:10CE5000E7809DF8380000F01400102840F0E080D2
:10CE60000D98059A801A089A801A401A0128C0F273
:10CE7000D7800890D4E09DF83A0062281AD068283C
:10CE800006D06A280CD06C281CD0712808D019E074
:10CE90002868286050F8041B28600B980880BFE0C1
:10CEA0002868286050F8042B28600B98C117C2E945
:10CEB0000001B5E02868286050F8041B28600B9832
:10CEC0000870ADE02868286050F8041B28600B98B3
:10CED0000860A5E02868C01D20F007022A60D2E99A
:10CEE000000108322A60CDE90001002903D50120A4
:10CEF00005902D200CE0BDF83800810703D50120F6
:10CF000005902B2004E0C00704D5012005902020C7
:10CF10008DF84400059911A808180390214600A82F
:10CF200000F0D8F97CE09DF83A206C2A0DD0712AE7
:10CF300018BF6A2A09D12868C01D20F007032B609A
:10CF4000D3E9000108332B6005E02968296051F816
:10CF5000040B29600021CDE90001682A08BF80B2D6
:10CF600007D0622A08BFC0B203D0742A18BF7A2A39
:10CF700002D10021CDE900019DF83800000730D52D
:10CF8000DDE90001002908BF00282AD044F0200074
:10CF9000782826D130208DF844008BF801400220FB
:10CFA00005901EE09DF83A00294600F0D8F8CDE93A
:10CFB0000001002904DA0598411C05912D210EE09D
:10CFC000BDF83800810704D50598411C05912B2137
:10CFD00005E0C00705D50598411C0591202100F802
:10CFE0000B10059911A808180390214600A800F01D
:10CFF000EDF815E0012005902868286050F8041B22
:10D0000028608DF844100BE0012005902520002CAD
:10D010008DF8440004D00598411C059100F80B40A0
:10D020000D980599401A0899401A0699401A0999CD
:10D03000401A0799401A0A99A0EB01089DF8380098
:10D0400040070FD420208DF84000002408E0012381
:10D0500010AA00A9504600F070FC00287AD1641C88
:10D060004445F4DB059C11AE0AE016F8011B02985A
:10D07000D047029000286DD00B98401C0B90641E86
:10D08000002CF2D130208DF840000026089C08E0EA
:10D09000012310AA00A9504600F04FFC002859D1E6
:10D0A000761CA642F4DB069C039E0AE016F8011BE0
:10D0B0000298D047029000284CD00B98401C0B904F
:10D0C000641E002CF2D130208DF840000026099C0F
:10D0D00007E0012310AA00A9504600F02EFCC8BBAF
:10D0E000761CA642F5DB03980699079C0E1809E00A
:10D0F00016F8011B0298D047029058B30B98401CB9
:10D100000B90641E002CF3D130208DF840000026D7
:10D110000A9C07E0012310AA00A9504600F00DFC6C
:10D12000C0B9761CA642F5DB9DF8380040077FF5B4
:10D130006CAD20208DF84000002400E0641C4445C4
:10D14000BFF663AD012310AA00A9504600F0F5FB1D
:10D150000028F3D04FF0FF3021B0BDE8F08F6228F7
:10D1600026D068281DD06A2808D06C2827D07128BE
:10D1700004D0742823D07A280CD020E00868C01D81
:10D1800020F007000860D0E9002308300860194645
:10D19000104670470A680A6052F8040B0A600021C2
:10D1A00070470A680A6052F8040B0A6000B20BE08C
:10D1B0000A680A6052F8040B0A6040B204E00A6888
:10D1C0000A6052F8040B0A60C11770472DE9FA4E45
:10D1D00005460A462F696F2A08BF082405D041F08A
:10D1E0002000782814BF0A2410243C26D5E9000129
:10D1F000642A18BF692A81468A4605D1002903DAC4
:10D20000D9F100096AEB4A0ABAF1000F08BFB9F177
:10D21000000F0CD1286B50B9082C36D195F8380086
:10D22000000732D530203B2687F83B002DE0E3177E
:10D2300048465146224606F03DF9A4FB0023A9EBDF
:10D2400002023032D2B2A6F1010B3A2A5E4603DB6B
:10D250009DF80030513B9A1881465FEA010A0BF8AD
:10D26000072008BFB9F1000F03D0E868F119884220
:10D27000DDD3082C09D195F83800000705D5F05DFD
:10D28000302802D0761E3020F055C6F13C00A8614F
:10D29000F119E960296B884208DA081A28624FF60A
:10D2A000EF71288F08402887BDE8F38E00290ED53E
:10D2B00095F8381001F01401102908D1696B6A69DA
:10D2C000891A2A6A891A081A0128A8BF2862BDE8A3
:10D2D000F38E00002DE9F24F04468EB0D4E9000130
:10D2E000CDE9020104AF9DF8380040F0200BBBF1FE
:10D2F000610F0AD0206B002848BF062004D408BF65
:10D30000BBF1670F01D1012020636168C1F30A50AE
:10D3100040F2FF7290421CD1080304BF206800282D
:10D3200009D10320A0619DF8380061381A2836D34E
:10D330000FF2486108E00320A0619DF838006138D1
:10D340001A2829D30FF22C61E0680322F4F7E0FFDA
:10D35000BEE1012816DA2046FFF73AFA012811DB70
:10D3600000250020BBF1610F20D1E168302201F8D7
:10D37000012B4A1CE2609DF83820612A0CBF7822FC
:10D3800058220FE0626840F2FE3161F31E52451AE6
:10D3900062604FF0FF30E5E70FF2D451D4E70FF2AF
:10D3A000D851D1E70A706169891C616110B9002602
:10D3B000002584E1BBF1610F40F09780206B0028CD
:10D3C0004CBF2126461CDDE90201D4E900AB002256
:10D3D0000023FFF785FA36B23ABF8BF00040CDE963
:10D3E00002A0CDE902AB06F101082D1F8DF8102037
:10D3F0000DF1110700E0C71DB8F1010F33DBDDE9C6
:10D40000020100220023FFF753FA2CD21C2102A8AC
:10D4100005F06AFFDDE90201F9F748FFA8F1070806
:10D42000B8F1010F814609DBFAF7EEFD02460B4623
:10D43000DDE90201F9F7DAF8CDE90201F81D07216B
:10D4400005E009F00F0200F8012D4FEA2919B9F1A2
:10D45000010F01DB491EF4D5491E5CBF002200F814
:10D46000012DF9D5C7E70DF11100391AB142B8BF46
:10D470000E4636B230000DF111072FD4884206DA7D
:10D4800004A9411849780829A8BF0F2100DA002112
:10D4900004AA821800E0761E12F80139401E8B4261
:10D4A000F9D00F2904D104A941184A78521C4A70B6
:10D4B000002802D504AF761C2D1D36B2701E0DD487
:10D4C000C1190A783032D2B23A2A03DB9DF83830DB
:10D4D0003A3B9A18401E01F80129F2D5206B00282A
:10D4E00040F1ED80701E2063E9E0DDE902010022D9
:10D4F0000023FFF7F5F93CBF81F00041CDE90201BF
:10D500002DB247F2975068434B49DFF8309190FBBA
:10D51000F1F52DB2C5F1070ABAF1010F90461CDBF7
:10D52000DDE902675FEACA7007D542464B463046DE
:10D530003946F8F75FFD06460F464FEA6A0A40464D
:10D54000494642464B46F8F755FDBAF1000F804672
:10D550008946E7D1CDE9026724E0CAF1000A002636
:10D56000374F14E05FEACA7007D542464B46304653
:10D570003946F8F73FFD06460F464FEA6A0A40462D
:10D58000494642464B46F8F735FD80468946BAF192
:10D59000000FE7D1DDE9020132463B46F8F702FF12
:10D5A000CDE90201BBF1660F216BDFF898900CBF4B
:10D5B00005F10A0006204618142EA8BF13263020B5
:10D5C0008DF810000DF11107012E3DDBDDE90201A0
:10D5D000F9F782FE07F1080104220A23B0FBF3F3F6
:10D5E00003EB8307A0EB4700303001F8010D0A2060
:10D5F000B3FBF0F000EB8007A3EB47033033521E80
:10D6000001F8013DE9D1083E012E01F10807DBDBFD
:10D61000DDE90201F9F760FEFAF700FD02460B466C
:10D62000DDE90201F8F7E2FF00224B46F8F7E2FCE1
:10D63000CDE90201CAE700BFA08601000000244036
:10D640000000F03F84D797410DF11100381A0DF119
:10D65000110702E0401E6D1E7F1C39783029F9D079
:10D66000BBF1660F02D12DB2691C04E0BBF1650F5E
:10D670000CBF01210021226B8E1836B2B042B8BF18
:10D68000064636B231001AD4814204DAC85D352824
:10D69000A8BF392000DA3020CA19521E00E0761ED9
:10D6A00012F80139491E8342F9D0392802D1C85DE8
:10D6B000401CC855002902D57F1E761C6D1C2DB25A
:10D6C0009DF83810009533B23A46204600F003F832
:10D6D0000FB0BDE8F08F2DE9F043054685B01E463A
:10D6E000D5F83080012E8946174602DA01260FF25E
:10D6F000902749F02000BDF93040662808BF641C1F
:10D7000017D0672840F0828014F1040FC0F28480A3
:10D71000444580F2818095F83800641C000702D4EB
:10D720004645B8BFB04624B2B8EB040848BF4FF036
:10D73000000824B2E868A969012C25DA4A1C3023C4
:10D740000B54B8F1010F03DA95F83810090702D528
:10D750002E211154521C18EB040FB8BFC8F100045D
:10D7600024B26142A044B045AA61B8BF464669628E
:10D7700036B2EE613246AB6939461818F4F7C8FD87
:10D78000A8EB0600A862C1E00818A64218DA3246E3
:10D790003946F4F7BDFDA9697118A01BA961B8F15C
:10D7A000010F686203DA95F83800000705D5EA68CA
:10D7B0002E208854E869401CE861C5F82880A5E05F
:10D7C00022463946F4F7A4FDA8692018361BB8F1A3
:10D7D000010F03DA95F83810090703D5EA682E21FE
:10D7E0008154401CA86136B2B045B8BF4646E868CF
:10D7F000AB6936B23246E1191818F4F789FDA86909
:10D800003018A861A8EB060068627FE0B9F1610FEB
:10D8100016D14FF0700918E0464504DA95F8381033
:10D82000090758BFB046B8F1010848BF4FF00008DB
:10D83000B9F1670F14BF4FF045094FF0650904E0D7
:10D84000B9F1410F08BF4FF05009A969E86817F80E
:10D85000013B0B544A1CB8F1010F05DA95F838105A
:10D86000090758BFAA6117D52E211154531CB8F1CE
:10D87000010FAB6110DB761E36B2B045B8BF46462D
:10D8800036B2324639461818F4F742FDA869301806
:10D89000A861A8EB06006862E868A9690F18200073
:10D8A00007F8019B03D42B2007F8010B03E02D217F
:10D8B00007F8011B644200260DF1080808E00A225F
:10D8C00000A805F06EFE019808F8010B761C009C7C
:10D8D00021B20129F3DA022E06DA49F02000652888
:10D8E00004BF302007F8010B4EB9302007F8010BB8
:10D8F00007E0761E02A8305C303007F8010B012EDD
:10D90000F7DAE868A9690818381AE86195F8380064
:10D9100000F0140010280DD16869A9690818696A17
:10D920000818E9690818A96A0818696B8842BCBF19
:10D93000081A286205B0BDE8F083F8B504460D4624
:10D9400016461F46002004E0E86A401CE8627F1E7D
:10D95000002047B116F8011BA868A047A86000285E
:10D96000F2D14FF0FF30F2BD686A6C747A4C00005F
:10D970006E616E004E414E00696E6600494E460073
:10D980003000000010B5DFF8A84500224FF4F07118
:10D990002046F4F78FFCDFF89C05606410BD0000A2
:10D9A00010B5DFF88C45A1894118A181E289801862
:10D9B000E081207A192803DA401C207284ED110AD4
:10D9C000DFED700AB4EE600AF1EE10FAC0F2958055
:10D9D00094ED111AB4EE601AF1EE10FAC0F28D80D7
:10D9E000207A1928C0F2898089B2C329C0F28580C3
:10D9F000207904EB800080ED280A84ED110AE0799B
:10DA0000002804D184ED120A84ED130A17E0D4ED46
:10DA1000120A9FED5D1A60EE810A9FED5C1A40EEDE
:10DA2000010AC4ED120A94ED130A9FED591A20EE73
:10DA3000010A9FED581A00EE810A84ED130AE0896D
:10DA4000B0F57A7F14DDA07904EB8000E16CC0F8BA
:10DA50004011A079401CA071C0B2142801D100204F
:10DA6000A071607A142801DA401C60720020E08105
:10DA70002279E17914290DD1501C142800D10020FD
:10DA800094ED0F0A04EB8000D0ED3C0A30EE600A02
:10DA900084ED0F0A04F1A00000F086F9207904EB70
:10DAA000800080ED3C0AD4ED0F0A30EE800A84ED50
:10DAB0000F0A207904EB8000E16C0165207904EB0A
:10DAC0004000A1890182E079142801DA401CE0714C
:10DAD000E07900EE100AB8EE400AD4ED0F0A80EEAD
:10DAE000800A84ED100A2079401C2071C0B21428ED
:10DAF00001D1002020710020A08110BDDFF830048A
:10DB000081794A1E00D51432891F00D5143100EBEB
:10DB1000810191ED500A00EB8200D0ED500A91EDA9
:10DB2000501A70EEC10AF5EE400AF1EE10FAD0ED8F
:10DB3000500A02DD30EEC00A704730EE600A7047CE
:10DB4000DFF8EC0381794A1E00D51432891F00D515
:10DB5000143100EB810191ED3C0A00EB8200D0ED25
:10DB60003C0A91ED3C1A70EEC10AF5EE400AF1EE66
:10DB700010FAD0ED3C0A02DD30EEC00A704730EEFC
:10DB8000600A70470100FA436666663FD0CCCC3D20
:10DB9000CDCC4C3FCCCC4C3E2DE9F84F2DED088B35
:10DBA000F0EE409A074688464FF000094C469FED3C
:10DBB000798ADFED788A9FED779A9FED76AAA24663
:10DBC000FFB2042F04D1DFED74AA9FED74BA03E015
:10DBD000DFED73AA9FED73BADFF8545395F807B0E1
:10DBE0005E46142E40F0CF80687A0728C0F2CB80C2
:10DBF000F5EE409AF1EE10FA40F3C580FFF77EFF94
:10DC0000F0EE40BAFFF79CFFF4EE6BAAF1EE10FACB
:10DC100034D5D5ED100AF5EE400AF1EE10FA02DD2A
:10DC2000B0EE601A01E0B1EE601AB4EE41BAF1EE66
:10DC300010FA23D5F5EE400AF1EE10FA01DCF1EE10
:10DC4000600A9FED7B1AF4EE410AF1EE10FA15D549
:10DC5000DFED780AB4EE600AF1EE10FA0ED528680E
:10DC6000002802D0A86BA8EB000A3B465246594652
:10DC70002879401E00F0E4F8814602E02046286042
:10DC8000A863B9F1000F7BD02868002803D1C5F83C
:10DC9000388001202860204605E005EB4101098A13
:10DCA0000C19A4B2401C80B201461429F5DB00EE29
:10DCB000104AB8EE400ADFED970A20EE200ADFEDA9
:10DCC0005F0A69EEA00A20EE200A2879411E00D5DD
:10DCD0001431801B00D5143005EB8101D1ED140AFD
:10DCE00005EB800090ED141A70EEC10A9FED521AF8
:10DCF000C0EE819AF4EE409AF1EE10FA02DBDFED0D
:10DD0000259A07E020EE000A09EEE90AF4F7B6FAD0
:10DD1000B0EE408AB5EE408AF1EE10FA01D0C9EEBD
:10DD2000888A687905EB8000C0ED648A6879401CB8
:10DD30006871C0B2142801D100206871A87A142833
:10DD400001DA401CA872002006E005EB800191ED8D
:10DD5000640A39EE009A401CA97A0A4680B29042C1
:10DD6000F3D3B2EE040A29EE000A00EE901AF8EEA0
:10DD7000600A80EE200ADFED680A20EE20AA02E0A9
:10DD800020466871A872B0EE4A0ABDEC088BBDE867
:10DD9000F18F000000000000CDCC4C3EA69B443B20
:10DDA000CDCC4C3D6F12033B10B49FED5C0ADFED10
:10DDB0005B0A9FED5A1ADFED591A00231AE0142C62
:10DDC00000DB143C02EE103AB8EEC22A32EE000A32
:10DDD00050F8244002EE904A70EEA20A02EE221A97
:10DDE00013FB03F402EE104AB8EEC22A72EE211AB7
:10DDF0005B1CDBB20C46A34205DA141B1C19641C25
:10DE0000DDD51434DEE702EE101AB8EE422A22EE17
:10DE1000011A00EE601A62EE210A40EE400A9FED00
:10DE2000400A30EE800A81EE000A10BC7047000004
:10DE30000AD7233C0AD7A33C8FC2F5BD3B89883C57
:10DE4000F0B51C460023002801D5143002E0142848
:10DE500000DB14381D461E46042C04D19FED310A08
:10DE6000DFED310A03E09FED2B0ADFED300A1C469F
:10DE70000CE0B4EE410AF1EE10FA06D5B4EE601AE9
:10DE8000F1EE10FA01D5761CB6B2641C0F46E4B26E
:10DE9000A446A7F1010EF4452EDAC71B67447F1C88
:10DEA00001D5143702E0142F00DB143F07F1010CF9
:10DEB000BCF1140F01DBACF1140CDFF874E00EEBD5
:10DEC0008C0C9CED141A0EEB8707D7ED141A31EE6B
:10DED000611AFFEE001A20EE212AB4EE421AF1EE8A
:10DEE00010FAC6D560EEA11AF4EE411AF1EE10FA5E
:10DEF000BFD56D1CADB2C8E7072A01D20C2000E0E7
:10DF00000A20B04201D2012302E0A84200D202233B
:10DF10001846F0BD6F12833ACDCCCC3D0000000016
:10DF2000BD3786356F12033B8FC2F53C8FC2753CFF
:10DF30000C8C030000407E44B5EEC00AF1EE10FAEE
:10DF400002D4B1EEC00A70476FF0004C00EE10CA68
:10DF5000FCF708BD10EE101A04204FF07E5C01EEB5
:10DF600090CA49004FEA510100EE101A88BF0820FC
:10DF7000B1F17E5F13D871EEC00ADFF838C031EE20
:10DF8000801A61EE200AF1EEE00A614586BF80F05A
:10DF9000040080EE800A80EE200AFCF7DBBB49001B
:10DFA00011F1807F9CBF6FF0004100EE101A7CF6EB
:10DFB000D9AC7047F404353F0268C2F3C752FF2A58
:10DFC00006D10068400201D101207047022070474D
:10DFD00003685B0016D0C2F19602521A012A11DBC7
:10DFE000182A04DB016801F00041016007E001210B
:10DFF00091400268491E11404A40026011B14FF041
:10E00000FF3070470020704710EE100A10EE901A93
:10E01000A4464FF0FF034FEA410103EAD0540A0E31
:10E020001CBF94EA030F92EA030F55D0B1EB400FE7
:10E030002ED24FEAC11141F0004100F000434FEAF7
:10E04000002040F000404FEA9000890864EB020491
:10E05000401A38BF01EB400018BF54F1000407D04C
:10E06000D1EB400038BF081818BFB4F10104F7D154
:10E0700040002CD0B0FA80F100FA01F0521A0EDB09
:10E0800043EA102000EBC25000EE100A64467047CD
:10E0900008BF00F0004000EE100A6446704743EAF3
:10E0A000102000EE100A02F17F024FEAC25100EE8A
:10E0B000901AF1EE100A20F4F851E1EE101A20EE59
:10E0C000200AE1EE100A10EE100A64467047184666
:10E0D00000EE100A6446704709421CBF94EA030F21
:10E0E00092EA030F1CD04FF0984201EE102A60EE26
:10E0F000810AB1EB400FCBD2244208BF20EE010AC7
:10E1000010EE901A03EAD152A2F119024FEA01214E
:10E1100091D110EE100A03EAD054A4F119048CE74F
:10E120004FF0807212EB400F2CBF6FF0004011F1E6
:10E13000807F644618BF6FF0004000EE100AFCF4C8
:10E1400011AC70470349044A096801B91146801AA5
:10E150004018704700AE03000000030070B504468D
:10E160003748384E0568B5B1287A88B16868A0424A
:10E170000ED1012028723078401C3070287A401E61
:10E180002872C0B210B9284605F012FAF9F788FED5
:10E19000ED68002DE8D170BD2B492C4A0A600021A2
:10E1A00000220B468C46A0E80E101038802181F327
:10E1B000118800BF00BF22490A68C2600860214878
:10E1C000407808B980F31188704730B51D4D04467A
:10E1D0002878401C287081B0A868217A39B960601D
:10E1E00001252572F9F75CFE284601B030BD616853
:10E1F000814208D01021204605F0F0F9207A00284D
:10E20000F8D1A8686060207A451C2572F9F748FEAD
:10E21000284601B030BD0B490A78521C0A70017AB9
:10E22000491E0172C9B2002918BFF9F739BE00B5FD
:10E2300081B005F0BDF901B05DF804EBF9F730BE2F
:10E24000F8AD0300A03D0300D0AD03005DF1000078
:10E2500000F5E0700268914203D343689A18914236
:10E2600002D380680028F5D17047DFF860070168A5
:10E2700091B94FF4803181604FF4805141604FF08B
:10E28000FF31C16001610421DFF844274161C2F818
:10E29000BC11DFF8401701600120704701F108034D
:10E2A00013F0070305D001F10803C3F1080303F0DD
:10E2B00007035918D21A8161C26042F001034B6012
:10E2C000511828234B60DFF804170969C1617047B2
:10E2D0002DE9F04F064601F1080010F0070083B069
:10E2E00008BF884607D001F10800C0F1080000F01F
:10E2F000070000EB010802F1080010F0070006D04B
:10E3000002F10800C0F1080000F00700821815466D
:10E31000A5EB0800A0EB030943F0030003EB080B97
:10E32000C8F80400AB4528BF05F076F92879C00786
:10E3300058BF05F071F9B9F1100F38BF05F06CF94D
:10E34000B069854209D1F0684844F060C6F818B059
:10E3500040F00100CBF804006DE1706985420BD1FB
:10E36000B0684844B060C6F814B040F00101CBF882
:10E37000041040F80B005EE1686800F00301012919
:10E3800040F0AD80C008C0000190C00820283AD2FB
:10E39000D5F808A0EF680090BD4208BF05F03CF931
:10E3A000554508BF05F038F968680099C008C000F5
:10E3B000B0EBC10F18BF05F02FF9009806EBC000B5
:10E3C00000F128018A4507D031698A45C0F0828072
:10E3D000DAF80C10A9427DD1574506D1009A306871
:10E3E000012191408843306076E02830874205D093
:10E3F000306987426ED3B868A8426BD1CAF80C70F6
:10E40000C7F808A068E0EF68D5F818A0AF420CD0B4
:10E41000A8683169884223D3C168A94204BFB9689A
:10E42000A9421DD1C760B8601CE005F1140007685F
:10E4300037B905F110000768A7B101E00846076881
:10E4400007F114010A68002A02BF07F110010A68E7
:10E45000002AF3D13169884202D30021016001E032
:10E4600005F0DAF8BAF1000F36D0E86906EB800063
:10E4700000F5987001688D4208D10760A7B9EA6974
:10E480007068012191408843706025E030698245C1
:10E4900008D3DAF81000A84214BFCAF81470CAF8FA
:10E4A000107001E005F0B8F8B7B13069874211D3B8
:10E4B000C7F818A0296929B1814226BF39618F6147
:10E4C00005F0AAF8686938B13169884202D37861E9
:10E4D000876101E005F0A0F801984519814468685A
:10E4E0004008400068604FEAD90549F00100CBF8C8
:10E4F000040049F80B90202D23D206EBC50000F153
:10E500002807B9F1100F38BF05F086F8306820FAF7
:10E5100005F1C907BA4604D40121A9400843306077
:10E5200006E0B868316988422CBF824605F074F86D
:10E53000C7F808B0CAF80CB0CBF808A0CBF80C703C
:10E5400079E05FEA192108BF002023D0B1F5803FB0
:10E5500028BF1F201ED2A1F58070000C00F008001B
:10E560008140A1F58052120C02F004029140A1F505
:10E5700080431B0CC0F10E0003F00203801AC01A86
:10E58000994000EBD130C11D29FA01F202F00101DE
:10E5900001EB4000CBF81C000022CBF81420CBF894
:10E5A000102006EB8001726822FA00F3DB0701F508
:10E5B000987107D4012303FA00F010437060C1F88A
:10E5C00000B01DE01F2809680EBF00204008C0F100
:10E5D000190009FA00F000E011464A68D208D2009A
:10E5E0004A4514D0C20F01EB820202F11003400031
:10E5F0001A68002AF0D1306983421AD3C3F800B0F8
:10E60000CBF81810CBF80CB0CBF808B013E0326997
:10E610008868914228BF90420BD3C0F80CB0C1F873
:10E6200008B0CBF80800CBF80C100020CBF818008D
:10E6300001E004F0F1FF08F1080000F005BE2DE94B
:10E64000FA4D0546DFF88403006884B008B9FFF787
:10E650000CFEDFF878030499806841182F31401EC2
:10E6600021EA00000499814280F0AB8105F5D8765B
:10E67000B16841B1D5F8B0218018824280F0A18103
:10E680008142C0F09E8104F0CBFF00281EBF0446EB
:10E69000D0F8008014F1010F00F09381D5F8B0019B
:10E6A0004044C5F8B0017168814238BF01467160CD
:10E6B000A86980BB286908B1844200D22C6134610A
:10E6C000C6F814800020F06105F12801BF480068F9
:10E6D00068624FF0FF3028620020C960896001F154
:10E6E0000802801C1031D26020289260F5D3B8480F
:10E6F000854203D1A8F12802214629E055F8040CEF
:10E70000C00805EBC000A0F1080108EB0400401AA6
:10E71000A0F128021CE005F5E071084600E08068E1
:10E72000D0B1026843689A189442F8D1027B12076C
:10E7300012D4AA6903689A420ED347683B449A42AE
:10E740000AD208EB07014160E868A96908EB0002FA
:10E750002846FFF7A3FD1EE128698442084638BF1A
:10E760002C6108EB040100E0806880B102688A42F5
:10E77000FAD1017B09070AD4046041684144416031
:10E780002146049B284606B0BDE8F04DA0E5AF69E0
:10E7900039462846FFF75CFD016840684018029042
:10E7A0002F3800F1080111F0070105D000F1080130
:10E7B000C1F1080101F00701081807F110018842B2
:10E7C00034BF0097009000980830019004F10801D0
:10E7D000009800F1180A11F007014FF0000BA8F1A2
:10E7E000280005D004F10801C1F1080101F007017A
:10E7F0000A19401AAA61E86040F0010151608018CE
:10E800002821416071480069E861019810F0070013
:10E8100018BF04F001FF00991B20486005F5E07166
:10E82000B1E80C500198A0E80C503461C6F814808F
:10E83000C6F81CB00198B061029800E08A46072231
:10E84000CAF804200AF104010A1D82420BF1010BEF
:10E85000F4D3BBF1020FB8BF04F0DEFE0098B8425B
:10E8600000F09980C01BC119C4084A6852085200C0
:10E870004A6040F001017960C051202C20D205EBA4
:10E88000C40101F12806102838BF04F0C5FE28682D
:10E8900020FA04F1C907B04604D40121A14008437D
:10E8A000286006E0B068296988422CBF804604F0E1
:10E8B000B3FEB760C8F80C70C7F80880FE606AE065
:10E8C000010A08BF002223D0B1F5803F28BF1F22D4
:10E8D0001ED2A1F58072120C02F008029140A1F53F
:10E8E00080531B0C03F004039940A1F58044240CD1
:10E8F000C2F10E0204F00204D21A121BA14002EB74
:10E90000D131CA1D20FA02F303F0010202EB4102E9
:10E91000FA6100237B613B6105EB82016B6823FA9E
:10E9200002F4E40701F5987105D4012090401843E2
:10E9300068600F601CE01F2A09680EBF00225208A1
:10E94000C2F1190200FA02F200E019464B68DB0836
:10E95000DB00834210D0D30F01EB830303F11004DB
:10E9600052002368002BF0D12869844211D327601C
:10E97000B961FF60BF600EE02A698868914228BFD4
:10E98000904206D3C7608F60B860F9600020B8611C
:10E9900001E004F041FEE8680499814211D2401A76
:10E9A000E860A969049A5218AA6140F00100506019
:10E9B000049840F00300486006B001F10800BDE88B
:10E9C000F08D002006B0BDE8F08D0000D8AC03004B
:10E9D000489003006859883C2DE9F04D044688466C
:10E9E00000265FEA1820C8F1000B08BF002123D0E1
:10E9F000B0F5803F28BF1F211ED2A0F58071090C01
:10EA000001F008018840A0F58052120C02F00402C7
:10EA10009040A0F580431B0CC1F10E0103F00203EE
:10EA2000891AC91A984001EBD030C11D28FA01F2A9
:10EA300002F0010101EB400104EB8100D0F830014C
:10EA400028B31F290EBF00224A08C2F1190208FA92
:10EA500002F2002300E052004768FF08FF00A7EB26
:10EA600008075F4503D25FEA070B06460BD04769EC
:10EA7000D50F00EB8500002F00691CBF87423B4685
:10EA80000028E8D1184600283CD1002E3CD10120B6
:10EA900088404000414208436168084000F06781B7
:10EAA00041420840411E080B00F0100021FA00F21C
:10EAB000510901F0080122FA01F39A0802F0040753
:10EAC000FB405A0802F00205081823FA05F2384400
:10EAD000C2F340032818181822FA03F1081804EBAF
:10EAE0008000D0F830010DE008464168C908C9002F
:10EAF000A1EB080159453CBF8B4606460169002938
:10EB0000F2D140690028F0D1002E00F03081A068D9
:10EB1000A0EB0800834580F02A8120698642C0F07E
:10EB200024817068C008C00008EB0B01884208EB24
:10EB3000060518BF04F070FDAE4280F01681F7683C
:10EB4000D6F818A0B7420CD0B0682169884223D308
:10EB5000C168B14204BFB968B1421DD1C760B86095
:10EB60001CE006F11400076837B906F110000768C9
:10EB7000A7B101E00846076807F114010A68002AF6
:10EB800002BF07F110010A68002AF3D12169884207
:10EB900002D30021016001E004F03EFDBAF1000F54
:10EBA00038D0F06904EB800000F5987001688E425F
:10EBB00009D10760380014D1F269606801219140E1
:10EBC0008843606026E02069824508D3DAF81000A7
:10EBD000B04214BFCAF81470CAF8107001E004F013
:10EBE0001BFDBFB12069874212D3C7F818A0306956
:10EBF00030B12169884226BF3861876104F00CFD7D
:10EC0000706938B12169884202D37861876101E077
:10EC100004F002FDBBF1100F0CD208EB0B0040F02A
:10EC20000300706008EB0B008019416841F001019E
:10EC3000416096E048F0030070604BF001006860AE
:10EC40004FEADB004BF805B020281DD204EBC001D1
:10EC500001F12807216821FA00F2D207BB4605D44A
:10EC6000012202FA00F00843206006E0B86821693A
:10EC700088422CBF834604F0CFFCBD60CBF80C501B
:10EC8000C5F808B0EF606CE05FEA1B2108BF002008
:10EC900023D0B1F5803F28BF1F201ED2A1F5807080
:10ECA000000C00F008008140A1F58052120C02F027
:10ECB00004029140A1F580431B0CC0F10E0003F04B
:10ECC0000203801AC01A994000EBD130C11D2BFA03
:10ECD00001F202F0010101EB4000E86100226A61EB
:10ECE0002A6104EB8001626822FA00F3DB0701F578
:10ECF000987106D4012303FA00F0104360600D60A0
:10ED00001CE01F2809680EBF00204008C0F1190050
:10ED10000BFA00F000E011464A68D208D2005A45CA
:10ED200010D0C20F01EB820202F1100340001A68FA
:10ED3000002AF0D12069834211D31D60A961ED60E2
:10ED4000AD600EE022698868914228BF904206D3E8
:10ED5000C5608D60A860E9600020A86101E004F052
:10ED60005BFC06F10800BDE8F08D04F055FC0020C6
:10ED7000BDE8F08D2DE9F84F0446884660684142B1
:10ED80000840411E080B00F0100021FA00F2510962
:10ED900001F0080122FA01F39A0802F0040223FAB2
:10EDA00002F56B0803F00203081825FA03F61018A1
:10EDB000C6F340051818284426FA05F1081804EB94
:10EDC0008000D0F830014168C908C9000646A1EBAF
:10EDD000080A09E008464168C908C900A1EB080112
:10EDE00051453CBF8A46064601690029F2D1406977
:10EDF0000028F0D120698642C0F0C4807068C00845
:10EE000008EB0A09C000484508EB060B18BF04F0E0
:10EE100003FC5E4580F0B680F768B569B7420CD058
:10EE2000B0682169884223D3C168B14204BFB96880
:10EE3000B1421DD1C760B8601CE006F1140007683C
:10EE400037B906F110000768A7B101E00846076866
:10EE500007F114010A68002A02BF07F110010A68CD
:10EE6000002AF3D12169884202D30021016001E028
:10EE700004F0D2FB002D34D0F06904EB800000F5E3
:10EE8000987001688E4209D10760380011D1F2698B
:10EE90006068012191408843606022E020698542DA
:10EEA00005D32869B04214BF6F612F6101E004F0FF
:10EEB000B3FBB7B12069874211D3BD61306930B16E
:10EEC0002169884226BF3861876104F0A5FB70691B
:10EED00038B12169884202D37861876101E004F08A
:10EEE0009BFBBAF1100F09D249F00300706009EBE7
:10EEF0000600416841F0010141603FE048F0030035
:10EF000070604AF00100CBF804004AF80BA0D4F876
:10EF100008804FEAD805202D28BF04F07DFBB8F10A
:10EF2000000F27D0D4F81490009504EBC50000F131
:10EF30002805B8F1100F38BF04F06EFB2068009967
:10EF400020FA01F2D1072F4605D4009A0121914001
:10EF50000843206006E0A868216988422CBF074664
:10EF600004F05AFBC5F80890C7F80C90C9F808706F
:10EF7000C9F80C50C4F808A0C4F814B006F1080091
:10EF8000BDE8F28F04F048FB0020BDE8F28F2DE9C8
:10EF9000F04F83B00546C046C046F52DDFF8C047A8
:10EFA00080F007810B2D31BF102705F10B00C00841
:10EFB000C7002168FE0821FA06F010F0030F42D0C6
:10EFC000C04300F00100861904EBC60000F12808D8
:10EFD000F700D8F808506868C008C000B84218BFE9
:10EFE00004F01AFBD5F80890454508BF04F014FB5F
:10EFF0004D4508BF04F010FB6868C008C000B84267
:10F0000018BF04F009FBC84505D120680121B140B3
:10F01000884320600DE02069814508D3D9F80C00B1
:10F02000A84204D1C8F80890C9F80C8001E004F0A7
:10F03000F3FA47F00300686078190835416841F039
:10F0400001014160FDE0A168B94280F0C480002860
:10F0500000F0A680012505FA06F149004A42B040B9
:10F060001143084041420840411E080B00F01000C7
:10F0700021FA00F2510901F0080322FA03F18A088B
:10F0800002F0040221FA02F6710801F002081818D1
:10F0900026FA08F11018C1F340064044301821FA4E
:10F0A00006F202EB000804EBC80000F128094FEA61
:10F0B000C80AD9F808607068C008C000504518BF79
:10F0C00004F0AAFAD6F808B04E4508BF04F0A4FA36
:10F0D0005E4508BF04F0A0FA7068C008C000504543
:10F0E00018BF04F099FAD94505D1206805FA08F14E
:10F0F000884320600DE02069834508D3DBF80C00CD
:10F10000B04204D1C9F808B0CBF80C9001E004F08B
:10F1100083FA47F003007060AAEB0708B819019062
:10F1200048F0010001994860019848F80080A768FC
:10F130004FEAD70ABAF1200F28BF04F06DFA47B39F
:10F14000CDF800A004EBCA00D4F8149000F1280A0E
:10F15000102F38BF04F060FA2068009920FA01F2FD
:10F16000D107D34605D4009905FA01F10843206080
:10F1700007E0DAF80800216988422CBF834604F0D2
:10F180004BFACAF80890CBF80C90C9F808B0C9F847
:10F190000CA0C4F8088006F108050198606150E0F1
:10F1A0006068C0B339462046FFF7E4FD050012D081
:10F1B00047E015F1400F28BF4FF0FF370BD205F1A4
:10F1C0000B00C008C700606828B139462046FFF729
:10F1D00003FC050035D1A068B8421CD3C11B62698D
:10F1E00010290AD3B8186061A16041F0010343609F
:10F1F000095047F0030050600AE00021A1606161FE
:10F2000040F0030151608018416841F00101416004
:10F2100002F1080515E0E06887420DD2C01BA16924
:10F22000E0607A18A26140F00100506001F1080529
:10F2300047F00300486004E039462046FFF7FFF935
:10F240000546C046C046284603B0BDE8F08F00B969
:10F2500070472DE9F047A0F10804C046C046DFF82A
:10F26000005528698442C0F07482616801F003028D
:10F27000012A00F06E82CA084FEAC208CA0708EBEA
:10F28000040936D4226811F0030F00F06482A41A36
:10F2900084429044C0F05D8269698C4200F0D8805D
:10F2A000D608202E70D2D4F80CA0A768544508BF09
:10F2B00004F0B2F9BC4208BF04F0AEF96068C008BF
:10F2C000C000B0EBC60F18BF04F0A6F905EBC600EE
:10F2D00000F128018F4205D029698F4251D3F96886
:10F2E000A1424ED1BA453DD128680121B1408843A1
:10F2F00028604C4580F02D82D9F80400C10740F108
:10F300002882810700F17A81A969894540F0B5809A
:10F31000E868AC614044E86040F0010161606969FF
:10F320008C4202D100216961A960E969814280F0C3
:10F330001282DFF83004006808B9FEF796FFA96969
:10F34000002900F00882E868292824BF2846FEF733
:10F350007FFFE869E968884280F0FD814FF0FF3067
:10F36000E861F8E12830824506D02869824508D353
:10F37000DAF80800A04204D1C7F80CA0CAF8087057
:10F38000B7E704F049F9B4E7E768A669A7420BD0EC
:10F39000A168814222D3C868A04204BFB868A042D5
:10F3A0001CD1CF60B9601BE004F114010F6837B9BC
:10F3B00004F110010F689FB101E011460F6807F1D9
:10F3C00014021368002B02BF07F110021368002B10
:10F3D000F3D1814202D30020086001E004F01CF95F
:10F3E000002E86D0E06905EB800000F5987001687A
:10F3F0008C4209D10760380011D1E26968680121A7
:10F4000091408843686074E72869864205D3306973
:10F41000A04214BF7761376101E004F0FDF8002FCE
:10F420003FF467AF28698742ABD3BE61216929B138
:10F43000814226BF39618F6104F0EEF860690028CF
:10F440003FF457AF296988429BD37861876150E7C1
:10F4500099F8040000F0030003287FF44AAFC5F8D0
:10F460000880D9F8040040084000C9F8040048F0BA
:10F470000100606048F804806DE16969894508D140
:10F48000A8686C614044A86040F0010161600051CF
:10F4900061E1C008C0004FEAD00ABAF1200F8044F1
:10F4A00036D2D9F80C70D9F80860B94508BF04F015
:10F4B000B3F8B14508BF04F0AFF8D9F80400C008AC
:10F4C000C000B0EBCA0F18BF04F0A6F805EBCA00E5
:10F4D00000F128018E4206D029698E42C0F0818059
:10F4E000F16849457DD1B74206D12868012101FA6A
:10F4F0000AF18843286076E02830874205D02869E1
:10F5000087426ED3B86848456BD1F760BE606AE049
:10F51000D9F80C70D9F818604F450DD0D9F808000B
:10F520002969884223D3C168494504BFB968494560
:10F530001DD1C760B8601CE009F11400076837B935
:10F5400009F110000768A7B101E00846076807F154
:10F5500014010A68002A02BF07F110010A68002A94
:10F56000F3D12969884202D30021016001E004F04F
:10F5700053F8002E37D0D9F81C0005EB800000F5B9
:10F580009870016889450AD10760380012D1D9F80E
:10F590001C206868012191408843686023E0286945
:10F5A000864205D33069484514BF7761376101E071
:10F5B00004F032F8BFB12869874212D3BE61D9F88E
:10F5C000101029B1814226BF39618F6104F024F8FF
:10F5D000D9F8140038B12969884202D3786187616B
:10F5E00001E004F019F848F00100606048F8048078
:10F5F000686984420BD1C5F80880ACE0400840003F
:10F60000C9F8040048F00100606048F804804FEA3F
:10F61000D807202F22D205EBC70000F12809B8F146
:10F62000100F38BF03F0F8FF286820FA07F1C90768
:10F630004E4604D40121B9400843286007E0D9F8B8
:10F640000800296988422CBF064603F0E5FFC9F887
:10F650000840F460A660C4F80C907CE05FEA1820D3
:10F6600008BF002123D0B0F5803F28BF1F211ED244
:10F67000A0F58071090C01F008018840A0F58052C6
:10F68000120C02F004029040A0F580431B0CC1F163
:10F690000E0103F00203891AC91A984001EBD03019
:10F6A000C11D28FA01F202F0010101EB4001E16104
:10F6B00000226261226105EB81006A6822FA01F38F
:10F6C000DB0700F5987006D4012303FA01F111431A
:10F6D000696004601CE01F2900680EBF0021490812
:10F6E000C1F1190108FA01F100E010464268D208A0
:10F6F000D200424510D0CA0F00EB820202F1100383
:10F7000049001A68002AF0D129698B4211D31C6084
:10F71000A061E460A4600EE02A698168904228BF7D
:10F72000914206D3CC608460A160E0600020A061BB
:10F7300001E003F071FF286A401E28620BD1D5F862
:10F74000C80100E080680028FCD14FF0FF3028623B
:10F7500001E003F061FFC046C046BDE8F08700004D
:10F7600048900300D8AC0300234A42F820107047A9
:10F770000146032001F053BF00F11001032001F006
:10F7800028BF10B50446FFF7F7FF1B4850F82410B8
:10F790000A0008D122460FF274010FF28800BDE87A
:10F7A0001040FBF787BE002C01D0012C01D1884707
:10F7B00003E0022C01D180688047002C01D0012C8D
:10F7C00003D12046BDE81040D2E710BD80B501222C
:10F7D0000A49032001F0B7FEF7F775FE084900203B
:10F7E000FFF7C2FF07490120FFF7BEFF06490220CD
:10F7F000BDE80440B8E7000068A9030000003940F4
:10F80000513201005B320100058300006D61696CBB
:10F81000626F78476E737344727668616E646C656C
:10F82000497271005B455D25733A2057726F6E67B0
:10F8300020696E746572727570742068617070658D
:10F840006E6564286576656E743A2025642900002B
:10F85000DFF8D0120A68002803D042F001000860E7
:10F8600070475008400008607047DFF8B8024FF05A
:10F87000FF314160092101604FF480710160002077
:10F88000E6E7F0B4DFF8A4120A6E086810F001038E
:10F89000DFF894020CD00A6ED0E902454FF014460E
:10F8A00047F23577A4197D41C0E9024501230B6079
:10F8B000DFF87C12A1FB0223D20B42EA4342D0E9DB
:10F8C0000245121955EBD333D0E90045101943EB2B
:10F8D0000501F0BC7047F8B505460E461746DFF83F
:10F8E00044422068400403D50FF24820FBF7E2FDB4
:10F8F0006FF00040854201D30F20EEE0B5F1804F5C
:10F900000CD30E2079004FF47A72B1FBF2F101EBC7
:10F910004601B1FBF2F101EB4505DEE0B5F1005F18
:10F920000CD30D20B9004FF47A72B1FBF2F101EB68
:10F930008601B1FBF2F101EB8505CEE0B5F1805F08
:10F940000CD30C20F9004FF47A72B1FBF2F101EB09
:10F95000C601B1FBF2F101EBC505BEE0B5F1006FE8
:10F960000CD30B2039014FF47A72B1FBF2F101EBA9
:10F970000611B1FBF2F101EB0515AEE0B5F1806FB8
:10F980000CD30A2079014FF47A72B1FBF2F101EB4A
:10F990004611B1FBF2F101EB45159EE0B5F1007F98
:10F9A0000CD30920B9014FF47A72B1FBF2F101EBEB
:10F9B0008611B1FBF2F101EB85158EE0B5F1807F88
:10F9C0000CD30820F9014FF47A72B1FBF2F101EB8C
:10F9D000C611B1FBF2F101EBC5157EE0B5F5000FE4
:10F9E0000CD3072039024FF47A72B1FBF2F101EB2C
:10F9F0000621B1FBF2F101EB05256EE0B5F5800FB4
:10FA00000CD3062079024FF47A72B1FBF2F101EBCC
:10FA10004621B1FBF2F101EB45255EE0B5F5001F93
:10FA20000CD30520B9024FF47A72B1FBF2F101EB6D
:10FA30008621B1FBF2F101EB85254EE0B5F5801F83
:10FA40000CD30420F9024FF47A72B1FBF2F101EB0E
:10FA5000C621B1FBF2F101EBC5253EE0B5F5002F63
:10FA60000FD3032040F6FE7101FB07F24FF47A73C7
:10FA7000B2FBF3F201FB0622B2FBF3F201FB052518
:10FA80002BE0B5F5802F0CD3022079034FF47A7266
:10FA9000B1FBF2F101EB4631B1FBF2F101EB45357F
:10FAA0001BE0B5F5003F0CD30120B9034FF47A7287
:10FAB000B1FBF2F101EB8631B1FBF2F101EB8535DF
:10FAC0000BE00020F9034FF47A72B1FBF2F101EB85
:10FAD000C631B1FBF2F101EBC535A560216821F417
:10FAE000705141EA80202060F1BD0E490A6800286B
:10FAF00003D042F480400860704722F480400860E0
:10FB000070470A490A6802F004021043086070470F
:10FB1000002006490A6812F004020A6000D00120A1
:10FB2000704700004000424048AD030030004240B2
:10FB300000CA9A3B5B495D525443205469636B2071
:10FB400069732072756E6E696E67200A000000008E
:10FB5000F0B492B213460246B1FBF3F403FB141067
:10FB6000110C01EB0041B1FBF3F0254600240646E1
:10FB7000274647EA164714EB06447D4103FB101065
:10FB8000000410FA82F0B0FBF3F000212018694164
:10FB9000F0BC7047012100F01F029140874A4009E4
:10FBA00042F820107047012100F01F029140844A62
:10FBB000400942F82010704710B5002403E02046A9
:10FBC00000F065F9641C072CF9DB0420FFF7EBFF5C
:10FBD0000420BDE81040DDE718B4342212FB00F029
:10FBE0000FF2BC3283185C68002C11D0805C00F0EE
:10FBF0000F00DA690092009A12686043714B53F863
:10FC0000243083409A4301FA00F0104300990860C1
:10FC100011BC704781B0342111FB00F00FF280312C
:10FC200042185368002B02D14FF0FF300DE0D2692B
:10FC30000092009A1268405C00F00F005843114691
:10FC4000C140604850F82300084001B0704718B424
:10FC5000342212FB00F00FF2483283189C68002C0B
:10FC600011D0805C00F00F001A6A0092009A1268AE
:10FC70006043544B53F8243083409A4301FA00F018
:10FC800010430099086011BC704781B0342111FB0A
:10FC900000F00FF20C3142189368002B02D14FF0A4
:10FCA000FF300FE0405C00F00F00116A00910099F6
:10FCB000096803FB00F2434850F8230090400140DC
:10FCC0000846D04001B0704718B4342212FB00F04F
:10FCD0000FF2CC228318DC68002C11D0805C00F07D
:10FCE0000F005A6A0092009A12686043354B53F82D
:10FCF000243083409A4301FA00F0104300990860D1
:10FD000011BC704718B4342212FB00F00FF290229D
:10FD100083181C69002C11D0805C00F00F009A6AD7
:10FD20000092009A12686043264B53F824308340B7
:10FD30009A4301FA00F010430099086011BC704723
:10FD400018B4342212FB00F00FF2542283185C69BD
:10FD5000002C11D0805C00F00F00DA6A0092009A4B
:10FD600012686043174B53F8243083409A4301FADA
:10FD700000F010430099086011BC704718B4342299
:10FD800012FB00F00FF2182283189C69002C11D08E
:10FD9000805C00F00F001A6B0092009A12686043BA
:10FDA000084B53F8243083409A4301FA00F0104383
:10FDB0000099086011BC70470000000000E100E0FD
:10FDC00080E200E0404503002DE9F8430F46154668
:10FDD0001E4600EBC0014FEA81080FF6780908EBD8
:10FDE00009040F21207CFFF7F7FE58F8090061692C
:10FDF00000910099096807228240914307FA00F0B8
:10FE00000843009908606768A0690090009800683E
:10FE1000FF21B94020EA0108012D0CD1802E0AD320
:10FE20004FF4B0720FF218110FF20810FBF742FBFB
:10FE30000020C046C046002D12D0012D05D146F04D
:10FE40008000B84040EA08080AE040F26B120FF266
:10FE5000F0010FF2E000FBF72DFB0020C046C0468A
:10FE60000098C0F80080206A00900120E16800FA44
:10FE700001F1009A1160E169009100990968A26896
:10FE8000904021EA000000990860BDE8F18310B5B8
:10FE900082B00FF2C07100EBC00201EB82040021BE
:10FEA000207CFFF799FEE06900900098006801212E
:10FEB000A26801FA02F21043009A1060206A0090D2
:10FEC000E06801FA00F00099086013BD0FF2847138
:10FED00000EBC00201EB8200007CD6E681B00FF29D
:10FEE000747100EBC00201EB8200C168006A0090EF
:10FEF000009800680246CA40D00703D50120884018
:10FF00000099086001B0704781B00FF2487100EBB2
:10FF1000C00201EB8200016A009100990968C06883
:10FF20000A46C240D00701D5012000E0002001B000
:10FF3000704700005B455D25732C2025640A000096
:10FF4000443A5C576F726B73706163655F31373130
:10FF5000335C4D4153535F4445565C706C6174662D
:10FF60006F726D5C6578796E6F73393631305C66AF
:10FF700069726D776172655C6F735C706C617466D9
:10FF80006F726D5C6578796E6F735C7372635C67BA
:10FF900070696F5C6770696F4472762E6300000051
:10FFA0000000000004000000010000000400000048
:10FFB00004000000020000000400000000001840DF
:10FFC00004001840080018400C00184010001840A9
:10FFD00014001840010000000400000001000000AF
:10FFE0000400000004000000020000000400000003
:10FFF0000000184004001840080018400C00184089
:020000021000EC
:100000001000184014001840020000000400000016
:1000100001000000040000000400000002000000D5
:1000200004000000000018400400184008001840B8
:100030000C00184010001840140018400300000085
:1000400004000000010000000400000004000000A3
:1000500002000000040000000000184004001840E6
:10006000080018400C0018401000184014001840F8
:100070000000000004000000010000000400000077
:1000800004000000020000000400000020001840EE
:1000900024001840280018402C0018403000184058
:1000A00034001840010000000400000001000000BE
:1000B0000400000004000000020000000400000032
:1000C0002000184024001840280018402C00184038
:1000D0003000184034001840020000000400000006
:1000E0000100000004000000040000000200000005
:1000F0000400000020001840240018402800184088
:100100002C00184030001840340018400000000057
:1001100004000000010000000400000004000000D2
:100120000000000000000000000062400400624087
:10013000080062400C0062401C0062401C006240EB
:1001400000000000040000000100000004000000A6
:1001500004000000000000000000000020006240D9
:1001600024006240280062402C0062403C00624053
:100170003C0062400000000004000000010000009C
:100180000400000004000000000000000000000067
:100190004000624044006240480062404C006240BF
:1001A0005C0062405C00624000000000040000004F
:1001B0000100000004000000040000000000000036
:1001C000000000006000624064006240680062401D
:1001D0006C0062407C0062407C00624000000000D5
:1001E0000400000001000000040000000400000002
:1001F00000000000000000008000624084006240B7
:10020000880062408C0062409C0062409C0062401A
:1002100000000000040000000100000004000000D5
:10022000040000000000000000000000A000624088
:10023000A4006240A8006240AC006240BC00624082
:10024000BC0062400000000004000000010000004B
:100250000400000004000000000000000000000096
:10026000C0006240C4006240C8006240CC006240EE
:10027000DC006240DC00624000000000040000007E
:100280000100000004000000040000000000000065
:1002900000000000E0006240E4006240E8006240CC
:1002A000EC006240FC006240FC0062400000000084
:1002B0000400000001000000040000000400000031
:1002C00000000000000000000001624004016240E4
:1002D000080162400C0162401C0162401C01624046
:1002E0000000000004000000010000000400000005
:1002F0000400000000000000000000002001624037
:1003000024016240280162402C0162403C016240AD
:100310003C016240000000000400000001000000F9
:1003200004000000040000000000000000000000C5
:100330004001624044016240480162404C01624019
:100340005C0162405C0162400000000004000000AB
:100350000100000004000000040000000000000094
:100360000000000060016240640162406801624078
:100370006C0162407C0162407C0162400000000030
:100380000400000001000000040000000400000060
:100390000000000000000000800162408401624013
:1003A000880162408C0162409C0162409C01624075
:1003B0000000000004000000010000000400000034
:1003C000040000000000000000000000A0016240E6
:1003D000A4016240A8016240AC016240BC016240DD
:1003E000BC016240000000000400000001000000A9
:1003F00004000000040000000000000000000000F5
:10040000C0016240C4016240C8016240CC01624048
:10041000DC016240DC0162400000000004000000DA
:1004200001000000040000000400000000000000C3
:1004300000000000E0016240E4016240E801624027
:10044000EC016240FC016240FC01624000000000DF
:10045000040000000100000004000000040000008F
:100460000000000000000000000262400402624040
:10047000080262400C0262401C0262401C026240A0
:100480000000000004000000010000000400000063
:100490000400000000000000000000002002624094
:1004A00024026240280262402C0262403C02624008
:1004B0003C02624000000000040000000100000057
:1004C0000400000004000000000000000000000024
:1004D0004002624044026240480262404C02624074
:1004E0005C0262405C026240000000000400000008
:1004F00001000000040000000400000000000000F3
:1005000000000000600262406402624068026240D3
:100510006C0262407C0262407C026240000000008B
:1005200004000000010000000400000004000000BE
:10053000000000000000000080026240840262406F
:10054000880262408C0262409C0262409C026240CF
:100550000000000004000000010000000400000092
:10056000040000000000000000000000A002624043
:10057000A4026240A8026240AC026240BC02624037
:10058000BC02624000000000040000000100000006
:100590000400000004000000000000000000000053
:1005A000C0026240C4026240C8026240CC026240A3
:1005B000DC026240DC026240000000000400000037
:1005C0000100000004000000040000000000000022
:1005D00000000000E0026240E4026240E802624083
:1005E000EC026240FC026240FC026240000000003B
:1005F00004000000010000000400000004000000EE
:10060000000000000000000000036240040362409C
:10061000080362400C0362401C0362401C036240FA
:1006200000000000040000000100000004000000C1
:1006300004000000000000000000000020036240F1
:1006400024036240280362402C0362403C03624062
:100650003C036240000000000000000000000000B9
:1006600000000000000000000007184000081840CB
:1006700000091840000A18400400000008000000AB
:100680000100000001000000010000000007184008
:100690000008184000091840000A1840080000002F
:1006A0001000000002000000020000000200000034
:1006B000000718400008184000091840000A1840B8
:1006C0000C00000018000000030000000300000000
:1006D00003000000000718400008184000091840F7
:1006E000000A1840000000000000000000000000A8
:1006F000000000000400000004071840040818402F
:1007000004091840040A1840040000000800000012
:10071000010000000100000005000000040718406F
:100720000408184004091840040A18400800000092
:10073000100000000200000002000000060000009F
:10074000040718400408184004091840040A184017
:100750000000000000000000000000000000000099
:100760000700000000076240000862400009624084
:10077000000A6240000000000000000000000000CD
:100780000000000008000000040762400408624006
:1007900004096240040A62400000000000000000FA
:1007A000000000000000000009000000080762408F
:1007B0000808624008096240080A62400000000020
:1007C0000000000000000000000000000A0000001F
:1007D0000C0762400C0862400C0962400C0A62403F
:1007E0000000000000000000000000000000000009
:1007F0000B000000100762401008624010096240C0
:10080000100A62400000000000000000000000002C
:10081000000000000C000000140762401408624051
:1008200014096240140A6240000000000000000049
:1008300000000000000000000D00000018076240EA
:100840001808624018096240180A6240000000005F
:100850000000000000000000000000000E0000008A
:100860001C0762401C0862401C0962401C0A62406E
:100870000000000000000000000000000000000078
:100880000F000000200762402008624020096240FB
:10089000200A62400000000000000000000000008C
:1008A000000000001000000024076240240862409D
:1008B00024096240240A6240000000000000000099
:1008C0000000000000000000110000002807624046
:1008D0002808624028096240280A6240000000009F
:1008E00000000000000000000000000012000000F6
:1008F0002C0762402C0862402C0962402C0A62409E
:1009000000000000000000000000000000000000E7
:100910001300000030076240300862403009624036
:10092000300A6240000000000000000000000000EB
:1009300000000000140000003407624034086240E8
:1009400034096240340A62400000000000000000E8
:1009500000000000000000001500000038076240A1
:100960003808624038096240380A624000000000DE
:100970000000000000000000000000001600000061
:100980003C0762403C0862403C0962403C0A6240CD
:100990000000000000000000000000000000000057
:1009A0001700000040076240400862404009624072
:1009B000400A62400000000000000000000000004B
:1009C0000000000018000000440762404408624034
:1009D00044096240440A6240000000000000000038
:1009E00000000000000000001900000048076240FD
:1009F0004808624048096240480A6240000000001E
:100A00000000000000000000000000001A000000CC
:100A10004C0762404C0862404C0962404C0A6240FC
:100A200000000000000000000000000000000000C6
:100A30001B000000500762405008624050096240AD
:100A4000500A6240000000000000000000000000AA
:100A5000000000001C00000054076240540862407F
:100A600054096240540A6240000000000000000087
:100A700000000000000000001D0000005807624058
:100A80005808624058096240580A6240000000005D
:100A90000000000000000000000000001E00000038
:100AA0005C0762405C0862405C0962405C0A62402C
:100AB0000000000000000000000000000000000036
:100AC0001F000000600762406008624060096240E9
:100AD000600A62400000000000000000000000000A
:100AE00000000000200000006407624064086240CB
:100AF00064096240640A624010B582B00446032073
:100B000001F05EF80549B0FBF1F0604300900098F9
:100B1000411E00910028FAD113BD0000404B4C004B
:100B200010B582B00446032001F04AF841F2883142
:100B3000B0FBF1F0604300900098411E0091002846
:100B4000FAD113BD70470000012100F01F0291404F
:100B50004E4A400942F820107047012100F01F0260
:100B600091404B4A400942F820107047F8B500EB1D
:100B70004004A500474E069CAF197C600127AF5189
:100B80000094FFF721F9F1BDF8B500260420FFF726
:100B9000E4FF34460AE02A460FF2FC010FF220106F
:100BA000FAF788FC2046FFF799F9641CE4B2254661
:100BB000072D21DA2046FFF7A7F90028F5D00126F6
:100BC00005EB4500800033494258002AE3D047181E
:100BD0007868002805D02046FFF778F979688847BB
:100BE000E3E72A460FF2B0010FF2BC00FAF762FC0D
:100BF0002046FFF773F9D8E7002E05D10FF29801D0
:100C00000FF2E000FAF756FC0420BDE8F2409BE743
:100C100070B504461320FFF7A0FF25462046FFF7D6
:100C200073F9002826D005EB450080001949425889
:100C3000002A14D046187068002805D02046FFF717
:100C400045F9716888471CE02A460FF2B0010FF29F
:100C50005800FAF72FFC2046FFF740F911E02A462A
:100C60000FF298010FF25800FAF724FC2046FFF724
:100C700035F906E02A460FF284010FF29400FAF7E4
:100C800019FC1320BDE870405EE7000000E100E0C1
:100C900080E100E0AC9A03006770696F5F495251D0
:100CA00048616E646C6572005B455D25732C206342
:100CB00062206E756C6C20282564290A00000000F3
:100CC0005B455D25732C20696E74207365656D73BB
:100CD000207375707572696F757320282564290AF1
:100CE000000000005B455D25732C206E6F20706551
:100CF0006E64696E6720696E740A00006770696FC0
:100D0000436D677049525148616E646C65720000B2
:100D10005B455D25732C20696E74206973206E6FAE
:100D2000742070656E64696E6720282564290A0046
:100D3000DFF8401908607047DFF8381951F83000C3
:100D40007047DFF8301901EBC0004068704780B58C
:100D50000120FFF7F1FF406C02BD10B504460120F1
:100D6000FFF7EAFFA0F84A4010BD2DE9F04F93B01D
:100D70000020FFF7E1FF074607F580760FF67414B1
:100D80000FF634150B223146284602F05FFC00288E
:100D90000BD00196009533460FF6081221460FF648
:100DA0002410FAF787FB0020F7E03069DFF8C83835
:100DB000984209D000900FF6EC0221460FF6401041
:100DC000FAF778FB0020E8E0DFF8A858AE60F06999
:100DD000C0192861706BC0192865706AC019A861B4
:100DE000F16AC919A965F16BC9192967B1697269F5
:100DF000891A6960316AF269891A6961B16B726B2B
:100E0000891A6965B16A726A8A1AEA61316BF36A92
:100E1000C91AE965316CF36BC91A6967A86746F2AC
:100E20002C41DFF858389A180A50A86F00F5C442D0
:100E30009C322A624FF4BE726A6200F5C8431B1DE1
:100E4000AB620023EB6200F5C24320332B636A637D
:100E500000F5C4428832AA630022EA63A86443F220
:100E6000900213182B64EA646A6400F5C8423832B1
:100E70002A66085868668318AB666020E866A86929
:100E8000E969081803F1600188420AD2B06A01904A
:100E9000602000900FF60C0221460FF69C00FAF736
:100EA00009FB686F0A90286F0990686D0890286D9B
:100EB0000790E86D0690A86D0590E8690490A86910
:100EC00003906869029028690190686800902B6817
:100ED000326921460FF69800FAF7ECFA0D20FFF779
:100EE00030FF12900D20FFF727FF11900C20FFF725
:100EF00028FF10900C20FFF71FFF0F900420FFF732
:100F000020FF0E900420FFF717FF0D900620FFF73B
:100F100018FF0C900620FFF70FFF06460820FFF78A
:100F200010FF07460820FFF707FF80460920FFF75C
:100F300008FF81460920FFF7FFFE82460320FFF7E6
:100F400000FF83460320FFF7F7FE12990B911199DA
:100F50000A91109909910F9908910E9907910D998D
:100F600006910C99059104960397CDF80880CDF869
:100F70000490CDF800A05B46024621460FF66400BF
:100F8000FAF798FA1E200090102340F20132214611
:100F90000FF6DC00FAF78EFAA86F13B0BDE8F08FF9
:100FA000FFF7BEBD01684068814201D10120704752
:100FB0000020704701684068491C01F00F01814220
:100FC00001D101207047002070472DE9F04182B027
:100FD00004460E4617460025002C01D1092000E0EA
:100FE0000820FFF7A9FE804640F20230874226DA49
:100FF00072B64046FFF7DEFF002814D1D8F8000093
:101000004FF4427101FB0080103007603A463146D0
:10101000001DF1F77DF9D8F80000401C00F00F002A
:10102000C8F8000009E00FF684020FF2C8610FF65D
:101030008C00FAF73FFA6FF0150562B60AE03B46FE
:101040000FF668020FF2AC610FF68400FAF732FA7D
:101050006FF01505002D12D12046401E8041C0437F
:10106000C00F002100F007F9050017D00FF63C0271
:101070000FF280610FF67400FAF71CFA0EE0D8F850
:101080000030D8F8040000900FF620020FF26461DF
:101090000FF67400FAF70EFA00F00FFA2846BDE8D2
:1010A000F68170B50C46002801D1092000E0082027
:1010B000FFF742FE0546002672B6FFF773FF0028D1
:1010C0000DD168684FF4427101FB00501030016887
:1010D00021606968491C01F00F016960061D62B654
:1010E000304670BD1CB50820FFF726FE0268436835
:1010F0008168C0680FF2FC540190009121460FF600
:101100002800FAF7D7F90920FFF716FE02684368AE
:101110008168C0680190009121460FF63800FAF707
:10112000C9F913BD00B583B0DFF84805806F00F53D
:10113000C840243081680191416800910368C26809
:101140000FF2B0510FF63800FAF7B4F907BDF8B551
:10115000DFF82045A06F002805D10FF64C010FF6EF
:101160005400FAF7A7F9002010E043F29001414340
:101170000022A36FCA50A36FCB185A60A36FCB187D
:101180009A600122A36FC918CA60401C0228ECDBD8
:10119000002000F02FFA002146F2201711E000EBAA
:1011A0004003A66F961916EB8306BD51A66F9619DC
:1011B00016EB830346F22416F550401C1E28EEDB86
:1011C000491C022921DA4FF4BE7000FB01F2002015
:1011D000A36FD31846F28C25E850A36FD31846F2BC
:1011E0008825E850A36FD31846F29025E8500120D7
:1011F000A36FD31846F29425E8500020A36FD318AC
:1012000046F29825E850FF25D8E7F1BD10B4DFF885
:101210006414896F4FF4BE7212FB001000F5C242D5
:101220002032002072B602F5B4714B68D2F86841E2
:10123000A3420CD003EB430002EB8000002282604B
:101240004A68521C1E2A00D100224A6010E08C68B5
:10125000002C0DD003EB430002EB800000228260E3
:101260004A68521C1E2A00D100224A6000228A606D
:1012700062B610BC70472DE9FE4F0E46DFF8F4133E
:10128000896F4FF4BE7212FB001101F5C24720377F
:10129000022802DA4FF0000801E04FF004084FF096
:1012A0000009002F06D0B8F1000F0FF248440FF2EA
:1012B000207515D043460FF218720FF238410FF225
:1012C0001C70FAF7F7F84FF0FF309DE009EB89004A
:1012D000009033462A4621460FF2D470FAF7EAF816
:1012E00072B607F5B47ADAF80800002840F08E806C
:1012F000D7F8680100EB400117EB810B08D12946B4
:101300000FF20070FAF7D6F862B64FF0FF307BE0CC
:10131000DAF81010002000F028F90290002844D0DC
:10132000002000F04AF9019002980090DAF810309D
:101330002A4621460FF2E460FAF7BCF80520FFF7D1
:101340002FFEDAF81010002000F00FF9002804D06A
:10135000484600F101090528F0DBDAF810100020FA
:1013600000F003F90346CDF80490DAF8100000907D
:101370002A4621460FF2CC60FAF79CF8DAF81010F2
:10138000002000F0F2F800280FD0DAF8101000204A
:1013900000F0EBF803462A4621460FF2E860FAF720
:1013A00089F862B64FF0FF302EE0CBF800600120E4
:1013B000CBF80800DAF81000CBF80400D7F8680181
:1013C000401C1E2800D10020C7F86801DAF8100080
:1013D000401C0F2800D10320CAF81000D7F868017C
:1013E000DAF80410884202D10120CAF8080062B677
:1013F000B8F1040F07D0BBF1000F24D0DBF80410C4
:10140000404600F00CF90020BDE8FE8F62B60520D2
:10141000FFF7C6FDDAF80800002804D0484600F1BE
:1014200001090528F3DBDAF8080000283FF44EAF85
:101430002A4621460FF2A060FAF73CF800F03DF88A
:101440004FF0FF30E0E74FF0FF30DDE77FB589492F
:10145000896F4FF4BE7212FB001101F5C2442034B3
:10146000012801D181A300E081A304F5B4700FF23B
:101470008425016903918168029140680190D4F844
:1014800068010090224629460FF27060FAF712F8C0
:1014900000260FE006EB4600800001198A680192E1
:1014A000496800910359324629460FF28060FAF7E5
:1014B00001F8761C1E2EEDDB7FBD38B50FF234240B
:1014C0000FF28C652A4621460FF29060F9F7F2FF81
:1014D0000120FFF7BBFF2A4621460FF29860F9F77B
:1014E000E9FF0020FFF7B2FF2A4621460FF29C6079
:1014F000F9F7E0FFFFF7F6FD2A4621460FF2A46058
:10150000F9F7D8FFBDE831400CE630B4594B9C6F79
:10151000002C16D046F224410A59521C0C19E568D9
:101520006D1CE5609C6F0D592C1946F23845285505
:10153000986F0B189B689A4202D100220A5000E073
:101540000A5030BC704710B44D4B03EBC0046160CF
:1015500003F8302010BC7047494911F830000028CA
:1015600001D0102070470020704710B4444A02EBAD
:10157000C003012412F830000028586804D0806AA3
:1015800004FA01F1084004E04069103104FA01F165
:10159000084010BC70473A4B03EBC000406800EBBA
:1015A0008200C0F880107047354A02EBC0004068E6
:1015B00000EB8100D0F880007047314901EBC00298
:1015C00011F830000028506801D040697047806AE7
:1015D000704710B42A4A02EBC003012404FA01F157
:1015E00012F830000028586801D0C16000E00162A4
:1015F00010BC704738B504464FF6FF750020FFF762
:10160000ABFF05FA00F01E4901EBC40211F83410DB
:101610000029516801D0C86031BD086231BD38B5BC
:1016200004460D46002C01D100F01CFE144800EBCE
:10163000C401012210F83400002804D002FA05F099
:101640004968C86131BD05F1100002FA00F049682F
:10165000886031BD0A4A02EBC000406801607047F3
:101660000448806F46F218410858704741324300E1
:1016700043324100EC8D030020C30200689BFFFF52
:101680008CAB030038B505460121FFF78DFF0446FA
:1016900002212846FFF788FF22460146002010431A
:1016A00034BD00006970635F6765745F636875626D
:1016B0005F6D6170000000004E616E6F68756220A2
:1016C0004F5300005B455D25733A2025733A202572
:1016D00070206861732077726F6E67206D61676933
:1016E00063206B65793A202573202D3E2025730AEF
:1016F000000000006E616E6F6875622D6970630096
:101700005B455D25733A2025733A206970635F76E7
:10171000657273696F6E20646F65736E2774206DD8
:10172000617463683A2041502025642C2043687519
:10173000623A2025640A00005B495D25733A202542
:10174000733A2077726F6E67207065727369737475
:1017500062756620616464723A25702C2025642CC1
:10176000206970635F656E643A307825780A0000FE
:101770005B495D25733A20636F6E74657874687594
:1017800062206D617020696E666F726D6174696F41
:101790006E28762575290A20626C2825702025641C
:1017A000290A206F73282570202564290A20697072
:1017B00063282570202564290A2072616D28257010
:1017C000202564290A2073686172656428257020C9
:1017D0002564290A2064756D7028257020256429E8
:1017E0000A0000005B495D25733A206970635F6DF4
:1017F000617020696E666F726D6174696F6E0A2028
:10180000697063282570202564290A206461746149
:101810005F633261282570202564290A2064617481
:10182000615F613263282570202564290A2065766E
:10183000745F633261282570202564290A2065764B
:10184000745F613263282570202564290A206C6F3B
:1018500067282570202564290A20706572736973D2
:1018600074627566282570202564290A000000002E
:101870005B495D25733A206970635F6D6170206418
:101880006174615F63683A73697A653A2564206FB1
:101890006E202564206368616E6E656C2E2065760F
:1018A000745F63683A25640A000000006970635F32
:1018B00077726974655F6461746100005B495D25DE
:1018C000733A2025733A2069732066756C6C0A00A0
:1018D0005B495D25733A2025733A20696E76616C09
:1018E00069642073697A653A25640A005B495D255D
:1018F000733A2025733A206661696C206279206111
:1019000064645F6576740A005B495D25733A20253F
:10191000733A206572726F723A2065713A25642CB1
:101920002064713A25640A005B495D25733A2061A1
:1019300032633A2065713A25642064713A25642047
:1019400066756C6C3A256420656D7074793A25640F
:101950000A0000005B495D25733A206332613A203A
:1019600065713A25642064713A25642066756C6C53
:101970003A256420656D7074793A25640A00000088
:101980005B495D25733A20746F6B656E3A25642C54
:101990002065713A25642C2064713A25642C2073EB
:1019A000697A653A25640A006970635F696E6974D3
:1019B000000000005B455D25733A206970635F6D30
:1019C0006170206973204E554C4C2E0A00000000B7
:1019D0006970635F6164645F657674005B455D2573
:1019E000733A2025733A20696E76616C69642069C8
:1019F00070635F6576742C206F776E65723A25642C
:101A00000A0000005B455D25733A20696E76616CC3
:101A10006964206375725F6576740A005B455D25B5
:101A2000733A2025733A206972713A2564207065F3
:101A30006E64696E673A307825782D3E3078257867
:101A40000A0000005B495D25733A2025733A207037
:101A5000656E64696E672069727120776169743A96
:101A60002070656E643A25642069727120256420B7
:101A7000647572696E672025642074696D65730AE8
:101A8000000000005B455D25733A2025733A20660F
:101A900061696C20746F20616464206576742062D3
:101AA000792070656E64696E673A307825780A002F
:101AB0005B495D25733A2025733A206576742025AD
:101AC0006420647572696E67202564206D732069D7
:101AD000732066756C6C0A005B455D25733A2025A2
:101AE000733A206661696C20746F206164642065BC
:101AF00076742062792066756C6C0A005B495D25FE
:101B0000733A20657674282570292D25733A20654F
:101B1000713A25642064713A25642066756C6C3ACC
:101B20002564206972713A25640A00005B495D25CD
:101B3000733A206576742564286576743A25642C9A
:101B40006972713A25642C663A2564290A000000FE
:101B50006970635F64756D70000000005B495D250E
:101B6000733A2025733A20613278206576656E7469
:101B70000A0000005B495D25733A2025733A206313
:101B80003261206576656E740A0000005B495D2550
:101B9000733A2025733A2064617461206275666629
:101BA00065720A005B495D25733A2025733A206C03
:101BB0006F67206275666665720A000001F05CBDA1
:101BC00080B50F280BDB23220FF240010FF230000B
:101BD000F9F770FC0020C046C046002002BDBDE8F9
:101BE000024001F089BE0F2801DB00207047102958
:101BF00001D30020704701F0C5BE01F000BF000016
:101C00005B455D25732C2025640A0000443A5C572F
